:020000040800F2
:10000000F0FF0010458C06081DF20008CDCC040856
:10001000E58C0608E58C0608E58C06080000000063
:1000200000000000000000000000000019F20008BD
:1000300015F200080000000011F20008999304086E
:10004000E58C0608E58C0608E58C0608E58C0608B4
:10005000E58C0608E58C060841DC04086DDD040823
:1000600031DD0408F5DC0408B9DC040885710608F4
:100070007571060865710608557106084171060814
:100080002D71060819710608E58C0608E58C06082E
:10009000E58C0608E58C0608E58C06087DDC04087E
:1000A000A97E0408297F0408997E04084D7F04086E
:1000B0001D7F04080D7F0408FD7E0408897A060868
:1000C000917A06087D7A0608857A0608E58C060886
:1000D000E58C0608A9970408ED96040831960408F3
:1000E00005DC0408E58C060849090108897E040836
:1000F000B97E0408797E0408DD7E040805710608CF
:10010000E58C06081D3D0608ED7E0408E58C060812
:1001100075950408B994040811020408FD01040847
:10012000F1700608DD700608C9700608B57006088B
:10013000A1700608E58C0608E58C0608E58C060823
:10014000E58C0608E58C0608E58C0608ADEB000892
:100150008D7006087970060865700608FD9304081E
:10016000717A0608797A0608E58C0608E58C060897
:10017000E58C0608E58C0608E58C0608E58C060883
:08018000E58C0608E58C060879
:08018800F487060001000000ED
:100190000E0201000200000040600020A06000206C
:1001A00000000000E809000814020100050000003A
:1001B000203E0020A460002000000000EA090008A2
:1001C0001302010004000000AC240020AC600020F9
:1001D00000000000F00900080D1001007000000090
:1001E000E45E0020B06000200000000061F403081D
:1001F0000400080080000000245E00202061002030
:1002000000000000000000000902010001000000E1
:10021000CC5D0020A061002000000000F40900086F
:10022000FD01010024000000845D0020A461002085
:10023000000000005F640408FB01010001000000F1
:10024000405D0020C861002000000000B97C050866
:10025000FC010100090000000C5C0020CC610020C2
:1002600000000000C17C0508F70101000600000045
:10027000005C0020D861002000000000F6090008A2
:10028000F901010004000000FC5B0020E061002097
:100290000000000009650408160215003F00000078
:1002A00040310020E4610020000000005D7C050872
:1002B0003400010010000000F05A002024620020E9
:1002C00000000000F594020811020100080000007F
:1002D000C85A00203462002000000000FC09000819
:1002E0001212010004000000C05A00203C620020ED
:1002F00000000000040A000818200100320000007D
:100300008C5A00204062002000000000458505084E
:100310001220010011000000AC590020746200207E
:1003200000000000080A0008000201000B000000A5
:10033000E856002088620020000000000000000055
:10034000FF1101000600000090560020946200207A
:10035000000000004D7C0508081203000F0000009B
:100360009C5600209C62002000000000617C050873
:10037000FA0101000300000088500020AC62002058
:1003800000000000E97C05080A8001002800000048
:1003900050500020B0620020000000003D14020810
:1003A000061001001C00000024310020D86200204B
:1003B00000000000457D0508020201000300000066
:1003C00098280020F46200200000000000000000D7
:1003D0000C0201000400000078280020F8620020D0
:1003E00000000000117D0508110001000C00000054
:1003F000A6440020FC62002000000000C1EF0308BA
:10040000FE010100140000004C3F002008630020A2
:1004100000000000ED7B0508FD07010076000000EC
:1004200048B20020C0B2002000000000957801080A
:10043000261001000E00000048B3002038B3002051
:10044000000000001D1C01080B3001001A00000014
:1004500000AD002088B30020000000001C0A000846
:100460001F300100240000003CAC0020A4B3002099
:1004700000000000380A0008050201000400000026
:10048000CCAE0020C8B30020000000005C0A0008C9
:10049000030101000A00000080AC0020CCB3002062
:1004A00000000000AD160108220201001C0100003E
:1004B00024CB0020DCCD002000000000FD840508D6
:1004C0000C200600CC000000A0C90020F8CE0020BF
:1004D000000000002DEE0308010201000B000000E7
:1004E00044C90020C4CF002000000000017D0508A1
:1004F0001B0201001000000018C90020D0CF00200E
:1005000000000000317D05081B1001000C000000F8
:10051000CCB50020E0CF002000000000097F0108DA
:1005200021020100F00000004CB40020ECCF0020BC
:1005300000000000D9A001082312010010000000F3
:1005400020C60020DCD0002000000000600A000867
:10055000371001002E00000088C80020ECD00020D9
:1005600000000000700A00081610010006000000DC
:1005700018C600201CD10020000000009E0A0008C0
:100580002F10010022000000B8CD002024D100204F
:1005900000000000A40A00081E000100090000007D
:1005A00040C5002048D1002000000000C60A000815
:1005B000051001000600000084C5002054D1002071
:1005C00000000000D00A0008F5810100680000006A
:1005D000DCB300205CD10020000000005591010830
:1005E0002320010010000000C4C50020C4D1002059
:1005F0000000000051150208F62101000C00000067
:1006000044DD0020FCDE002000000000D80A0008C5
:100610001C0202001C000000E8DC00204CDF00206F
:1006200000000000318605082820010018000000A5
:1006300004DD002068DF002000000000993002087F
:100640000412010002000000BCDE002080DF002058
:1006500000000000E40A00080F0201000100000091
:10066000B8DE002084DF002000000000E60A000859
:100670001400010004000000E0DC002088DF0020FE
:1006800000000000E80A0008012001000C00000042
:10069000E4D400208CDF002000000000EC0A0008F9
:1006A0000EF003009E010000CCD2002098DF002055
:1006B000000000003D950208130001000400000046
:1006C000BCD8002038E1002000000000F80A000833
:1006D000010101000400000018D200203CE10020CC
:1006E0000000000000000000000101000400000004
:1006F00010D2002040E1002000000000FC0A0008A9
:1007000002010100030000000CD2002044E100209F
:100710000000000069EE0308190001000500000058
:1007200030EB002014EC002000000000000B00085B
:100730001A0001000E000000B8EA00201CEC0020A6
:1007400000000000060B0008203201000A00000033
:1007500084E900202CEC002000000000199502081C
:1007600015001000700000001CE7002038EC00208D
:1007700000000000000000002A00080060000000E7
:1007800078EB0020A8EC002000000000CD940208C7
:100790002C0004001000000018ED002008ED0020DF
:1007A00000000000A59202082B00120024000000A7
:1007B0004CED002028ED0020000000007992020896
:1007C0002920140078000000BCE4002070ED002017
:1007D00000000000000000001902010010000000ED
:1007E000F0E30020E8ED002000000000F17C0508A7
:1007F000030001000100000094F10020C4F100207A
:100800000000000000000000031201003D00000095
:100810003CF10020C8F1002000000000140B00088B
:1008200025201E002C010000A0EE002008F2002070
:100830000000000000000000101001000200000095
:1008400034EE002034F3002000000000520B0008BA
:10085000F8210100060000007CEE002038F30020A3
:1008600000000000540B0008020001000C00000012
:10087000D0FB002064FC002000000000000000000D
:10088000290201004000000020F6002070FC00203A
:10089000000000005A0B00080A02010014000000CA
:1008A00090F50020D0FC002000000000F9ED0308C6
:1008B0002802040004000000F0000120CC02012006
:1008C000000000002D7D0508270204000400000040
:1008D000EC000120D002012000000000217D05086D
:1008E0001F0208001000000048FE0020D402012072
:1008F00000000000057C05081A0201003C00000011
:100900000CFE0020E402012000000000B58505086F
:10091000381001000100000004FD00202003012028
:10092000000000009A0B00082700010004000000EE
:10093000E0030120E8040120000000009C0B0008F7
:100940000B1201003C000000A0060120001801204D
:1009500000000000A00B00080D12010014000000B0
:10096000541301203C18012000000000DC0B00089B
:100970000702010002000000E817012050180120C2
:1009800000000000F00B00081D020200060000003D
:10099000B0170120541801200000000000000000E2
:1009A000060203000C000000BC1701205C2101209E
:1009B00000000000BD8605083900010005000000A8
:1009C000C81701206821012000000000D97C05081B
:1009D000100201000100000008550120045501200B
:0809E00000000000F20B00080A
:1009E8000000000000FF00000000010000000000FF
:1009F800010000000000000001010101FFFFFFFFEE
:100A080000000001000005533430350000000002EA
:100A180000000000AE014A015E012C0164000200E2
:100A2800000001000A019A01001E0A0000020000ED
:100A380000000000000100000005000001020300A2
:100A4800000000000000000000000000000000009E
:100A58000080070000000000000000000000000007
:100A6800000000000000000020003200C800D0078D
:100A780096001400320028004C044006000550007F
:100A880014000F00080064000100010005000A00BE
:100A98000000F4019600C4090000190000000000DD
:100AA800000000000000000000000000000000003E
:100AB8000000000000000000000000000000000529
:100AC80001000000000000002000030100000000F9
:100AD8000000000001000000020200000000000009
:100AE80003000023E8036400040A000114001E0048
:100AF80000204030900100000000280100007E0521
:100B0800EA05B4053200E803D00700000000000041
:100B180000000000000000000000000000000000CD
:100B280000000000000000000000000000000000BD
:100B380000000000000000000000000000000000AD
:100B48000000000000000000010000050101F401A0
:100B58001400000000000000000000000000000079
:100B6800000000000000000000000000000000007D
:100B7800000000000000000000000000000000006D
:100B8800000000000000000000000000000000005D
:100B9800000000002003000000000000000000002A
:100BA800000000000000000000000000000000003D
:100BB800000000000000000000000000000000002D
:100BC800000000000000000000000000000000001D
:100BD800010000000000000000000000000000000C
:0B0BE8000000000000000000003C00C6
:100BF3000403090412010002EF0201408304563288
:100C0300000201020301000012010002020200407F
:100C1300830440570002010203010800FFFFFFFFA6
:100C2300006002401060024000000000000000006D
:100C3300000B0000000000000000000000000000A6
:100C43000060024028600240010000000000000034
:100C5300060C00000000000000000000000000007F
:100C630000600240406002400200000000000000FB
:100C7300100D000000000000000000000000000054
:100C830000600240586002400300000000000000C2
:100C9300160E00000000000000000000000000002D
:100CA3000060024070600240040000000000000089
:100CB300200F000000000000000000000000000002
:100CC3000060024088600240050000000000000050
:100CD30026100000000000000000000000000000DB
:100CE30000600240A0600240060000000000000017
:100CF30030110000000000000000000000000000B0
:100D030000600240B86002400700000000000000DD
:100D1300362F00000000000000000000000000006B
:100D23000064024010640240000000000000000064
:100D33000038000000000000000000000000000078
:100D4300006402402864024001000000000000002B
:100D53000639000000000000000000000000000051
:100D630000640240406402400200000000000000F2
:100D7300103A000000000000000000000000000026
:100D830000640240586402400300000000000000B9
:100D9300163B0000000000000000000000000000FF
:100DA3000064024070640240040000000000000080
:100DB300203C0000000000000000000000000000D4
:100DC3000064024088640240050000000000000047
:100DD30026440000000000000000000000000000A6
:100DE30000640240A064024006000000000000000E
:100DF300304500000000000000000000000000007B
:100E030000640240B86402400700000000000000D4
:100E13003646000000000000000000000000000053
:100E23007D00000015830008118300080D8300086E
:100E330001830008FD820008098300080583000878
:100E43000000000059910008FDAD0008D190000892
:100E53003DAF0008319200088583000871830008C4
:100E6300558300087DA70008558A00085D94000893
:100E7300D19400085195000801970008390F010823
:100E83005D8300084D830008010000000000803FDF
:100E9300D1380108D53D01084D390108D50F0108A6
:100EA300B9110108E50F010801100108AD0F010890
:100EB3009D0F01080000000000000000090220004F
:100EC300010104C0320904000002080650050705A9
:100ED300810240000007050102400000090264008E
:100EE300030100C0320904000001030000000921CE
:100EF300110100012226000705830308000A080BDD
:100F030001020202010009040100010202010005BD
:100F13002400100105240100020424020205240612
:100F23000102070582030800FF09040200020A0008
:100F33000000070501024000000705810240000090
:100F430009024300020100C0320904000001020249
:100F530001000524001001052401000104240202FC
:100F63000524060001070582030800FF09040100A8
:100F7300020A000000070501024000000705810284
:100F830040000000FF00000000FF00000000000020
:100F93000000AA550701000001AA55050100000839
:100FA30088C40608FF1FFF1F05010905A101A10051
:100FB300050109300931093209330935093409407A
:100FC30009381581257F750895088102C0C0000086
:100FD30009022200010100E03209040000010301BB
:100FE30002000921110100012226000705830308DD
:100FF300000A0000000000000102030401020304D0
:10100300060708092D202D2D202D2D2D2D202D2DCA
:101013002D2D000000000000000000000000000073
:10102300000000AA550B010000AA5505010000AA03
:10103300550902000000AA5503009F0001000000AB
:10104300C012000080B300200000000058B300204D
:101053000000000001000000186D0708206D07085C
:1010630000000000D9EE0308A08601000400000080
:10107300000000000000000000000000000000006D
:10108300000000000000000000000000000000005D
:101093000000000000000000186D0708286D070815
:1010A3000000000091740408E8030000040000003D
:1010B300000000000000000000000000000000002D
:1010C300000000000000000000000000000000001D
:1010D3000000000000000000306D07080000000061
:1010E30000000000296003087D000000FF000000ED
:1010F30000000000000000000000000000000000ED
:1011030000000000000000000000000000000000DC
:10111300000000000000000018F3070800000000B2
:1011230000000000917003087D000000FF00000034
:1011330000000000000000000000000000000000AC
:10114300000000000000000000000000000000009C
:101153000000000000000000DC8107080000000020
:1011630000000000D5B603087D000000FF0000006A
:10117300000000000000000000000000000000006C
:10118300000000000000000000000000000000005C
:101193000000000000000000386D07080000000098
:1011A30000000000F56A0408E803000003000000E3
:1011B300000000000000000000000000000000002C
:1011C300000000000000000000000000000000001C
:1011D30000000000000000003C6D07080000000054
:1011E300000000008D240308102700000300000006
:1011F30000000000000000000000000000000000EC
:1012030000000000000000000000000000000000DB
:1012130000000000000000002CEF070800000000A1
:10122300858E020881CD04085F760000050000006A
:1012330000000000000000000000000000000000AB
:10124300000000000000000000000000000000009B
:101253000000000000000000BCF2070800000000CE
:1012630000000000A1E904081027000001000000AD
:10127300000000000000000000000000000000006B
:10128300000000000000000000000000000000005B
:101293000000000000000000486D07080000000087
:1012A3000000000029610408E803000005000000B5
:1012B300000000000000000000000000000000002B
:1012C300000000000000000000000000000000001B
:1012D3000000000000000000546D0708000000003B
:1012E30000000000C9F20308204E000003000000C4
:1012F30000000000000000000000000000000000EB
:1013030000000000000000000000000000000000DA
:101313000000000000000000646D070800000000EA
:1013230000000000B1F00308204E0000030000009D
:1013330000000000000000000000000000000000AA
:10134300000000000000000000000000000000009A
:101353000000000000000000746D0708000000009A
:101363000000000009710408400D030003000000A1
:10137300000000000000000000000000000000006A
:10138300000000000000000000000000000000005A
:101393000000000000000000846D0708000000004A
:1013A3000000000069290408102700000100000064
:1013B300000000000000000000000000000000002A
:1013C300000000000000000000000000000000001A
:1013D30000000000000000008C6D07080000000002
:1013E300000000006DAD010810270000030000009D
:1013F30000000000000000000000000000000000EA
:1014030000000000000000000000000000000000D9
:101413000000000000000000906D070800000000BD
:101423000000000091700208A08601000100000086
:1014330000000000000000000000000000000000A9
:101443000000000000000000000000000000000099
:101453000000000000000000986D07080000000075
:10146300000000007569040850C30000010000007B
:101473000000000000000000000000000000000069
:101483000000000000000000000000000000000059
:101493000000000000000000A06D0708000000002D
:1014A300000000000D1C0108A086010000000000E0
:1014B3000000000000000000000000000000000029
:1014C3000000000000000000000000000000000019
:1014D3000000000000000000AC6D070800000000E1
:1014E300000000005D660408A86100000100000020
:1014F30000000000000000000000000000000000E9
:1015030000000000000000000000000000000000D8
:101513000000000000000000B86D07080000000094
:1015230000000000E9060208A08601000100000097
:1015330000000000000000000000000000000000A8
:101543000000000000000000000000000000000098
:101553000000000000000000C46D07080000000048
:1015630000000000519C0408A00F000001000000CF
:101573000000000000000000000000000000000068
:101583000000000000000000000000000000000058
:101593000000000000000000D06D070800000000FC
:1015A30000000000E5010208102700000100000010
:1015B3000000000000000000000000000000000028
:1015C3000000000000000000000000000000000018
:1015D3000000000000000000DC6D070800000000B0
:1015E3000000000011EF0308A00F0000010000003D
:1015F30000000000000000000000000000000000E8
:1016030000000000000000000000000000000000D7
:101613000000000000000000E86D07080000000063
:10162300000000006DDC01081A4100000100000009
:1016330000000000000000000000000000000000A7
:101643000000000000000000000000000000000097
:101653000000000000000000EC6D0708000000001F
:1016630000000000E516010810270000010000003B
:101673000000000000000000000000000000000067
:101683000000000000000000000000000000000057
:101693000000000000000000F86D070800000000D3
:1016A30000000000AD4B020850C300000100000021
:1016B3000000000000000000000000000000000027
:1016C3000000000000000000000000000000000017
:1016D3000000000000000000FC6D0708000000008F
:1016E3000000000035200108400D03000000000049
:1016F30000000000000000000000000000000000E7
:1017030000000000000000000000000000000000D6
:101713000000000000000000046E07080000000045
:1017230000000000E1EF0308400D0300000000008B
:1017330000000000000000000000000000000000A6
:101743000000000000000000000000000000000096
:1017530000000000000000000C6E070800000000FD
:1017630000000000D1EA010850C30000030000009C
:101773000000000000000000000000000000000066
:101783000000000000000000000000000000000056
:101793000000000000000000186E070800000000B1
:1017A300000000008106040840420F000000000012
:1017B3000000000000000000000000000000000026
:1017C3000000000000000000000000000000000016
:1017D3000000000000000000246E07080000000065
:1017E3000000000085F7030850C30000000000005C
:1017F30000000000000000000000000000000000E6
:1018030000000000000000000000000000000000D5
:1018130000000000000000000100000000000100C3
:10182300E0010000FFFFFFFF01007EFFFFFFFFFF5E
:101833000800000042570200000001064257020060
:101843000000010601FFFF00FFFFFFFF0101010090
:10185300550A02080000000000000000C0CE060880
:101863008CD60020E0D60020C9250208F123020807
:101873000000000028E706087DF9010800000000C9
:10188300000000008CE6060869260208000000003C
:101893000000000044E6060800000000000000000D
:1018A30000000000F4E4060800000000000000004F
:1018B30000000000ACE50608000000000000000086
:1018C3000000000058E506080000000000000000CA
:1018D300CD22020881D80020D601FF2D202D2D20F6
:1018E3002D2D2D2D202D2D2D00000000000000009A
:1018F300000000000000000000000000FFFFFFFFE9
:1019030059290208000000000000000084E40608D2
:1019130001000000FA0000000100000001000000C7
:10192300010000000001010100000000DED40020DE
:101933000000F40101000000DCD400200000F401E9
:1019430001000000DAD400200000F40101000000CF
:10195300D8D400200000F40101000000D6D40020F8
:101963000000F40101000000D4D400200000F401C1
:1019730001000000D2D400200000F40101000000A7
:101983008D120208511202080000000004D106085B
:10199300C2D4002005320100D0D400206400F40139
:1019A30001000000CED400206400C409010000003F
:1019B300C0D40020E803D00701000000BED40020FB
:1019C300E803D00701000000BCD40020E803D007DF
:1019D30001000000BAD400201E00B80B0100000073
:1019E300C8D4002005000F0001000000CAD4002065
:1019F30003000A0001000000B8D400201E00F40117
:101A030001000000CCD400200200000090D10608A1
:101A1300B6D400201400640001000000C4D40020E8
:101A23003200E80301000000B4D400200000C80025
:101A3300010000008DD4002000C801008CD40020D8
:101A4300005001008BD40020005A010089D40020EB
:101A5300020000009CD10608247907082C790708A6
:101A63007A5F00200100C40900000000785F0020B5
:101A73000100C40900000000765F00200100C409D2
:101A830000000000745F00200100C4090000000092
:101A9300705F00200100C40900000000725F002095
:101AA3000100C409000000006E5F00200100C409AA
:101AB300000000006C5F00200100C409000000006A
:101AC30037D2002000C8010036D2002000C8010030
:101AD30034D200200000FFFF0A00000032D20020B1
:101AE3000100C8000100000030D200203200307530
:101AF300320000002ED20020058205002CD20020E7
:101B030005002C01050000002AD20020055A05001B
:101B130027D2002000FF010029D20020020000008C
:101B2300F00F002025D2002003000000A8C60608FD
:101B330026D2002000FF010028D20020020000006E
:101B4300F00F002024D2002003000000A8C60608DE
:101B5300E11102087111020800000000A8D1060873
:101B6300F4D40020EE02CA0801000000F2D40020E1
:101B730000C8010064000000F1D4002000C8010087
:101B830064000000F0D4002002000000B4D2060874
:101B93001ED2002080C1803E050000001CD2002020
:101BA30080C1803E0500000016D2002080C1803E27
:101BB3000500000014D2002080C1803E0500000013
:101BC3000FD2002000FF01000AD200206400F401BC
:101BD3000100000008D2002004000000C0D2060863
:101BE30007D2002002000000D4D20608BDD2002094
:101BF3000D000000E0D20608BAD200200064010004
:101C0300B8D20020320010270A000000B6D200200C
:101C13000D000000E0D20608B5D200200D00000040
:101C2300E0D20608B4D200200200000018D3060850
:101C330000000000000000000000000024D306089C
:101C4300FAD400203E0000005CD30608F8D400203C
:101C53000100FF7F01000000F7D400200200000014
:101C630058D40608BFD200200300000068D4060839
:101C7300BED200200300000068D406087AD40020F6
:101C8300000A010078D400200000E80301000000EE
:101C930076D400200000E8030100000074D4002083
:101CA3000000E8030100000072D400200000E803F4
:101CB300010000006AD400200000E80301000000D6
:101CC30070D400200000E803010000006ED400205F
:101CD3000000E803010000006CD4002000140100A0
:101CE30088D400200200000078D4060886D400209F
:101CF3000000F4010100000084D400200000F4017E
:101D03000100000082D400200000F4010100000063
:101D130080D400200000F401010000007ED40020E4
:101D23000000A00F010000007CD400200000A00FE1
:101D330001000000A1D4002019640100A0D40020F8
:101D43000200000084D406089ED40020E803D007D4
:101D53000A0000009CD40020006401000A00000077
:101D630091D400200064010090D40020006401009D
:101D730098D40020006401000A00000097D40020DA
:101D8300006401000A00000096D4002000640100F2
:101D93000A0000009BD4002000FF01000A0000009D
:101DA3009AD4002000FF01000A00000099D400200B
:101DB30000FF01000A00000095D4002001FF01008C
:101DC3000A00000094D4002001FF01000A00000073
:101DD30093D4002001FF01000A000000C8D20020B4
:101DE3000000F40101000000C6D200200000A00F93
:101DF30001000000C4D200200000A00F0100000079
:101E0300C2D200200000A00F01000000C0D20020B9
:101E13000000A00F01000000D1D8002000C801007D
:101E2300D0D8002000640100CFD800200064010056
:101E3300CED8002000640100CDD80020006401004A
:101E4300CCD80020FF080100CBD80020016401009A
:101E5300D91002089D1002080000000090D4060863
:101E6300D4D8002001320100D3D8002001000000A3
:101E730000D50608D2D800200400000008D50608C3
:101E8300CAD8002000640100C8D800201400E80369
:101E930001000000C6D80020E80330750A000000E6
:101EA300C4D8002000C80100C3D8002000C8010026
:101EB300C2D8002000C80100C1D8002000320100B0
:101EC300D6D80020004B0100D5D800200400000024
:101ED3001CD50608C0D80020006401000A000000D9
:101EE300E4D800200000D00701000000DFD8002064
:101EF30000C80100DED8002000C80100DDD80020A2
:101F030000C80100E2D800200000D0070100000053
:101F1300DCD8002000C80100DBD8002000C8010085
:101F2300DAD8002000C80100E0D800200000D00764
:101F330001000000D9D8002000C80100D8D8002033
:101F430000C80100D7D8002000C80100910E020884
:101F5300790E02080000000030D50608B1D2002037
:101F6300005A0100B0D2002000C80100AED2002008
:101F7300E803D0070100000000000000000000009B
:101F83000D230208CCD5060853544D333246343062
:101F93003500000023D200200003010022D20020DC
:101FA30000030100B50D0208690D020800000000DE
:101FB30020D60608290D0208E10C020800000000E3
:101FC300BCD60608010E02083D29020800000000E5
:101FD3003CD7060820D20020010301006913020840
:101FE3003D1302080000000094DA06086D0C020895
:101FF300290C02080000000004DB0608A10E0208F9
:10200300912A020800000000A0DB0608592E0208EE
:10201300951302080000000048DC0608F10E0208D0
:102023000000000000000000D4DC0608CD0F020809
:10203300750F02080000000038DD06086110020871
:102043002510020800000000E0DD0608598B020895
:1020530015110208000000006CDE0608B3D400204E
:1020630001060100390F0208050F020800000000F5
:1020730068DF06088D8A02085D2B02080000000055
:10208300D8DF0608A18B0208252C020800000000F7
:1020930028E10608B2D4002001030100490E02081A
:1020A300190E020800000000FCE10608F98B020883
:1020B300000000000000000060E20608B10C020806
:1020C3002529020800000000E0E2060800000000E5
:1020D30000000000000000006CE30608491102083C
:1020E3009D2C020800000000DCE30608000000004D
:1020F3000000000000000000F4E5060878AE0020B0
:102103009CFF2C0100000000F8D90020E0150C17FB
:10211300000000004CCD0020020000002CE6060861
:1021230003D200200200000038E60608FED100209A
:1021330088136F170100000000D2002088136F1767
:1021430000000000BE5F002000000000000000004F
:10215300BC5F00200000000000000000BA5F002008
:102163000000000000000000B85F00200000000035
:1021730000000000B65F0020000000000000000027
:10218300B45F00200000000000000000D80500201C
:102193000000000000000000D4D100200300000074
:1021A3008CE70608FCD1002088136F17010000009C
:1021B300C2AE002088136F17000000000D0B020849
:1021C30000000000000000009CE70608C5D70020BF
:1021D30001000000F0E70608C4AE00200100000083
:1021E300FCE70608BAAE00200200000004E8060877
:1021F30000000000000000000000000010E80608D6
:10220300F90A02080000000000000000ACE806081C
:1022130000000000000000000000000000E90608C4
:1022230000000000000000000000000070E9060844
:1022330002D2002002000000A8E90608BEAE00207A
:10224300E0150C170000000001010000FFFFFFFF75
:102253000000803F000000000000000000000000BC
:10226300000000000000000000000000000000006B
:1022730000000000000000000000803F000000009C
:1022830000000000000000000000803F000000008C
:1022930000000000000000000000803F000000007C
:1022A3000000000000000000010000000000FA43ED
:1022B3000000FA430000803F792B0408000000006F
:1022C3000000000000000000FFFFFFFFFF00000010
:1022D30000000000C0FC0020080000000000000017
:1022E300B0FC00200800000029380108C9100108CB
:1022F300C137010800000000990F0108A940010837
:10230300113701085D3301080000000000000000E0
:10231300590F010825830008198300085D90000800
:102323007990000841900008259000080990000862
:10233300E1370108A5100108153701080000000066
:10234300710F010861330108E5360108BD32010848
:102353000000000000000000650F0108685E0C002B
:1023630002010000A00F0000B80B000002FFFF01F4
:10237300FFFF000020EF0708000008020503030029
:102383000000000028EF070801000802050403000D
:1023930000000000EC9607080200FE010110030094
:1023A300000000008C7C07080300140200030000F7
:1023B3000000000030EF070804001F0202000800BD
:1023C3000000000038EF070805001F0202010800A3
:1023D30000000000FFFFFFFF1A03000000000000E1
:1023E30000000000000000000000000000000000EA
:1023F3000000000004030904120100020000004071
:10240300830420570002010203010B01E58D050837
:10241300B98D05085D8D0508F97D0508798D0508D9
:102423001D8D0508F57D0508C41A0020D58E050805
:10243300F58E0508C58E0508D97D0508818E05082A
:10244300398E0508C97D0508A01A0020F9860508FC
:10245300E17D0508DD7D0508D57D05084188050872
:10246300D17D0508CD7D0508CC3F0708454001080F
:1024730085100108253F010800000000000000004E
:10248300BD360108CD350108000000000000000042
:10249300000000004D0F0108817E0508757E0508C8
:1024A300458F0508618F05082D7E0508298F0508CE
:1024B3000D8F0508FFFFFFFF0100000050C3000060
:1024C300010100001F0000001C0000001F000000AD
:1024D3001E0000001F0000001E0000001F0000007F
:1024E3001F0000001E0000001F0000001E0000006F
:1024F3001F0000000068214C012500006C3C070808
:102503006C490708E81A0020008002021F0000003F
:1025130053544D202020202050726F647574202066
:102523002020202020202020302E30310080020265
:102533001F00000053544D202020202050726F6450
:10254300757420202020202020202020302E3031A0
:10255300AB160108A71601089F1601088914010884
:102563009D1F0108C91F0108F91E010895160108DE
:1025730085160108751601086516010881140108FE
:10258300FF010000F4010000FF000000000004014F
:10259300000000000000000210000000070000001F
:1025A3000000000000000000010203040607080900
:1025B30001000000501B002000000000000000008C
:1025C3000000000000000000000000000000000008
:1025D30000000000000000000000000000000000F8
:1025E30000000000000000000000000000000000E8
:1025F30000000000000000000000000000000000D8
:1026030000000000000000000000000000000000C7
:082613000000000000000000BF
:0828000000C00F0800001008E1
:10800000F0B401292A4C2B4D23684FF0000694BF91
:1080100000270127EE626662A6626763676B47EA24
:1080200042076763EE63EC6B002A38D144F4957421
:10803000EC631C6824F001041C601C68E407FCD499
:10804000490289085960D8601968EAB921F04001ED
:10805000196019498B421DD018494FF47410C8603B
:10806000196841F01E011960596941F08001596198
:10807000196841F00101196022B90E4AD36A43F030
:108080000803D362F0BC704741F0400119600A490F
:108090008B42E1D14FF0746041F8500CE0E744F0BE
:1080A0001A04EC63EC6A44F00804EC62C1E700BF18
:1080B000B01B0020002C01405864024000640240C4
:1080C0001148002302461178032902F1060216D056
:1080D0000133062BF7D10D4AD36D052B0ED0591C59
:1080E00003EB4303D16500EB4303032040F2EB3184
:1080F00040F2FF32187059809A807047704703EB46
:10810000430300EB4303F0E7E81B0020B01B002013
:1081100070B4C3080D4CE25C00F00706B24004EBFB
:10812000D004D2B20020C6F108038B4228BF0B4610
:10813000C3F108052A419840C91A40EA02004FF0ED
:10814000000614F8012FEED170BC7047501C0020BF
:10815000084AD2E9343199420AD0D118013391F852
:10816000D8100170C3F30A03C2F8D0300120704761
:1081700000207047B01B0020064AD2F8D838D2F849
:10818000DC28934294BF4FF400600020013B9B1A0F
:1081900018447047B01B0020012380F8513070470D
:1081A00007B501A8FFF7D4FF0028FAD09DF8040016
:1081B00003B05DF804FB044BD3E93403984288BF55
:1081C00003F50063181A7047B01B002001207047A8
:1081D000024BC3F8E028C3F8E4187047B01B002036
:1081E000024BC3F8E828C3F8EC187047B01B002016
:1081F0007047704730B4134DD5E934239A4286BF97
:1082000003F50064A21A9A1A0A44B2F5006F13D853
:10821000A9B101444A1E013810F8014FE918824201
:1082200003F1010381F8D840C3F30A03F4D1C5F880
:10823000D430002030BC7047022030BC7047084664
:10824000F8E700BFB01B0020212838B50C4605D048
:1082500022282ED0202813D0002038BD0029FBD0A2
:10826000072AF9D11A4BD3F8F00893F8F41893F8C9
:10827000F52893F8F638206021716271A371EBE75D
:108280000029E9D0072AE7D1114DD5F8E4381BB110
:108290000968D5F8E0089847206821796279A379C0
:1082A000C5F8F00885F8F41885F8F52885F8F6384B
:1082B000D2E70029D0D0022ACED1054AD2F8EC3834
:1082C000002BC9D00988D2F8E8089847C4E700BF56
:1082D000B01B0020024B0020C3F8F808704700BF15
:1082E000B01B0020044B00200522C3F8F828C3F877
:1082F000EC08C3F8E4087047B01B0020704700BFCB
:10830000704700BF704700BF704700BF704700BF95
:10831000704700BF704700BF042301480B807047BF
:108320008801002010B4074A074B92F8FC08122479
:1083300003F114020C8001280CBF184610465DF8AA
:10834000044B7047B01B00208C0100200048704790
:10835000381C002000487047381C0020034B93F85D
:108360008400032894BF002001207047B01B002028
:10837000034B93F88400032894BF0020012070472A
:10838000B01B0020034B93F88400003818BF012075
:10839000704700BFB01B0020A0B182680D4B12B126
:1083A00007229A7070471978DA6003294FF00400A9
:1083B0000CBF80214FF48071C3E901111A611A7555
:1083C00098707047034B41F2D45101225A545A70AD
:1083D000704700BF1C9300200378022B10D0006967
:1083E00008B9012070470B4B1B78032B0EBF0A4BBB
:1083F00080B24FF6F773984294BF00200120704777
:10840000064A43681268B3EB422F2CBF01200020BC
:10841000704700BF1C930020F7FFFF0F5CA90020EE
:108420000378022B14D030B4104A4368006941F23B
:10843000386441F230611559515841F22C642B4097
:1084400012595B0A023801FB0030104430BC7047FF
:10845000064B426841F2246103F5B1505B58006855
:1084600000EB430000EB5220704700BF1C9300203C
:1084700008B5124BD3F8BC00828940F2E933028977
:10848000013B12F0020F9BB212D0FF23838140F216
:10849000E9330289013B12F0010F9BB202D08089BF
:1084A000C0B208BD002BF4D145F074FEC0B208BDC7
:1084B000002BE4D145F06EFEC0B2F8E7B01B0020FF
:1084C00070B505460E460924FFF7D2FFFF2803D1F9
:1084D000013CF9D1012070BDFE2801D0022070BD01
:1084E000064933462A46D1F8BC0000215EF084FEDE
:1084F000FFF7BEFFFFF7BCFF002070BDB01B0020E0
:1085000010B51D4C0023C4F88030FFF7B1FFD4F83C
:10851000BC00828940F2E9330289013B12F0020F6C
:108520009BB217D0FD23838140F2E9330289013BDE
:1085300012F0010F9BB212D08389FFF799FFFF2839
:1085400012D1FFF795FFFF280ED10423022084F8F3
:10855000843010BD002BDFD145F01CFEEDE7002B71
:10856000E4D145F017FEE8E7D4F800396367092342
:10857000002084F8843010BDB01B002070B582B09C
:1085800040F040060C0E05460A0A080C95238DF8AB
:1085900001408DF804108DF800608DF802008DF810
:1085A00003208DF805300824FFF762FFFF2802D072
:1085B000013CF9D125BB1A4BD3F8BC0006258389B1
:1085C0006E464FF47A734FF6FF713EB316F8012BE7
:1085D0000489013BA4079BB215D593B283814FF464
:1085E0007A730489E40703F1FF3211D5013D8289D2
:1085F000EBD10924FFF73CFFFF2802D1013CF9D160
:10860000FF2002B070BD8B42E2D145F0C3FDF0E720
:1086100093B28B42E5D145F0BDFDEAE7FF22D7E7F3
:10862000B01B00202DE9F041684C00234FF4F0729C
:108630002021064604F6081084F8043963F01FF977
:1086400004F6E8204FF4F072202163F018F994F852
:10865000C90C10B194F8CA2C1AB900252846BDE8F7
:10866000F08144F015F80746C4F8D40C44F0E4FA5D
:1086700005460028F1D00FB12323FB80092138469D
:1086800040F098F8D4F8D40C514F44F0F7FA94F82D
:10869000CA0C013840B245F0E7FE0223102184F8ED
:1086A000CC3CC4F8D00C5EF075FD798D494845F09E
:1086B00027FDD4F8D40C44F0DBFAFF218C205AF0CB
:1086C0009FFA8046D4F8D40C44F0D8FAD4F8D00CF1
:1086D00004215EF05FFDB8F11B0F05D0D4F8D40C77
:1086E000202140F067F8B8E7D4F8D43C012284F8A0
:1086F00004290BB12322DA80798D364845F000FD3C
:10870000D4F8D40C44F0B4FA40210A205AF078FA94
:10871000FF218A205AF074FAC0F38013D4F8D40CE5
:1087200084F8D83C44F0AAFAD4F8D00C04215EF0C6
:1087300031FD94F8C83C012B3FD0022B37D0CBB38E
:1087400094F8D93C182B08D194F8D82C7B8DA4F838
:10875000DC6CA4F8DE2CA4F8E03C798D1D4845F0D3
:10876000CFFC798D1B4845F0CBFCD4F8D40C44F0F9
:108770007FFA022100205AF043FAD4F8D40C44F0D6
:108780007DFA0421D4F8D00C5EF004FD94F8E92CB5
:1087900094F8EA3C94F8E81C84F8E41CC2F1200246
:1087A000C3F1100384F8EB2C84F8EC3C56E7082363
:1087B0007B85C5E710237B85C2E7002EF7D094F8B0
:1087C000D83C002B14BF08231023F1E7B01B002076
:1087D000880100207C2800202DE9F84F564B984254
:1087E00010D003F568530833984267D0534B0020EC
:1087F000A3F8480DA3F8540DC3F84C0DC3F8500D61
:10880000BDE8F88F4D4C4E4E02224FF0000BC4F8DD
:10881000F02C04F6F445D9464FF4007A4FF48078F2
:10882000F26A01275A455946BB4403D0D4F8640D77
:1088300053F014FC94F8682D85F82420D4F8640DC6
:10884000A5F804A04FF000724FF48031A960EA60EF
:10885000A5F8108085F81290A5F806802F7628627A
:10886000B72153F0F1FDD4F8F02C364B6F769345D9
:1088700045F8283BD4DB84F8569DD4F8F01CB4F8B6
:10888000F82CD4F8003DD4F8FC0CB4F8045DC4F81E
:108890006C3D12FB01F203FB01F3A4F8482DB4F880
:1088A000FA1C294AC4F84C0DC4F8503DA4F8545D94
:1088B000A4F84A1DC4F8442D0120A1E71F4C204E06
:1088C0000223C4F8F03C04F6F4454FF0000B4FF4DB
:1088D000806A4FF040094FF40068F26A01275A4558
:1088E0005946BB4403D0D4F8640D53F0B7FBD4F819
:1088F000641D94F8682D296285F824204FF4003116
:108900004FF00062C5E90212A5F804A0A5F8109086
:10891000A5F80680AF74FFF7D3FB28466F7653F0B7
:10892000E5FCD4F8F02C094B45F8283B9345D4DB03
:1089300084F8567DA1E700BF1971EF00B01B00203D
:108940008801002020B9060878B906084CB9060845
:10895000F8B51A4C94F8703D002BFBD159B3014483
:108960004E1E451ED4F8DC28D4F8D81815F8017F1F
:10897000531CC3F30A038B422CBF4FF4006000204A
:10898000C91A22440144012982F8747DC4F8DC38F4
:108990000FD1012040F05CFCD4F8D838D4F8DC18B2
:1089A0008B4294BF4FF4006200225B1A1344012BE8
:1089B000EFD0B542D6D10020F8BD00BFB01B0020DB
:1089C00010B5094CD4F8F838084611465BB1D4F814
:1089D000F838052B07D1002AD4F8003903DDFFF75A
:1089E000B7FFD4F8003910BDB01B002010B590F8C7
:1089F0005010002380F8503081B10B4CD4F8F82887
:108A000072B1D4F8F828052A0CD13C30D4F80039DA
:108A1000FFF79EFFD4F80039012010BD0120FCE7CC
:108A20001046FAE71846F8E7B01B0020002280F84D
:108A30005120DBE790F85020531C0244DBB280F851
:108A4000503082F83C1090F851200AB1132B00D915
:108A5000CCE770472DE9F04143794F4C002B14BF10
:108A60000122002284F8B02003D184F88430BDE8CC
:108A7000F08190F8018008F1FF3676B20546304665
:108A80000F4645F0F1FC0223C4F8BC0084F8B8306E
:108A90002B78002B5BD1ED78002D4CD14FF48071F9
:108AA000D4F8BC00C4F8C0505EF074FB4FF47A7088
:108AB00040F0CEFBD4F8C00044F0E0F8D4F8BC009D
:108AC0000A2683894FF6FF714FF47A73FF270289D4
:108AD000950719D587814FF47A730289D20703F17C
:108AE000FF3524D5013E8289F1D12C4B02899207B2
:108AF00013D5028912F080020FD1D4F8001984F83E
:108B0000782001236167B0E7013B9BB28B42DED145
:108B100045F040FBD4F8BC00E7E7013BE6D194F810
:108B2000782084F88430531C84F878309FE7ABB207
:108B30008B42D2D1ECE7284643F0AAFD054608B1A6
:108B40001E23C380092128463FF034FEA6E706EB2A
:108B500086063E44414696F90320002041F00AF87B
:108B6000064630B140685DF00BF8B36884F8CE304B
:108B700018B9002384F8C4308DE7094A431E02EB7C
:108B8000431317210022C4F8C8305DF00BF801230D
:108B900084F8C4307FE700BFB01B0020A18601002D
:108BA000B80100202DE9F04FCF4DDFF87083DFF8DA
:108BB000789384460F4616460FCD44462DED068B1E
:108BC0000FC40FCD0FC495E807008BB099F87E3421
:108BD000029684E80700CDE906C7042B00F25C8109
:108BE000DFE813F0BD015A0155010500CD019FEDED
:108BF000BF8ADFEDBF8ABF49C8F81C10BE49BF4B12
:108C0000BF4AC8F818100299002918BF134638EE59
:108C1000887AF5EE006A86EE87AAC8F82430B94F44
:108C2000B94B03930026DFEDB97A9FEDB99A28EE90
:108C3000278AF0EE679A079BB34200F02281039BDC
:108C400013F8014B039306F1010B5FFA8BF2002C32
:108C500000F09881DFF8D4C2002303E00133152B24
:108C600000F0908103EB43015D001CF80100A0427D
:108C7000F4D14944049291F89914002900F08A81B2
:108C800020463FF06DFB03680593824618463FF08F
:108C900053FB9AF805103FF083FB90F800C0BCF13D
:108CA000000F40F06F8109EB05002509013D049A92
:108CB00080F8D9240321052D80F8D814059B04F0F1
:108CC0000F0000F23781934C04EB450CBCF8B0C0A8
:108CD0004CFA00FE1EF0010E00F03E81012303FA63
:108CE00000F0013800EA0C00254404925FF032FEE7
:108CF00095F8BC50DFF838C2049A28440CEBC00544
:108D00000321A971EA715CF830007D6100F13F41F7
:108D100001F57E0104EB9124012394F8C4109AF824
:108D2000082001F01F044909032903FA04F300F0A5
:108D30000E81042900F00681022900F0FE80AB8834
:108D40000893B3FA83F3C3F11F03C3F3CC0100EB21
:108D5000810103F007030C6A9B000F259D4024EA64
:108D600005040C620C6A02FA03F323430B6202232C
:108D700008A909930BF0E0FCDAF80030029A002A07
:108D800000F0A280B9F87C2400EE102AB8EEC00AE8
:108D9000FCEEC07A17EE901A5F4A934200F0818091
:108DA000A2F5806293427CD002F58042934278D053
:108DB00002F58062934274D002F58062934270D0D3
:108DC000D9F8042850084FF6FF73B0FBF1F21A44AB
:108DD000120CB0FBF2F20298002865D0B2FBF1F160
:108DE00099F87E0404288BB263D007EE902AF8EE3F
:108DF000676A66EE887A29EE677A99F87F040699A1
:108E00000091A6EEA87A019051463846C7ED027A45
:108E100087ED037A36F0E4FE002E60DD7B68D8F83B
:108E2000382093425DD0012E59D0D8F8502093427B
:108E300057D0022E53D0D8F86820934251D0032E39
:108E40004DD0D8F8802093424BD0042E47D0D8F88C
:108E50009820934245D0052E41D0D8F8B0209342B7
:108E60003FD0062E3BD0D8F8C820D31A18BF012314
:108E70005E460122082E3B747A7407F118077FF4CE
:108E8000DAAE26480BB0BDEC068BBDE8F08F9FED47
:108E9000248AF0EE488AAEE69FED228AF0EE488AF8
:108EA000A9E6D9F804088EE799F87E040428194643
:108EB0009BD107EE901A07EE102AF8EE677AF8EECB
:108EC000476A67EEA97A96E7B0EE4A0A049360F023
:108ED00063FEFCEEC07A049B17EE901A5CE7012358
:108EE000C6E70023C4E700BFA4B90608ACC5A7378E
:108EF000ACC5A73685F00308F5640408D5E9030876
:108F0000E9640408480000102B3100206F12833AF6
:108F100000007A4420B90608000401401400001043
:108F2000282930386F120339A82C00204031002046
:108F3000AC310020C7F814C020E717494C6C23431C
:108F40004B64FCE614490C6B23430B63F7E61249B0
:108F50000C6C23430B64F2E6C7F814E00EE79FEDB8
:108F60000F8A0F4BC8F8183000230E4A06930123CE
:108F70000293C8F81C200C4BF0EE488A47E69FEDA0
:108F80000B8AEEE70A4A084BC8F81C20C8F82430C0
:108F9000002077E70B68FFDE003802406F12833A4B
:108FA000F564040885F00308E96404080000000083
:108FB000CDEC0308F8B5114ED6F804480546006814
:108FC0000F4664080BF0BCFAB4FBF7F1B1F5803F33
:108FD00003D3012CFAD96408F6E72246284689B261
:108FE0003FF03CF841F26C03054AF250284605492F
:108FF000BDE8F84000223EF0B1BF00BFA82C002021
:1090000021FD0108143D002010B5044C04480A4617
:1090100021460AF0D7F8204610BD00BF1C3D0020B5
:10902000306C070810B5044C04480A4621460AF083
:10903000C9F8204610BD00BF1C3D0020406C070849
:1090400010B5044C04480A4621460AF0BBF82046F5
:1090500010BD00BF1C3D00204C6C070810B5044C2F
:1090600004480A4621460AF0ADF8204610BD00BF6C
:109070001C3D0020586C070810B5044C04480A46F3
:1090800021460AF09FF8204610BD00BF1C3D00207D
:10909000646C070810B50C4C94F8CD200023C4F87C
:1090A00080300AB1094AD3675AF098FE20B10423F0
:1090B000022084F8843010BDD4F800396367092396
:1090C00084F8843010BD00BFB01B0020A03D0020FC
:1090D00070B50D4D95F88430042B04460E460AD029
:1090E000082B06D1EB6F83420CD0FFF7D3FF022889
:1090F00001D0012070BD0823C5E91F4685F88430E2
:10910000022070BD022070BDB01B002010B50AF017
:109110002DF8104C58B194F88430032B12D894F8E1
:1091200078300133DBB2072B84F8783003D9002381
:1091300084F8843010BDD4F800396367012384F8C3
:10914000843010BDD4F8BC004FF480715EF022F87A
:10915000E5E700BFB01B002070B54379234C002B1E
:1091600014BF0123002384F8B03003D1002384F816
:10917000843070BD1E4D002195F98320032040F0FE
:10918000F9FC0028F2D0466830465CF0F9FC84F81F
:10919000CC000028EAD095F88130003B18BF0123AD
:1091A000304684F8CD305AF0EDF909F0DFFF38B9D8
:1091B00094F8783084F88400013384F8783070BDF6
:1091C0005AF0F2FE40B194F878300022013384F86E
:1091D000783084F8842070BDD4F8002984F87800B1
:1091E0000123626784F8843070BD00BFB01B00208B
:1091F000A03D002010B55AF0D7FE58B10B4C94F8A2
:1092000078300133DBB2072B84F8783003D90023A0
:1092100084F8843010BD09F0A9FF0028F7D0D4F8F5
:1092200000396367012384F8843010BDB01B00202F
:109230002DE9F041874C94F8B050002D00F0F780F4
:1092400094F88420844F0226531E082B40D8DFE870
:1092500003F036389D3F674F153F05005AF0BEFDBD
:10926000002840F0EB80636FD4F80029FA33934272
:109270002BD2FFF7BFFF94F88420E5E75AF0AEFD4C
:109280000028F0D0D4F880300022012B84F8782018
:1092900040F2D880E16F94F8CD00013B0131C4E980
:1092A0001F1308B16C4BDA67082284F88420A2F1FE
:1092B0000805B5FA85F56D092846BDE8F08184F802
:1092C00084605AF08BFD002841D194F88420531E0D
:1092D000DBB2022B09D8D4F80039616F5B1AC82BB6
:1092E000E5D9FFF787FF94F88420042ADFD1E3E76C
:1092F000236B002BDBD1E66ED4F8003963670722BD
:1093000084F88420002ED2D0D4E91821236F0120C4
:10931000B047DAE7636FD4F8001964338B42C6D2E2
:10932000D4F82C80B8F1000FF4D15AF057FD002882
:10933000A1D0E66E84F87880042384F88430002E6F
:109340007AD0D4E91821236F4046B047BDE75AF0E0
:10935000EBF90028B9D197F88530002BA3F102036F
:10936000B3FA83F314BF022201225B0984F8792047
:1093700084F87A305AF0D8F900287FF47AAFD7F819
:10938000D030C4F88830032384F884305AF0CCF904
:1093900000289AD1304BC4F8800093F8B460B3F839
:1093A000B600D3F8B8E0D3F8B8C0D3F8B870D3F8A3
:1093B000B82084F88E6093F8BC10A4F88C0093F861
:1093C000BD6084F8922093F8BD00D3F8C020C4F8A3
:1093D0009420B3F8C680B3F8C62084F89310B3F88D
:1093E000C610C2F30B1343EA182303F00F0301F076
:1093F0000F024FEA1E6E4FEA1C4C3F0A360900F07E
:109400000F0003F5FA63042184F8990084F88FE0D3
:1094100084F890C084F8917084F89860A4F89A3029
:1094200084F89C2084F884102846BDE8F08184F8F4
:1094300084502846BDE8F08105463DE7042384F8C2
:10944000843039E7FAD1FFF725FE94F88420531EC3
:109450003EE700BFB01B0020A03D00202DE9F843EF
:109460001A4C94F88460042E0546894690461F469F
:1094700008D0082E02D00020BDE8F883FFF740F89E
:109480000228F8D1D4F8C00043F0F2FB94F87A3007
:1094900093B969021120FFF771F898B9D4F800392F
:1094A000C4F860900522C4E91B87656684F88420AF
:1094B00063670120BDE8F88329461120FFF75EF8B5
:1094C0000028EBD009F028FED5E700BFB01B002034
:1094D00070B51E4C94F88430042B06460D4608D017
:1094E000082B22D1E36F83422DD0FFF709F8022821
:1094F0001BD1D4F8C00043F0BBFB00213720FFF79D
:109500003DF829461720FFF739F8B0B994F87A30BA
:109510006BB971021920FFF731F870B90823C4E95B
:109520001F6584F88430022070BD012070BD314673
:109530001920FFF723F80028F0D009F0EDFDFFF720
:10954000E5FD032070BD022070BD00BFB01B0020F0
:109550002DE9F043694D91B006460F469046994675
:1095600095F88430042B0DD0082B07D1EB6FB34254
:1095700000F0C080FEF7C4FF0228F1D0012011B036
:10958000BDE8F083D5F8C00043F072FB95F87A305F
:10959000002B40F09E8071021820FEF7EFFF00289C
:1095A00040F0A28095F88440FEF762FF082C0CBFC3
:1095B000FC22FE22D5F8BC00818940F2E933018902
:1095C000013B11F0020F9BB24FD093B2838140F266
:1095D000E9340389013C13F0010FA4B276D08389EA
:1095E00095F8C430002B48D001A80AF0D1FDD5F879
:1095F000BC30D5F8C82095F8CE10506803970C33CE
:109600004022029300234906CDE9083304920B93CC
:109610004FF4806206930A934FF40073079201910E
:1096200005930AF0F3FDD5F8C83001A958680AF08F
:10963000C1FDD5F8C830D5F8BC2059680B6843F097
:1096400001030B6093889BB243F0020393800122D5
:1096500006230020C5E91B892F666E6685F8682001
:1096600085F8843011B0BDE8F083002BA7D144F019
:1096700091FD95F8C430002BB6D1D5F8BC00BE469C
:1096800083894FF480724FF47A744FF6FF71BEF104
:10969000000F19D01EF8013BB0F808C0013C1CF0C7
:1096A000020FA4B217D09BB283814FF47A74B0F842
:1096B00008C01CF0010F04F1FF3311D0013A838977
:1096C000C5D0BEF1000FE5D1FF23E5E7002C80D126
:1096D000CDE7314660E78C42DED144F05BFDB6E772
:1096E0009CB28C42E3D1F8E709F016FDFFF70EFDBE
:1096F000032044E7FEF7BCFEFC225BE7B01B002022
:109700002DE9F04FA44C94F8B06087B0002E00F023
:10971000D68194F88420DFF88892DFF888829F4F02
:109720004FF6FF75531E082B00F29580DFE813F00B
:10973000A700D1006B01930082000900140193007F
:10974000FF0094F8C430002B40F03E82D4F8BC00F7
:10975000236E94F868E0828903EB0E2C4FF480713D
:109760004FF47A73BCF1000F00F0B7811CF801AB25
:109770000289013B92079BB240F1EE811FFA8AF306
:1097800083814FF47A730289D20703F1FF3A40F1E3
:10979000EB8101398289E5D10EF1010E5FFA8EFE6F
:1097A000BEF1020F84F868E052D1D4F8BC0083897E
:1097B00040F2E9330289013B12F0020F9BB200F044
:1097C000C7810023838140F2E9330289013B12F013
:1097D000010F9BB200F0B4818389838940F2E933A1
:1097E0000289013B12F0020F9BB200F0A581002319
:1097F000838140F2E9330289013B12F0010F9BB2F1
:1098000000F094818389FEF733FE00F01F000528E5
:1098100000F0A182FFF77AFCD4F86CA0BAF1000F37
:1098200000F0CC810022236F616E0120D04794F8B4
:10983000842077E7206E4FF40071FEF741FE012887
:1098400000F0A481022800F0A881002800F0EF8138
:1098500094F88420531EDBB2022B00F23A81D4F834
:109860000039616F5B1AC82B00F22F81A2F1080644
:10987000B6FA86F67609304607B0BDE8F08FD4F820
:10988000C00043F0F5F900210846FEF777FE824656
:1098900009F042FCBAF1010FDAD10023D4F8C0007C
:1098A00084F8793043F0E4F940F2AB110820FEF778
:1098B00065FE052800F08581012800F0118109F07E
:1098C0002BFC94F87920002A00F04282022384F8CD
:1098D0008430D4F8C00043F0CBF994F87930022BEF
:1098E0000CBF4FF0804A4FF0000A00213720FEF7EE
:1098F00045FE51462920FEF741FE824609F00CFC48
:10990000BAF1000FA4D194F87930022B00F0A481B1
:1099100084F87AA0D4F8C00043F0AAF90021092005
:10992000FEF72CFE00283FD009F0F6FB90E74FF041
:10993000080AFEF79DFDFF2800F02082BAF1010A17
:10994000F7D1636FD4F80029FA33934280D2FFF73E
:10995000DDFB94F88420E5E6FEF78AFDFF284FF052
:10996000080A06D0BAF1010AEBD0FEF781FDFF2804
:10997000F8D1D4F880300022012B84F8782040F20E
:109980000382E26F08210132013BC4E91F2384F8FE
:1099900084100A466AE700BFB01B00200064024042
:1099A0000F64024000600240C5481021FEF788FDA8
:1099B00083460028B8D101217F20FEF7A9FB0128AA
:1099C0008246B1D158460221FEF7A2FB002800F0E2
:1099D000A0810128A8D116213A20FEF799FB013079
:1099E0008002C4F8880009F097FBD4F8C00043F067
:1099F0003FF900210A20FEF7C1FD002840F06481F4
:109A0000032384F88430102102A8FEF759FD0028B2
:109A10007FF41EAF9DF815309DF816109DF81020AC
:109A20009DF809009DF80AC01B01DBB243EA11133F
:109A300003F5FA63A4F89A30DDF8113001F00F0154
:109A400084F89C101BBA110902F00F024CEA0020A6
:109A500084F8981084F899209DF808109DF80B2040
:109A6000C4F89430039BC4F89030A4F88C0084F8B8
:109A70008E1084F88F2009F04FFB94F87A307BB970
:109A8000D4F8C00043F0F4F84FF400711020FEF752
:109A900075FD824609F040FBBAF1000F7FF457AF25
:109AA000D4F8BC0004215DF075FB0022042330468D
:109AB000C4F8802084F8843007B0BDE8F08F3046C9
:109AC00084F8846007B0BDE8F08FFFF71FFB94F8BF
:109AD0008420042A7FF4CAAECDE64FF0FF0A47E6A1
:109AE000D4F8BC004FF0040E838902A94FF47A73B6
:109AF0004FF0FF0C028992073CD5A0F80CC04FF440
:109B00007A730289D20703F1FF3A3AD5828992B279
:109B100009B101F8012BBEF1010EEBD19DF80B301C
:109B2000AB2B04BF022384F87930C8E6002B7FF406
:109B300062AE44F02FFB66E6002B7FF451AEF8E7EF
:109B4000002B7FF442AE44F025FBD4F8BC0044E681
:109B5000002B7FF42FAEF6E7AB427FF409AE44F062
:109B600019FB94F868E017E61FFA8AF3AB427FF41A
:109B70000AAEF4E7013B9BB2AB42BBD144F00AFB17
:109B8000CCE71FFA8AF3AB42BBD1F7E7636FD4F897
:109B9000002964339342BFF45BAE09F0BDFAFFF7CE
:109BA000B5FAD4F86CA0BAF1000F07D00022104625
:109BB000236F616ED04794F88420B3E594F8842035
:109BC000B0E584F879A07AE6D4F8C8305968DB6942
:109BD000494594BF4046384613F0005F00F08B8043
:109BE000D0F804C0DFF8DCE003EA0C0C1CEA0E0F2E
:109BF0003FF43CAE03EA0E03C3600B68D4F8BC002C
:109C000023F001030B600389D90703D583890389F6
:109C1000DA07FBD403899B07FCD503891906F9D41D
:109C2000838823F002031B041B0C8380BFE5019093
:109C300009F072FAE56E019884F87800042384F83C
:109C40008430002D3FF417AED4E91821236FA847C4
:109C500094F88420531EFEE5D4F8C00043F008F8C1
:109C600051463A20FEF78AFCD4F8BC1082468B8914
:109C70004FF0040E4FF47A7302A84FF0FF0C0A89DC
:109C8000920728D5A1F80CC04FF47A730A89D2073D
:109C900003F1FF3B2AD58A8992B208B100F8012B63
:109CA000BEF1010EEBD1BAF1000F0DD109F034FA7B
:109CB000029B1BBAC3F3807384F87A302AE600BF94
:109CC000501C00207D0F7D0F09F026FAFFF71EFAC9
:109CD00094F8842026E5013B9BB2AB42CFD10846E5
:109CE00044F058FABAF1000FEED1DFE71FFA8BF318
:109CF000AB42CBD1F3E7D0F800C0DFF8ACE003EA29
:109D00000C0C1CEA0E0F3FF4B1AD03EA0E038360A6
:109D100073E704212C20FEF7FBF9032183464E2034
:109D2000FEF7F6F90C21034636200193FEF7F0F911
:109D3000019B421C02339A400AFA0BFAA2FB0A0169
:109D4000420A42EAC152C4F8882009F0E5F94CE61B
:109D500084F884208AE5E56ED4F800396367072229
:109D600084F88420002D3FF481ADD4E91821236FBD
:109D70000120A84794F88420531E6CE509F0CCF923
:109D8000042384F8843076E508D0042384F88430F2
:109D900009F0C2F994F88420531E5CE5FEF7B0FB8D
:109DA00002287FF455ADBFE57D0F7D0F2DE9F04F03
:109DB000C14C94F8E01083B00546C1F34001D4F8DB
:109DC000E80042F061FF94F8E010D4F8E400C943E1
:109DD00001F001016F1E42F057FFFBB20193002D0D
:109DE00000F0D080B54EDFF8DC82B54D4FF01009A1
:109DF000D4F8E80042F02CFFD4F8E40042F028FF49
:109E0000B4F8F030002B40F04E8194F8F210D4F802
:109E1000F40042F039FF4FF0FA0A4FF47A71012052
:109E2000D8F80430C3F30803002B40F00F81EFF3A0
:109E30001183002B40F00A81D6F80029D5F808C01C
:109E4000D6F800399A42F7D1D4F818319C45F3D8A6
:109E5000D4F8147101FB07F3A3EB0C03B3FBF7F386
:109E600001FB0232D8F80430C3F30803002B40F0A2
:109E7000AB80EFF31183002B40F0A680D6F80039B9
:109E8000D5F808B0D6F80079BB42F7D1D4F81871EC
:109E9000BB45F3D8D4F8147101FB07FCACEB0B0CF9
:109EA000BCFBF7FC01FB03C39B1AB3F57A7FD9D344
:109EB000BAF1010AB4D1D4F8E80042F0C9FED4F8EE
:109EC000E40042F0C5FEB4F8F030002B40F0DF8033
:109ED00094F8F210D4F8F40081F0010142F0D4FEBD
:109EE000FA204FF47A714FF0010CD8F80430C3F324
:109EF0000803002B40F08980EFF31183002B40F022
:109F00008480D6F80029D5F808E0D6F800399A42BE
:109F1000F7D1D4F818319E45F3D8D4F814A101FB39
:109F20000AF3A3EB0E03B3FBFAF301FB0232D8F8FA
:109F30000430C3F3080343BBEFF311832BBBD6F804
:109F40000039D5F808B0D6F80079BB42F7D1D4F87B
:109F50001871BB45F3D8D4F814A101FB0AFEAEEB8F
:109F60000B0EBEFBFAFE01FB03E39B1AB3F57A7FEF
:109F7000DDD30138B9D1019B5F1EFBB2FF2B0193EA
:109F80007FF436AF03B0BDE8F08FEFF3118A89F3A9
:109F90001288AF682B68DB0344BFC4F810C1AF68F8
:109FA000D6F80039D4F810E15FFA8AFA8AF31188FA
:109FB000D4F814A1734401FB0AFEAEEB070EBEFBFE
:109FC000FAFE01FB03E3D0E7EFF3118E89F3128869
:109FD000D5F808B02B68DF0344BFC4F81001D5F8EA
:109FE00008B0D6F80039D4F810C15FFA8EFE8EF3AF
:109FF0001188D4F81471634401FB07FCACEB0B0C23
:10A00000BCFBF7FC01FB03C34EE7EFF3118E89F3B2
:10A010001288D5F808A02B68DA0344BFC4F810C131
:10A02000D5F808A0D6F80039D4F810215FFA8EFED2
:10A030008EF31188D4F814E11A4401FB0EF3A3EB5C
:10A040000A03B3FBFEF301FB023270E7EFF3118C5E
:10A0500089F31288D5F808E02B68DB0344BFC4F805
:10A060001001D5F808E0D6F80039D4F810215FFACD
:10A070008CFC8CF31188D4F814711A4401FB07F39B
:10A08000A3EB0E03B3FBF7F301FB0232EAE6D4F8CD
:10A090000C31002B3FF424AFD4F8F830C3F800A003
:10A0A00084F809A11CE7D4F80C31002B3FF4B3AEBF
:10A0B0003FF092F9AFE600BFA03D0020B01B0020AA
:10A0C00010E000E000ED00E02DE9F04FBD4CBE4E89
:10A0D00094F8E010D4F8E800DFF8F482BB4D83B0C8
:10A0E000C1F3400142F0D0FD94F8E010D4F8E40050
:10A0F000C94301F0010142F0C7FD052301934FF070
:10A100001009D4F8E80042F0A3FDD4F8E40042F0CE
:10A110009FFDB4F8F030002B40F04C8194F8F21021
:10A12000D4F8F40042F0B0FD32274FF47A710120E8
:10A13000D8F80430C3F30803002B40F00F81EFF38D
:10A140001183002B40F00A81D6F80029D5F808C009
:10A15000D6F800399A42F7D1D4F818319C45F3D893
:10A16000D4F814E101FB0EF3A3EB0C03B3FBFEF3F5
:10A1700001FB0232D8F80430C3F30803002B40F08F
:10A18000AB80EFF31183002B40F0A680D6F80039A6
:10A19000D5F808B0D6F800C96345F7D1D4F818C18E
:10A1A000E345F3D8D4F814E101FB0EFCACEB0B0C47
:10A1B000BCFBFEFC01FB03C39B1AB3F57A7FD9D32A
:10A1C000013FB5D1D4F8E80042F042FDD4F8E400F4
:10A1D00042F03EFDB4F8F030002B40F0E08094F8FF
:10A1E000F210D4F8F40081F0010142F04DFD32206C
:10A1F0004FF47A710127D8F80430C3F30803002B19
:10A2000040F08B80EFF31183002B40F08680D6F86E
:10A210000029D5F808E0D6F800399A42F7D1D4F8E9
:10A2200018319E45F3D8D4F814A101FB0AF3A3EB2F
:10A230000E03B3FBFAF301FB0232D8F80430C3F388
:10A24000080343BBEFF311832BBBD6F80039D5F8D5
:10A2500008B0D6F800E97345F7D1D4F818E1F34512
:10A26000F3D8D4F814A101FB0AFEAEEB0B0EBEFB33
:10A27000FAFE01FB03E39B1AB3F57A7FDDD30138C5
:10A28000B9D1019B5F1E17F0FF0301937FF439AF33
:10A2900003B0BDE8F08FEFF3118A89F31288D5F887
:10A2A00008B02B68DB0344BFC4F81071D5F808B0C0
:10A2B000D6F80039D4F810E15FFA8AFA8AF31188E7
:10A2C000D4F814A1734401FB0AFEAEEB0B0EBEFBE7
:10A2D000FAFE01FB03E3CEE7EFF3118E89F3128858
:10A2E000D5F808B02B68DB0344BFC4F81001D5F8DB
:10A2F00008B0D6F80039D4F810C15FFA8EFE8EF39C
:10A300001188D4F814E1634401FB0EFCACEB0B0C98
:10A31000BCFBFEFC01FB03C34EE7EFF3118E89F398
:10A320001288D5F808A02B68DA0344BFC4F810716E
:10A33000D5F808A0D6F80039D4F810215FFA8EFEBF
:10A340008EF31188D4F814E11A4401FB0EF3A3EB49
:10A350000A03B3FBFEF301FB02326EE7EFF3118C4D
:10A3600089F31288D5F808E02B68DA0344BFC4F8F3
:10A370001001D5F808E0D6F80039D4F810215FFABA
:10A380008CFC8CF31188D4F814C11A4401FB0CF333
:10A39000A3EB0E03B3FBFCF301FB0232EAE6D4F8B5
:10A3A0000C31002B3FF423AFD4F8F8301F6084F851
:10A3B00009711CE7D4F80C31002B3FF4B5AE3FF027
:10A3C0000BF8B1E6A03D0020B01B002010E000E03B
:10A3D00000ED00E000F01F0240090123032803FA0A
:10A3E00002F304D004280CD0022805D07047074A95
:10A3F000116C0B4313647047044A516C0B43536454
:10A400007047024A116B0B431363704700380240D8
:10A4100000285FD00368374A2DE9F04103F13F443B
:10A4200004F57E0402EB9422012492F8C42002F089
:10A430001F055209032A04FA05F456D0042A4FD006
:10A44000022A48D08588B5FA85F0C0F11F00C0F314
:10A45000CC0603EB860600F0070082000F24306A6A
:10A46000944020EA04003062306A01FA02F20243AA
:10A47000002132624FF0010E0A464FF0030C022712
:10A480000EFA02F838EA050002F101021CD1186840
:10A490000CFA01F420EA04001860186807FA01F6C3
:10A4A00006431E609E6826EA04069E6098689860CF
:10A4B000586820EA0800586058685860D86820EA50
:10A4C0000400D860D868D860102A01F10201D7D101
:10A4D000BDE8F0817047084A556C2C435464B1E7DD
:10A4E000054A156B2C431463ACE7034A156C2C43E7
:10A4F0001464A7E720B9060800380240002861D09C
:10A500000368384A03F13F4101F57E0102EB9122D5
:10A510002DE9F04192F8C42002F01F0452090121F4
:10A52000032A01FA04F158D0042A51D0022A4AD051
:10A530008588B5FA85F2C2F11F02C2F3CC0403EBA1
:10A54000840402F00702216A92000F20904021EA61
:10A5500000012162206A0C2101FA02F2024300216B
:10A56000226208464FF0010E4FF0030C02270EFA4C
:10A5700000F838EA050200F101001DD11C680CFA50
:10A5800001F224EA02041C601E6807FA01F4344355
:10A590001C609E6826EA02069E609E6816439E60C6
:10A5A0005C6824EA08045C605C685C60DC6824EA3F
:10A5B0000202DA60DA68DA60102801F10201D6D10D
:10A5C000BDE8F0817047084A546C21435164AFE7FD
:10A5D000054A146B21431163AAE7034A146C214313
:10A5E0001164A5E720B906080038024058B18388F5
:10A5F0004FF00042B3FA83F332FA03F303D0024977
:10A600000A6813430B607047003C0140134B02681B
:10A61000196821EA02011960596821EA02015960AA
:10A6200019680A431A609968026821EA0201996070
:10A63000D96821EA0201D9604179102907D001F1D6
:10A64000804303F59E3319680A431A60704799687E
:10A6500011439960D9680A43DA607047003C0140B1
:10A66000002864D0F0B58388B3FA83F3202B0A4620
:10A6700085B00446C3F11F0143D02D4D2D4E05EB8F
:10A6800081037718C3F81C21002197F8CC703EF0A5
:10A6900091F8B4F804C02268274CBCFA8CFCCCF1C9
:10A6A0001F0303F0FC0101F1804101F59C3103F02F
:10A6B000030398004FF00F0E02F13F438A680EFA31
:10A6C00000FE22EA0E0203F57E038A60C3F38723AD
:10A6D000834088684FF0004222FA0CF203433D4465
:10A6E0008B6002A8626101234FF400618DF80E3087
:10A6F0000292ADF80C10FFF789FF95F85C31F02B52
:10A7000001D805B0F0BD3E44F02196F8DC308DF85C
:10A71000043003224FF4807301A885F85C118DF892
:10A720000520ADF8063009F0C9FC05B0F0BD704752
:10A73000A03D002020B90608003C014010B4B8B18B
:10A740000D4CD4F86431102B05D15DF8044B052174
:10A7500000203EF017BB03EB4302224482F869114C
:10A7600001210B4482F8680182F86A11C4F864314F
:10A770005DF8044B704700BFA03D0020C078202149
:10A78000DCE700BF2DE9F04FDFF87CA32DED028B55
:10A790009AF8AC110022CAE96722CAE9692297B087
:10A7A000CAF8982119B19AF8AD218AF898219AF837
:10A7B000AE211AB19AF8AF218AF8A7219AF8B221EE
:10A7C0001AB19AF8B3218AF8A2219AF8B0211AB1E5
:10A7D0009AF8B1218AF89D219AF8B43105935A1E4E
:10A7E000D3B257B204937B1C00F0AA80BC4ABD4E82
:10A7F00052F83780029602EBC702002312790193C8
:10A8000008EE102A1D4634469946267839463046C9
:10A8100045F0D8F883463046BBF1000F1ED041F01A
:10A8200037FFEA1D1321D2B220B14FF0000E827122
:10A8300080F807E03DF0BEFF207845F0F5F84FF0D6
:10A84000070309F1010223714FF0010384F802901C
:10A850006070CDF804B05FFA82F9E3700135042D21
:10A8600004F10504D1D118EE100A029ECDF80C9027
:10A87000FFF7B0FD9C499D4A4868024042F44032CF
:10A880004A600FB9019B5BB9994C4820FFF7A2FDC4
:10A89000204602215DF00EF9A26842F00102A2609A
:10A8A0009148934A4168BAF8B64141F400014160C9
:10A8B000516821F480515160916B21F4401141F4B1
:10A8C00080119163D16841F46001D160956B85F48A
:10A8D0004011C1F3015101EB81011F2000FA01FC7D
:10A8E00025EA0C0C112505FA01F141EA0C019163EE
:10A8F000D16841F4E011D160956BC5F30151C1F10C
:10A900000401C9B201EB810188404FF0100C25EA27
:10A9100000000CFA01F108439063E4B1BAF8B811F1
:10A92000CAF8C041A1B1BAF8BA21CAF8C41162B1DB
:10A93000019B7048521A90FBF2F2CAF8C8216BB919
:10A9400017B0BDEC028BBDE8F08F6B4A1288EFE7C1
:10A950006A4A1188E7E76A4A1488DFE740460399A4
:10A960005DF0A8F85F4B012003F114090723F2788A
:10A97000441CE4B252B375783279A5F10A0101EBB7
:10A98000410105EB450C092D03FA01FE03FA0CFB0E
:10A9900002FA01F140F28E80D8F80C2022EA0E0E65
:10A9A00041EA0E01C8F80C10421E02EB82021F2180
:10A9B000062801FA02FC05FA02F261D8D8F8341030
:10A9C00021EA0C010A432046C8F834200536B14577
:10A9D000CDD1D8F80820049942F40072C8F80820B4
:10A9E000D8F8082042F48072C8F80820D8F8082067
:10A9F000574442F00102C8F8082097F9BC21022010
:10AA00003FF0B8F8044600289AD040685BF0B8F8E8
:10AA1000059A06215BF0C6F8606809F0F7FB07A805
:10AA200009F0B6FB039EA368364A0793012E8CBF3C
:10AA30004FF48060002000230D9008F14C054FF486
:10AA40000060089509920A934FF480720C930E905F
:10AA50004FF4003360680B9607A94FF40055CDE919
:10AA60000F52119309F0A6FB6268136843F00103CB
:10AA70001360D8F8083043F08043C8F808305FE727
:10AA8000C11FA0F10D0201EB81014FF01F0E02EB7F
:10AA900082020C280EFA01FC0EFA02F005FA01F10E
:10AAA00013D8D8F8302022EA0C0211432046C8F807
:10AAB00030108BE7D8F8101002FA0CF221EA0B0BD9
:10AAC00042EA0B02C8F810206EE7D8F82C1005FAFD
:10AAD00002F221EA00010A432046C8F82C2075E75B
:10AAE00004BA0608383F002000230140E030FCFF94
:10AAF00000200140803801002E7AFF1F2C7AFF1FB2
:10AB00002A7AFF1F6C3F0020A03D0020F8B5264E9A
:10AB100000EBC00406EB8404D4F8D851002D36D0E5
:10AB200094F8E9C10CF0FF07BCF1000F2FD14900E8
:10AB30004FF0010CC9B284F8EA1184F8EB2184F8D3
:10AB4000EDC184F8EE7184F8ECC184F8E9C184F8B1
:10AB5000E871AA88C4E97C33940502D501273846F8
:10AB6000F8BD2B88D9050CD44FF4805301E0013B8C
:10AB700010D02A889205FAD42B889BB243F48073B4
:10AB80002B80AB889BB243F44073AB80E6E7002791
:10AB90003846F8BDB6F8403201339BB2A6F84032D1
:10ABA0005CF070FCDBE700BFA03D002070B44E4AB3
:10ABB00092F8423203EB430002EBC000590090F8D8
:10ABC000440203281ED8DFE800F00E200250C81807
:10ABD00002EBC000D0F848420CB3013CC0F8484238
:10ABE000002070BC7047414890F82061002E63D06F
:10ABF0003F4C002001E086425ED0258801308C3435
:10AC0000002DF8D0012070BC7047C81802EBC000BE
:10AC1000D0F84842002CE0D1022480F84442194484
:10AC200002EBC10191F850020138C0B281F8500224
:10AC3000B0BB304892F80457D0F83002D1F84C42FB
:10AC4000013303F00303421E0326AB42224481F882
:10AC50004462B2FBF0F4C1F84842D3D090429CBFAA
:10AC600004F1FF34C1F84842CCE7194402EBC101BA
:10AC7000D1F8480290BB92F804178B42C2D001333E
:10AC800003F00304A14282F84242BBD004EB440328
:10AC900002EBC3020223C2F8480282F84432B2E750
:10ACA000144BD3F83022012002F2E73370BCB3FB1F
:10ACB000F2F3C1F8483270470E480B44D0F8301216
:10ACC00002EBC302012001F51C530F3370BCB3FB30
:10ACD000F1F382F84402C2F8483270470138C1F8F3
:10ACE000480200208FE700BFA03D002014000010A4
:10ACF0004440002088010020064B93F80527002AD5
:10AD0000FBD141F2682204499B5801F10C001B68F9
:10AD1000184700BFA03D0020A84400202DE9F84FAF
:10AD20003249DFF8D4B091F8851001240229074692
:10AD300019461046CBF82C404FF000022C4C1D4613
:10AD400018BF7F02FDF75CF92A4B63626B02A362B6
:10AD5000E36A40F2FF5943F093034FF400704FF45D
:10AD60008A62E3620121C4F83890A0601020E2609A
:10AD700058F026FE012D40F251434E46C4F838905B
:10AD8000CA4640F252488EBF4FF0120998464FF023
:10AD900011090A25C4F838A00121A7604846C4F863
:10ADA0000C8058F00DFE03464FF0000C40F2774245
:10ADB00001213720A6632BB900231846CBF8283091
:10ADC000BDE8F88FA663C4F808C0E26058F0F8FD4B
:10ADD000013DA6630028EFD015F0FF05DAD1034648
:10ADE000CBF82C50CBF82830BDE8F88FA03D0020E0
:10ADF000002C014000E1F505B01B00202DE9F843CF
:10AE0000184C94F88460042E0546894690461F46E7
:10AE100008D0082E02D00020BDE8F883FEF73AF9EA
:10AE20000228F8D101234A4628460021FFF776FF81
:10AE300050B1FEF7DFF9E56E002DECD00022236F54
:10AE4000616E1046A847E6E7D4F80039C4F8609070
:10AE50000522C4E91B87656684F8842063670120A6
:10AE6000BDE8F883B01B00202DE9F84F2F49DFF82B
:10AE7000C49091F885101E4602292D4B07464FF0CD
:10AE8000010418BF4702012E40F259481C6398BFC5
:10AE90004FF48B683B469346474640F2FF55B04619
:10AEA0008CBF4FF0190A4FF0180A0A241E4640F2D0
:10AEB000FF53C9F838300121C9F808605046C9F875
:10AEC0000C7058F07DFD03464FF0000C40F27742C5
:10AED00001213720C9F83850A3B95846414601220C
:10AEE000FDF78EF84646134A134B5362760296627C
:10AEF000D36A43F09103D3620D4B00210846996257
:10AF0000BDE8F88FC9F83850C9F808C0C9F80C2056
:10AF100058F056FD013CC9F838500028DDD014F037
:10AF2000FF04C4D1024B1C63BDE8F88FA03D002094
:10AF3000B01B0020002C014000E1F5052DE9F04791
:10AF4000374C82B005460E461746984694F8840062
:10AF500004280CD0082806D1E36FAB4207D0FEF7D7
:10AF600099F80228F2D0012002B0BDE8F087DFF89E
:10AF7000B8A02666DAF87C906566C9F34F210F29E0
:10AF80004FEA592223D8D4F880300193FBB194F8CA
:10AF9000CD00E0B1B9F5005F13D0224831464FF43F
:10AFA0000072484460F00AFC09F50072C2F34F21B8
:10AFB0001029CAF87C204FEA522202D0019B012BB3
:10AFC00021D192B2013A174EAD1A0B4600E001238F
:10AFD00032462846062601250021E766C4F870801F
:10AFE00084F8685084F88460FFF73EFF0028BBD0E7
:10AFF000FEF700F9E66E86B12846236F616E0022E7
:10B00000B0470320B0E7E26F013B01320421C4E9FD
:10B010001F2384F884100220A6E70320A4E700BFC2
:10B02000B01B00201C630020A03D002070B52E4DF9
:10B0300095F87441022C84B01AD0012C02D0002063
:10B0400004B070BD95F97841631CF8D0032CF6DC90
:10B050000091134695F87911024620465CF068FB92
:10B060000028ECD0204604B0BDE870405CF0FCBB8A
:10B07000D5F87C3113B11C689B886383D5F878615F
:10B08000B38940F2E9343389013C13F0020FA4B2D2
:10B0900019D084B2B48140F2E9343389013C13F011
:10B0A000010FA4B21BD0B389134630460A460021D3
:10B0B0005CF0A2F8D5F87C31A3B11A689B881383A1
:10B0C000012004B070BD002CDDD13046CDE9021264
:10B0D00043F060F8DDE90212D5F87861E4E7002C6E
:10B0E000DBD1F2E70120ABE7984E002010B50278E3
:10B0F000022A044613D0012A01D0002010BD2D4B96
:10B1000090F9040083F8B421421CF6D00328F4DC43
:10B110000A4603F5DA736179BDE81040F6E4836806
:10B1200013B11A689B8853836368988940F2E932A7
:10B130001889013A10F0020F92B225D089B2998194
:10B1400040F2E9321989013A11F0010F92B22BD085
:10B150009A899A8940F2E9321989013A11F0020F6D
:10B1600092B21ED001229A8140F2E9321989013A45
:10B1700011F0010F92B20ED09B89A368BBB11A687F
:10B180009B881383012010BD002AD1D1184643F0BB
:10B1900001F86368DDE7002AE8D1184642F0FAFFBB
:10B1A000EBE7002AD8D1F8E7002ACBD1EEE701205F
:10B1B00010BD00BF984E002010B50C4C94F87431AF
:10B1C000022B11D1D4F87C0141F058FDD4F87C0158
:10B1D00008B12123C38001213DF0ECFABDE8104005
:10B1E0000348082142F08CBF10BD00BF984E0020DC
:10B1F0000C50002073B50D4E05460C46FF230A4641
:10B20000014630468DF8073043F0ACF801230DF1CC
:10B21000070245F08001304643F068F89DF80700CA
:10B22000031B5842584102B070BD00BF0C500020B3
:10B23000094B93F87E34042B08D9053B032B08D81F
:10B2400001231A4600B10370104670470023012203
:10B25000F8E700231A46F5E7A82C0020F0B40D68A3
:10B2600000240CE0BCF1050F18D8A0F137030A2B1D
:10B2700014D104EB840415F8010B03EB4404A0F192
:10B280003003DEB2092EA0F16107A0F1410CF0D924
:10B29000052FE7D8A0F157030A2BEAD00D60146000
:10B2A000F0BC70479FED737A07EE901A20EE070A04
:10B2B000F8EE677A27EE800AFDEEC07A17EE903A34
:10B2C0002033402B00F2C780DFED6B7AB4EEE70A43
:10B2D000F1EE10FAF0EE407A0CDD9FED686ADFEDDA
:10B2E000686AB0EE677AB4EEE67AF1EE10FA77EEBD
:10B2F000C67AF6DC9FED637AF4EEC77AF1EE10FAC7
:10B300000CD59FED5E6ADFED606AB0EE677AB4EE51
:10B31000E67AF1EE10FA77EE867AF6D49FED5B7A54
:10B32000F4EEC77AF1EE10FA00F38D809FED587AB3
:10B33000F4EEC77AF1EE10FA44BF9FED527A77EE41
:10B34000677A27EEA76ADFED535A9FED537ADFED58
:10B35000536AA6EE257A67EE865AE6EE076AB6EEDF
:10B36000007AE5EEA67A27EE877ADFED486A70EE7E
:10B37000267ABDEEE76A16EE103A2033402B67D8E6
:10B38000B4EEE60AF1EE10FA0CDDDFED3C5A9FED6B
:10B390003C6AF0EE676AF4EEC66AF1EE10FA77EEF8
:10B3A000E57AF6DCDFED376AF4EEE67AF1EE10FAD4
:10B3B0000CD5DFED325A9FED346AF0EE676AF4EE99
:10B3C000C66AF1EE10FA77EEA57AF6D4DFED2F6AB1
:10B3D000F4EEE67AF1EE10FA40DDDFED276A76EE64
:10B3E000E77A67EEA75A9FED2B5A9FED2B6ADFEDA8
:10B3F0002B6AA5EE856A27EEA55AE5EE866AB8EEB9
:10B40000006AE5EE267A67EE867AC7EE206A0023A8
:10B41000836143610362C361B7EE006A76EE865AC8
:10B4200076EE666A86EE257A67EE277A66EE876A9A
:10B43000C0ED017AC0ED037A80ED007A80ED027AEA
:10B44000C0ED046A70479FED0C7A77EE677A78E773
:10B45000DFED137AD9E79FED127A86E7DFED0C6A0C
:10B46000F4EEE67AF1EE10FA44BFDFED066A76EE0E
:10B47000E77AB6E727D4D236DB0F4940DB0FC94065
:10B48000E4CB1641DB0F49C0E4CB16C1DB0FC93F4B
:10B49000DB0FC9BF92E741B99730083C15A82ABE17
:10B4A000000000002DE9F0418C4B82B093F8B521EB
:10B4B0000190002A40F00C8193F8D821B3F8DA11FA
:10B4C000DFED876AB3F8DC81864D07EE102A07EEC0
:10B4D000901AB8EEC76AB7EE007AB3F8D611A5F89D
:10B4E0003481F0EE475A4FEA4804E6EE665A8C4241
:10B4F000B8BF0C46A6EE267AA6B20121F8EEE77A8E
:10B50000A5F8386167EEA67AC5ED4A5A85ED4B7A03
:10B51000C5ED4C7A83F8B511002A00F0D680DDED38
:10B52000017A9FED710AF8EE677AA4B280EE270ADD
:10B530005EF078FB6400B0FBF4F4012CB8BF01248A
:10B54000E4B2B0FBF4F39BB2074685F83C4100EE51
:10B55000103ABBEEED0A85ED500A5EF063FB634BDB
:10B56000DFED636AB8FBF0F0A3FB0737FF0807EED7
:10B57000907AF8EEE77A022886EEA77AB8BF022022
:10B580005C4985F8440100239FED5B1A9FED5B6ADF
:10B59000DFED5B1ADFED5B5A9FED5B2ADFED5B2A87
:10B5A0009FED5B3ADFED5B3A9FED5B4A85ED527AAA
:10B5B00007EE903AB8EEE77AF0EE467AE7EE017AD7
:10B5C000FDEEE76A16EE902A2032402A7AD8B4EED1
:10B5D000E17AF1EE10FA0CDDDFED506A9FED507A62
:10B5E000B0EE675AB4EEC75AF1EE10FA77EEE67A8B
:10B5F000F6DCF4EEE57AF1EE10FA0CD5DFED476AF1
:10B600009FED487AB0EE675AB4EEC75AF1EE10FAE1
:10B6100077EEA67AF6D4F4EEC67AF1EE10FA49DDAA
:10B6200074EE677A67EEA76AF0EE624AE6EE824A47
:10B63000F0EE430AE6EEA40AB7EE007A27EEE65AE9
:10B6400077EE677AB6EE007AE5EE207A67EE877AD3
:10B650000133202BE1EC017AAAD107EE904AF8EEF3
:10B66000E77AF7EE006A86EEA77A2F4B2F4AC5F8E5
:10B67000E83703F12801A833C5F8E4171020C5F80E
:10B68000F4372021142385F84546A5F8E007A5F8EE
:10B69000F01707EE906AF8EE677AA5F8EC3782EDBE
:10B6A000007AC2EDAC7AC2EDAD7AC2EDAE7A02B0EC
:10B6B000BDE8F081F4EEE37AF1EE10FA48BF75EEE2
:10B6C000E77AAFE7F6EE007AC2E7194B1A7026E781
:10B6D000044D95F83C41B5F83861BEE7984E00201E
:10B6E0000AD7233C1400001000247449ABAAAAAA6C
:10B6F000DB0FC941600100103C8C4F3EDB0FC93F9E
:10B700000100F840DB0F49C092E741B99730083C8F
:10B7100015A82ABEDB0FC9BFDB0F4940DB0FC940AC
:10B72000E4CB1641E4CB16C11CBA06085C06001037
:10B73000000000100848002302461178022902F197
:10B74000060204D00133062BF7D10020704703EB2B
:10B75000430300EB43007047E81B002010B50021B5
:10B76000094C82B00846C4F8E01134F01BFA074BCC
:10B770000193042304F5F2700DEB0302062142F05D
:10B780007BFD02B010BD00BF984E00205475C52A45
:10B7900070B5461E00F13105344614F8011F601ED5
:10B7A000801BFF29C0B201D034F0FCF9AC42F4D1C7
:10B7B000A02051F041FA0121022034F0F3F90E4D9E
:10B7C00040F2E93401E0013C05D04221284642F034
:10B7D00005FD0028F7D16221074842F0FFFC132144
:10B7E000242034F0DFF92520092134F0DBF9BDE80D
:10B7F0007040A02051F020BA7C5000202DE9F04F7D
:10B800002DED108B034697B004331593DFEDCACAB4
:10B81000149002238A4613928B461293149C4FEA8B
:10B82000DB0604EB461202EB06103101A6EB8603A1
:10B830004FEAC60806EB4605CDE9000100EBC3035D
:10B84000043108F104001196204421442C01C6EB78
:10B85000C60C0394EC00119D04944FEACC040594AB
:10B860006C0106EB860E0294159D009C03EB4617B7
:10B870004FEACE0E02EBC6064FEACB094FF0000CA2
:10B8800051ED01AAD3ED001A92ED007A94ED005A21
:10B8900096ED004AD7ED007A15ED012A50ED016AC8
:10B8A00032EE07BA76EE840A7AEE855A31EEA70AAE
:10B8B0003BEE256A70EE804A76EEC46A36EE244A84
:10B8C00036EE646A05ED014A82ED006AD0ED00BAF9
:10B8D000D6ED012AD3ED019A95ED00AA92ED016A09
:10B8E00097ED013A91ED00CAD4ED014A7BEEE23AC0
:10B8F00036EEE19A32EE472A73EEE98A3AEE464A8C
:10B9000039EE279A78EE838AB0EE428AA9EE6C8AE5
:10B91000DC44E24573EEC33AB0EE441AA8EEEC1AEA
:10B9200076EEE77A33EEA97A7CEE643A77EEA17A86
:10B930003AEE066A7AEEC51A3CEE24AA74EECC4AB8
:10B9400039EE833A35EE6A5AF0EE639AF0EE48AA81
:10B95000E7EE2C9AA8EEAC4AE7EE2C4AE7EE6CAA8A
:10B96000F0EE418AB0EE427AB0EE612A7BEE656A73
:10B970007BEEA22A76EE4A5AA9EE2C7AA7EEAC2AE2
:10B98000A7EEAC5AE7EEEC8A32EE83BA76EEC3BA93
:10B9900035EEE09A75EEC07A36EE0A6A76EEE26A25
:10B9A00036EE0BAA76EE836A77EEA07A34EE423A50
:10B9B00077EE290A36EE4B6A7BEEA22A39EE000AB0
:10B9C00073EEAA3A78EE244A37EE697A31EE055AD8
:10B9D00071EEA85A32EE044A85ED00AA82ED016AA2
:10B9E0004D4441ED012A4A44C4ED006A81ED000A4C
:10B9F000C4ED017A494440ED010A4C4487ED007AD8
:10BA0000C6ED003AC3ED004A80ED003A87ED014AE9
:10BA1000484486ED015A4F44C3ED015A4E444B440D
:10BA20003FF62EAF119B072B40F2C781029D149E5B
:10BA3000019B03980499059A083575190C330E95E6
:10BA4000354608F108080EF10804EB1808300831F3
:10BA5000083246442C1928186918AA18079305F1CA
:10BA60000C030D960C940B900A91099208934FF0D9
:10BA700001084FF0000E129B9E44139B03EBCE0374
:10BA800003EBCE02109302EBCE0303EBCE01029147
:10BA900001EBCE0101EBCE0505EBCE06D6ED007A2B
:10BAA0000F93AEEB8E03019106EB031303EBCE076E
:10BAB000D3ED01AACDED067A019BD5ED007A97ED85
:10BAC00001BACDED057AD3ED007A029BCDED047A73
:10BAD000D3ED007A0F9BCDED037A07EBCE0CD3EDBF
:10BAE000007ADCED01BACDED027A0CEBCE01D2ED9D
:10BAF000007A109A009101EBCE00014691ED01DA37
:10BB0000CDED017A0099D2ED007A91ED01CA00EBFA
:10BB1000CE0000EBCE0494ED01EAD0ED01DACDEDDC
:10BB2000007ADDE90776DDE90954DDE90B01DDE99D
:10BB30000D23C44602E000BFF304353F94ED009AA4
:10BB400090ED00FA91ED006AD5ED007AD3ED006A30
:10BB500057ED014A92ED005A56ED013A96ED00AAD2
:10BB600035EE060A73EEA65A39EE278A34EE8F7A3E
:10BB700070EE082A75EE87EA35EE465A3EEEA26A66
:10BB800073EEE63A06ED016AD1ED019AD2ED01FAC3
:10BB9000D4ED016AD3ED011A95ED013AD0ED018A99
:10BBA00097ED004A3FEEE96A35EE491A76EE660AED
:10BBB00031EE271A3AEE612A75EE677A70EE830A43
:10BBC0003FEEA95A74EECF9A77EE897A7AEE211A6F
:10BBD000B0EE42AA74EE68FAA0EEECAADC44E245AC
:10BBE00035EEC77AB0EE639A74EE285A38EEC44A3E
:10BBF000F0EE698AA1EE6C9AE7EEAC8A36EE436A03
:10BC00007FEE644A36EE266AA0EEAC2AF0EE4A0ACF
:10BC1000E7EEEC0AE7EEAC4AF0EE687AF0EE498A1D
:10BC200036EE833AE6EE6C8AE1EE2C3AB0EE6F1A0D
:10BC3000A6EE2C1A71EEE56AA6EE2C4A71EEA55A14
:10BC400075EE031A7EEEE22A37EE43FA75EEE1EA6C
:10BC5000B0EE686A76EEC08A39EE044A7FEE86FA64
:10BC600076EEC86A33EE816A38EE888A73EEC13A9E
:10BC700037EE457A2CEE2E1A3FEE055A22EECC9A7C
:10BC80009DED03FA70EE266A33EE077AAFEE221AC4
:10BC9000AFEE2E9A7AEE244A9DED01FA79EEA09A43
:10BCA00025EE4BAA72EE670A37EE822A6BEE087A0F
:10BCB000AFEE08AAEFEE057A2DEEA63A9DED05FA55
:10BCC00067EE6D8AAFEE073AEFEE268A66EE6A2AD5
:10BCD0009DED00FA2AEEA00AEFEE202A6EEE02EAAF
:10BCE000DDED060A23EECE5AE0EEA3EA2BEEA98A9A
:10BCF000DDED023AAFEE060AA3EE848A24EE6B7AFB
:10BD00006DEE246A9DED044A2FEECD6AA0EE825AB4
:10BD1000A3EEA97AE4EE2F6AA4EE246A75EEA15A86
:10BD2000C6ED005A83ED001A83ED019A4E4447EDAB
:10BD3000017A87ED00AA4B4480ED003AC0ED018AFC
:10BD40004F4482ED000A4844C2ED012AC5ED00EAE5
:10BD500085ED015A4A44C1ED006A81ED016A4D4406
:10BD600084ED008A84ED017A49444C443FF6E6AE06
:10BD70000E9B08330E930D9B08330D930C9B0833D9
:10BD80000C930B9B08330B930A9B08330A93099B74
:10BD900008330993089B08330893079B08330793DC
:10BDA000119B08F1010843457FF465AE129BDDF855
:10BDB00044B0DB009BB2129330E517B0BDEC108BA2
:10BDC000BDE8F08F30B5044683B000BF806840F016
:10BDD0004FFF4CF2050301AA6946ADF800306068D8
:10BDE000032300258DF802505BF006FAA06840F0AE
:10BDF00045FF00BF9DF8060003B030BDF0B5BE4F53
:10BE0000BE4885B0242200215FF039FD97F8F1612A
:10BE1000002E3AD1BA4C3546D4F8443D5BB39B6A08
:10BE20004BB3B848984783682BB30388DFF8CCC27C
:10BE3000013B9BB26046664600213778032F06F12E
:10BE400006061BD001310629F7D10022017802290C
:10BE500000F1060000F0A5800132062AF6D1E16D5E
:10BE6000052908D0481C02FB01C2E0650220002120
:10BE7000938010705180284605B0F0BD062303FB67
:10BE800001414B8F013B9BB2DFE797F8F00107F5CB
:10BE9000FC73C7F8F43110B9994C0025BCE740F0A9
:10BEA000F7FB0446C7F8000240F0C6FE054600282E
:10BEB000F2D0013E022370B287F8F83142F0D4FA92
:10BEC0000028E9D0C7F8FC010CB12023E38020460C
:10BED00009213CF06FFCD7F8F431894C986840F0A8
:10BEE000CDFED7F8F431102158685BF053F9864B3A
:10BEF000D7F8F421C4F8642D93E8030001230090DF
:10BF000032208DF8041084F8683D00263DF0A0F939
:10BF1000052302AA6946D7F8F4018DF80A608DF866
:10BF2000096042F025F99DF80A009DF809109DF876
:10BF30000B20764B000240EA01401043984200F08B
:10BF4000AE8032DCA3F5F11398425ED042DD704B37
:10BF5000984252D00233984262D14FF400724FF4AB
:10BF60008073A4F8482DA4F8543DB4F8542DB4F8C7
:10BF7000483D120202FB03F300204FF48071B3F13D
:10BF8000807FC4F84C2DC4F8503D84F8560DA4F8B9
:10BF90004A1D7BD85F4BC4F8443D012284F85D2DD7
:10BFA0003AE7062101FB02C260E75B4B984234DCB2
:10BFB000053B984234DD594B0344032B77D801A24B
:10BFC00052F823F00BC00008FBBF0008EDBF0008CB
:10BFD0005BBF0008A3F52203013B984267D051DD07
:10BFE0004F4B984209D00133984219D14FF48073D6
:10BFF000A4F8483DA4F8543DB7E780224FF480737D
:10C00000A4F8482DA4F8543DAFE740224FF48073C4
:10C01000A4F8482DA4F8543DA7E7424B9842E5D038
:10C020000023A4F8483DA4F8543DC4F84C3DC4F89E
:10C03000503DFCF7D1FB034600287FF4EDAE9DF8A0
:10C040000B009DF80A209DF80C10000240EA024007
:10C05000354A0843904232D0A4F8483DA4F8543DF4
:10C06000C4F84C3DC4F8503DFCF7B6FB064600282A
:10C070007FF4D2AE97F8F00140F00AFB42F020F8CE
:10C080003546C9E6294B9842B0D0C9E70123D4F818
:10C09000640D84F85C3DB72150F0D6F97AE74FF48F
:10C0A00080621023A4F8482DA4F8543D5DE72022B7
:10C0B0004FF48073A4F8482DA4F8543D55E71C4B69
:10C0C000C4F8483D4FF4003140234FF00062012690
:10C0D000A4F8543DC4F84C1DC4F8502D84F8566D96
:10C0E000FBF7EEFF074884F85D6D50F0FFF8114B49
:10C0F000C4F8443D90E600BF984E0020E81B0020A5
:10C10000B01B0020F428002044BB06081640E000C5
:10C110001720C20020B906081940EF00EABF10FF3F
:10C1200017BA20001870EF0021AAEF001860010074
:10C13000000400084CB906082DE9F041C44BC54E77
:10C14000C54DC64C0822C3F88820336B82B043F03B
:10C150000103336307464FF4C052284640F20233CE
:10C1600088466946CDE9002308F0E6FA6B6AC4F810
:10C17000E88723F470436B626B6AC4F8F07743F48A
:10C1800020436B626B6AB649C4F8EC1723F4702342
:10C190006B626B6AB348C4F8040243F420236B62F9
:10C1A000736CB149C4F8081243F480437364736B31
:10C1B000AE48AF49C4F8140243F08003022573630C
:10C1C000AC4F84F80C52AC4EAC4DC4F858124FF042
:10C1D000A043C4F81032AA4AC4F8207203F53463AD
:10C1E000A1F5D071C4F85C52C4F82462C4F860327E
:10C1F000C4F828120123DFF8B8C2C4F81CC207F53E
:10C200001077A5F5E465A6F5A066A1F58C61C4F8E4
:10C210006472C4F81852C4F8D06284F80F3205F57D
:10C22000A075536106F5B076C4F8941284F81633FD
:10C230001946944B944AC4F89C52A7F5BC67A035A4
:10C24000C4F8A862914EC4F8A472C4F8AC3207F5E1
:10C25000D45703F56953C4F8B0524FF0502500206D
:10C26000DFF850E2C4F8D422ACF5687C02F5A042B5
:10C27000C4F8D872C4F8DC6207F5A04706F5A046FA
:10C28000C4F8E032C4F8E452A3F5485304F501754C
:10C29000C4E9BB76C4F8E822C4F81033C4F898E2C5
:10C2A000C4F8A0C202462B4684F81803402683F83F
:10C2B0001C21A3F822210132042AC3E9496083F832
:10C2C0001D1183F81F01C3F8300103F12803EED1DB
:10C2D000002211462B46402083F87423A3F87A23CA
:10C2E0000132042AC3E9DF0183F8751383F8771359
:10C2F000C3F8881303F12803EED14FF0A04364483C
:10C300009A6822F001029A60DA6842F04002DA602C
:10C3100007F098FA94F80D320022212161F31742B8
:10C320000BB142F4801294F80712D4F810320129AC
:10C330009A6300F0E480DA68D4F81063D4F8140249
:10C34000C2F3076121F0600141F0400161F31F6217
:10C350000021DA603160026861F3CC22026094F857
:10C360000F22012A00F0B88010214A4807F0BCFDD6
:10C37000484807F09FFDD4F8140294F805320022D3
:10C380004FF0FF31026142618161C26153B305F137
:10C390001407414E114607EB83074FEA830C4FF019
:10C3A000FF0E56F8042F1368002BACBF00234FF08C
:10C3B0009043B74213601161C2F808E0F1D105F172
:10C3C0005003364963440027FF2651F8042F1568AF
:10C3D000002DACBF00254FF09045994215601761C4
:10C3E0009660F2D1036994F8071243F4807301292F
:10C3F000036161D0D4F810222948002393610029F9
:10C400004FF0FF336FF0804151615360516114BFB1
:10C4100000231023906143F470139069D4F8EC1753
:10C4200043F4605343F0080303439361936809683E
:10C4300043F00103936088471A4B1B4ADA60684651
:10C440001A4B009307F03AFE02B0BDE8F08100BF3E
:10C4500000E100E00038024000000240984E002059
:10C46000BC03002008040100400040010008005007
:10C47000000B00502009005040090050200B0050D4
:10C48000003C0140C005005000100050003000503A
:10C49000A85000209C500020B0500020EC500020FC
:10C4A0000008008000ED00E00005FA0543020001ED
:10C4B0000009005020050050D4F81022144B0363EB
:10C4C0006FF08041134D00234FF0FF3093615161B5
:10C4D0005060516195619EE701680F4A0F4E41F02F
:10C4E00003010160802159629E62C3F80421E022A9
:10C4F000C3F80821C0F24002C3F80C2134E79A685F
:10C5000022F03E0141F02A0161F307029A6012E72E
:10C510000301810000080080A0004000800020008E
:10C5200010B51A4C94F8FA07C0B9194B83F8B1004A
:10C53000C3F8B40094F8FD37012B05D0022B21D0AD
:10C54000D4F800381BB910BD124BC4F8003812499A
:10C550005B68BDE81040A1F10C00184740F098F866
:10C5600094F8FC270A49003A18BF012281F8B1204B
:10C57000C1F8B4000028DDD01F22C28020213CF089
:10C5800019F9D7E7054BC4F80038E0E7984E0020CA
:10C59000B01B0020FC0300209C560020D803002084
:10C5A00099B10A6B824216D9154BD3F844289142AF
:10C5B00021D34C3991421ED30B6B9842F9D38B6B2C
:10C5C0009842F6D80B46184670470D4BD3F84418DE
:10C5D0000A6B904212D30B680BB9F4E70A6B9042D6
:10C5E0000B4602D38A6B9042EDD951F84C3F002B99
:10C5F000F4D1184670470023184670470A46D8E71A
:10C60000984E00202DE9F047CC0143D10346224A41
:10C6100043F8082B4FF0FF324260022418467E2672
:10C62000DFF87880D8F848982644013E051D494631
:10C630006FF070474FF0010A08E0A3421CD0631C62
:10C6400045F8043C321B1C460435CAB10B6BA342AF
:10C6500002D88B6BA34204D22046FFF7A1FF01460C
:10C6600090B10A794B6B002AE7D1A34204D0E6D2FD
:10C6700045F8042C631CE5E745F8047C631CE1E7FE
:10C68000C8F84818BDE8F08745F804AC321B631CB5
:10C690004946D8E78026C3E7F8FFFF0F984E0020F1
:10C6A000036870B55E6A26B133460522BDE8704066
:10C6B000184704460D464E1D00E023689B6820463F
:10C6C00098470028F9D0236815F8011B1B682046FD
:10C6D0009847B542F1D170BD036870B55E6A26B166
:10C6E00033460822BDE87040184704460D4601F164
:10C6F000080600E023689B68204698470028F9D088
:10C70000236815F8011B1B6820469847B542F1D1F4
:10C7100070BD00BF2DE9F047164D0746002095F982
:10C72000559805F65C0684B007EB010805F6FC2574
:10C7300004464FF0B60A3368ABB193F83830142B87
:10C7400011D0B9F1FF3F01D04B450CD10022694611
:10C750003046CDE90244CDE90078ADF808A08DF867
:10C760000E4034F0DDF8E036B542E4D104B0BDE867
:10C77000F08700BF984E00202DE9F743124E0124A8
:10C78000A02318255FFA84F8FF2B14DCD6F8FC0AE6
:10C79000E9B2C1F11C0282725F1C026880F80B8052
:10C7A000DBB20093C1F11B01D2F81890002342467E
:10C7B000C9B2C8473B46013DE6D10134052CE0D162
:10C7C00003B0BDE8F08300BF984E002010B50A4CBE
:10C7D00094F8190B003818BF0120FBF723FF50B164
:10C7E000064904F5306041F0FBFB04F5306010F0C1
:10C7F0002DFA04F5306010BD984E00204CBB0608A1
:10C8000070B4447941BB03684FF400524FF4007692
:10C81000202502213CBB1A8C22F001021204120CCA
:10C820001A841A8B188C22F0F30280B2120420F0C2
:10C830000A00120C014342F0010241F001011A8387
:10C8400019841A8B22F00C021204120C1A831A8B10
:10C8500092B270BC1A8370470022036816461546D0
:10C860001146002CD7D0042C21D0082C38D0198C9C
:10C8700021F480510904090C19849C8B1D8C45F608
:10C88000FF7040F6FF4128402140024342F48052AD
:10C8900041F4807199831A849A8B22F440621204C5
:10C8A000120C9A839A8B92B270BC9A8370471A8C3E
:10C8B00022F010021204120C1A84188B198C89B2FF
:10C8C00040F6FF4221F0A00102400D4342F4807285
:10C8D00045F010051A831D841A8B22F44062B3E7D9
:10C8E0001A8C22F480721204120C1A84998B1A8CFE
:10C8F00021F0F30192B2090422F42062090C3243C0
:10C9000042F4807241F0010199831A849A8B22F0DB
:10C910000C02C4E738B50F4D0446006807F010FE5E
:10C92000D5F80428204652084FF6FF713BF096FBDD
:10C9300020460021FFF764FF41F27003064AEA50E7
:10C9400005F5835120460022BDE8384010313BF008
:10C9500005BB00BFA82C0020E5CD01082DE9F0475C
:10C960009AB0DDE9226ADDF8909004460D4617463C
:10C97000984602E020683DF05BF920683DF060F9E0
:10C980000028F7D10146642201A85EF078FF264B0B
:10C990008DF80450CDF85CA00293002D40D0AB1E62
:10C9A000012B3FD9042D14BF002203221F4B0396F5
:10C9B000D3F800398DF805201E440123CDE90594F4
:10C9C00004968DF85B3037B14246394607A85EF0D1
:10C9D000F5FE8DF85A80164E96F86A9B0023189340
:10C9E000B9F1000F19D196F8690B642202FB0060BF
:10C9F00001A900F66C305EF0E1FE012386F8699B28
:10CA000086F86A3B236843B143463A4629462046A6
:10CA10001AB0BDE8F04712F039B81AB0BDE8F08797
:10CA20000522C3E70222C1E7C0590020B01B002045
:10CA3000984E00200C480D4BD0F8EC1B10B40C4C59
:10CA4000C0F8DC3B8A1E2231B0F8063C1B01A4FB77
:10CA500003C3DB08A3F5B06322F8023F9142F3D190
:10CA60005DF8044B704700BF984E00204520020837
:10CA7000CDCCCCCC70B5084C251D2E4614F8010B3E
:10CA800034F012F928B1037805F8013BB442F5D12E
:10CA900070BDFF23F8E700BFC05A00202DE9F04722
:10CAA0001D4F012607F10805B2464FF03C094FF033
:10CAB000000817F8010B3FF0EBFD044690B180F839
:10CAC0000690C671FB7803F07F02012A18D013F09C
:10CAD000800F20460DD185F8048040F0C9F885F814
:10CAE00005802C600136052E05F10805E1D1BDE871
:10CAF000F08785F804A040F0C1F885F805A0F0E7BC
:10CB00001B0605D4012120463BF054FEFB78DEE7EE
:10CB100040F0B4F8F6E700BFC85A00202DE9F04F06
:10CB2000DFF8E491DFF8E4A183B009F10C050124FA
:10CB300019F8018BB8F1000F00F0C0804FEA181708
:10CB4000013F052F08F00F0200F2BB800AEB4703FC
:10CB5000B3F8B00040FA02F616F0010600F0C38008
:10CB600001239340013B184057445BF0F3FE97F8D4
:10CB7000BC305F4E184406EBC00604236E61F471AE
:10CB8000B371002303E00133152B00F0978059495E
:10CB900003EB43025F00895C4145F4D1564B1A44D4
:10CBA00092F89914002900F0A08040463BF0D8FB91
:10CBB000804600683BF0C0FB98F805103BF0F0FBA6
:10CBC0000378002B7AD14C4B3B44042283F8D944A0
:10CBD00083F8D824002E58D0336898F8080003F161
:10CBE0003F4202F57E020AEB9222012792F8C4200E
:10CBF00002F01F015209032A07FA01F169D0042A41
:10CC000062D0022A6AD0B6F804C0BCFA8CF2C2F133
:10CC10001F02C2F3CC0103EB810102F007020E6A8E
:10CC200092000F27974026EA07060E620E6A904090
:10CC30003043002208624FF0010B11460BFA01FE4F
:10CC40003EEA0C001CD118680326964020EA060034
:10CC500018601F6802209040384318609F6827EAD8
:10CC600006079F6098689860586820EA0E00586030
:10CC700058685860D86820EA0600D860D868D8603C
:10CC80000131102902F10202D8D11C4B1C4AB3F821
:10CC9000581CB3F85A3C0091002001340190B2FBBB
:10CCA000F3F328469BB24146E4B232F099FF0123E8
:10CCB000092C6B7405F118057FF43AAF03B0BDE899
:10CCC000F08F00266E615CE70E4F3A6B0A433A63C1
:10CCD00099E70C4A176C3943116494E7094A576C79
:10CCE000394351648FE76E614BE70B68FFDE00BF8D
:10CCF000AC31002040310020A82C0020984E0020AC
:10CD000040420F0000380240F45A002020B90608C3
:10CD100070B5044684B04FF4004035F059FC80B340
:10CD200000234FF4E131032590F904000293CDE98B
:10CD300000151A464FF4004135F0ABFC124BC3F816
:10CD4000280DF0B1012C40F6980208BF4FF496620E
:10CD50000E480F4DA3F8342D4FF461710D4AC3F8FE
:10CD6000400D0A2683F82C4DC3F8306DA3F8361D0C
:10CD7000A3F8381DC3F83C5DC3F8442D012004B06E
:10CD800070BD0020FBE700BF984E002081CE010857
:10CD9000FD820108F18201082DE9F041214E224F68
:10CDA00096F8673D87F8E03006F6645607F1E4052B
:10CDB00000244FF0050816F8010B20BB2860013451
:10CDC000032C05F10405F6D197F8E010D7F8E4003C
:10CDD000C94301F001013FF057FF97F8E010D7F881
:10CDE000E80081F00201C1F340013FF04DFF97F8E8
:10CDF000E010D7F8EC0081F00401BDE8F041C1F388
:10CE000080013FF041BF3FF043FC01340121286025
:10CE1000E3B210B180F80680C37128683BF0CAFC09
:10CE2000CEE700BF984E0020A03D00202DE9F04144
:10CE30002A4C2B4DB4F86C6DA5F8F06082B0EEB9B9
:10CE400094F8680D3FF024FC94F8692DC5F8F400BF
:10CE5000003A18BF012285F8F22048B194F86A1D03
:10CE60002B22002914BF11210121C2803BF0A2FC1A
:10CE7000002002B0BDE8F04140F07CBE94F8688D1F
:10CE8000002240462B213BF0DBFA074640463FF0AC
:10CE9000FFFBF8B1F7B12B22C5F80C01C280397A3B
:10CEA000FDF7B6FA4FF000080E4AB2FBF6F3C3F3F3
:10CEB0004F0000909BB23946CDF8048005F1F80090
:10CEC000A4F86E6D32F08CFED5F8F830C3F800800F
:10CED00085F8098102B0BDE8F08100BF984E0020BE
:10CEE000A03D002040420F002DE9F84F254C94F85A
:10CEF0007C3D84F8703D04F67357002604F55964B0
:10CF00005FFA86FB0BF101085FFA88F8012117F838
:10CF1000010F42460E448A463BF092FA4FF0000958
:10CF2000054640B3387804F80E9C04F80D9C04F8CC
:10CF30000FBC04F810AC44F8045C3FF0A9FB18B136
:10CF400080F806A080F80780297AFDF761FA0E4A7A
:10CF5000002128463BF082F80C4B23600C4B221D2D
:10CF600021462846C4E901393AF0F8FF6979286872
:10CF70004A4632F0C9FD082E04F11C04C0D1BDE8B8
:10CF8000F88F00BF984E002040420F0041FB03087D
:10CF9000A1E7030870B52C4C2C4B94F8A80EC4F8EC
:10CFA000A03E00220221C4F8602EC4F8642EC4F80A
:10CFB000682EC4F89C2EA4F8A42E3BF041FA002859
:10CFC00041D0234B0668054603F1C0015A7C12B1DB
:10CFD0005A6896422BD018338B42F7D1002394F82D
:10CFE000A80EC4F88C5D84F8803D3FF051FB08B179
:10CFF0000223C380297AFDF70BFA2846154A00213F
:10D000003BF02CF8144A1549C4F8901D0026111F56
:10D010002846134BC4F8943DC4F8986D3AF09EFF2F
:10D02000697928683246BDE8704032F06DBD3046FF
:10D0300057F082F9328D0B4992B2531CB0FBF3F0DA
:10D0400081F89802CAE770BD984E002000FFFF00EB
:10D050004800001040420F002C5C0020C9E7030884
:10D0600069E90308880100202DE9F04FB64DDFF88B
:10D0700014A385B00B460446C02205F134000021FC
:10D0800001935EF0FCFB9AF8A93E002B71D09AF850
:10D09000AA3E002B00F08C80DFF8CCB29BF88C34D9
:10D0A000012B00F0AE80022B00F08F80A74BA84E22
:10D0B00002931C460FCE0FC40FCE0FC49BF8827490
:10D0C0009BF87E3496E80700A24EC5F80C613E1E20
:10D0D00018BF0126072B84E8070085F84C6900F289
:10D0E0000981042B00F21381DFF89C82DFF880A213
:10D0F0000026019B5FFA86F909F10107FFB2B342EE
:10D100003A464FF0030129DD1AF8014B20463BF067
:10D1100097F9034620461C4613B33FF0B9FAC8F806
:10D12000140018B14FF003038371C7719BF87F346B
:10D130009BF87E24002B00F0E880E37983F0010364
:10D1400049462046013658F00DFE48B14FF0010324
:10D15000082E88F8113008F11808CAD1029B06E0A1
:10D160007D4B7E4AC5F81831C5F810210023C5F85B
:10D170004839D5F8483963B10022019883F82C006A
:10D18000012183F82D101A6383F82E2005B0BDE825
:10D19000F08F734E734C0FCE0FC40FCE0FC496E8B2
:10D1A0000700A4F1200384E80700C5F84839EDE73B
:10D1B0006D4B019993F88024003A204618BF012254
:10D1C000FBF7F0FCC5F84809D3E79BF88234002B45
:10D1D0003FF46CAF9BF87E34082B12D15C4E5D4F50
:10D1E0000FCE05F1F40402940FC40FCE0FC496E8DD
:10D1F0000700012384E8070085F84C39C5F80C7155
:10D200007BE05A4C019BC5F850390FCCDFF86881A0
:10D21000A8E80F000FCCA8E80F0094E807009BF8DF
:10D2200082349BF87E448AF8E44E003B18BF012309
:10D2300088E807000026A8F5106285F84C394C4BA9
:10D24000039208F128078AF8AC6E02930BE03FF0D6
:10D250000FFD039AFB685361082E02F1180307F1D2
:10D26000200703934DD0D5F85039B34249DD029BD6
:10D2700013F8018B029340463BF016F904464046F2
:10D280003FF006FA9BF87F2494F8078081460AB1A4
:10D2900088F0010808F0010495F84C2901348AF857
:10D2A000AB4E0AB188F0010848463FF0C5FC0028A3
:10D2B0003DD0484640F09CFC6101013641F0090137
:10D2C00079617860C7F80C9087F81080F2B2B9F1F4
:10D2D000000F05D04FF0030389F8063089F80720C6
:10D2E00048463BF067FA18F0010F4846AFD13FF0CF
:10D2F000C5FCAEE7082B7FF4F7AE1E4BC5F85439DA
:10D30000F2E61D48C5F8480933E7E37918E79BF8CA
:10D3100081341A4AC5F85429012B05D0022B06BFC7
:10D32000B7FA87F35B09002385F85839DCE60B4A26
:10D33000134BC5F83029C5F82C39074AC5F83829E8
:10D3400001238AF8AC3EDDE714000010080100104C
:10D35000C8BB0608CD170608E9640408F164040890
:10D360009CBB0608485D0020A82C0020F4BB0608E2
:10D370002B3100203165040828090010616504087C
:10D38000F5640408984E002048000010F8B56E4F70
:10D3900097F8000C97F8015C3FF07AF960B12D2303
:10D3A000C380202104463BF005FA0A203BF032FE00
:10D3B000204640F013FC18B9D7F8E83EDA0000D553
:10D3C000F8BD013D092DFBD897F8FF4BD4B940209B
:10D3D00035F0FEF80028F3D090F9043097F8D51B0B
:10D3E000092BC8BF143B3B440A2993F8EC4E00F0CC
:10D3F0009D8093F8F83E97F8FE2B002A08BF1C4644
:10D40000002CDDD020463FF043F90546002800F00F
:10D4100085802D23C38001213BF0CCF901210846F2
:10D420003FF03AFC2B68AA881A833C203BF010FF9F
:10D43000002101203FF030FC97F8013C002B4CD03C
:10D44000424C00261FE02B68AA885A833BF0E2FD7D
:10D4500094F8E010D4F8E40001F001013FF014FC6E
:10D4600094F8E010D4F8EC00C1F380013FF00CFC1C
:10D470002B68AA881A8378203BF0CCFD97F8013CF2
:10D4800001369E4229DA94F8E010D4F8E400C9434A
:10D4900001F001013FF0F8FB94F8E010D4F8EC0043
:10D4A00081F00401C1F380013FF0EEFB7820002DF4
:10D4B000C9D178203BF0AEFD94F8E010D4F8E40038
:10D4C00001F001013FF0E0FB94F8E010D4F8EC002B
:10D4D000C1F380013FF0D8FBCDE797F8FF3BABB934
:10D4E00097F8003C002B7FF46BAF97F8023C012BC0
:10D4F0007FF466AFD7F8E83E13F080537FF460AF57
:10D5000087F8013CBDE8F8404AF0A6B932203BF06C
:10D510009FFE284600213BF04DF9E1E701213BF059
:10D5200049F9012108463FF0B7FB7EE7D7F8103FE5
:10D530005B057FF545AF09F069FD00287FF440AF3A
:10D54000002C7FF45FAF3BE7984E0020A03D002009
:10D55000094BD3F8140FD3F8182FD3F81C3F90427F
:10D5600002DC114602460846984204DD9A42B8BFE2
:10D570001A46104670477047984E00200B6810B44A
:10D5800014681B1B036054684B681B1B43608B684B
:10D5900092685DF8044B9B1A836070472DE9F04751
:10D5A000041E0D4612DB092C26DC824A0B468248FB
:10D5B000A0FB0410C00800EB8000A4EB4000002199
:10D5C000125C1A7059702846BDE8F08764422D231A
:10D5D000092C01F8013B24D8764A774BA3FB0403BE
:10D5E000DB0803EB8303A4EB43030020D35C487008
:10D5F0000B702846BDE8F0876F4B632CA3FB042615
:10D600004FEAD60621DC6B4A0B466B49A1FB0601AB
:10D61000C90801EB8101A6EB4101515C03F8011B34
:10D62000C5E7654A632CA2FB04364FEAD60637D815
:10D63000604A614BA3FB0603DB0803EB8303A6EB05
:10D640004303D35C01F8013BC7E7A3FB0627B4F50E
:10D650007A7F4FEAD7070DD2564A0B465649A1FBAF
:10D660000701C90801EB8101A7EB4101515C03F8F7
:10D67000011BCAE7A3FB072842F20F7294424FEA4C
:10D68000D80836D84B4A0B464B49A1FB0801C908BC
:10D6900001EB8101A8EB4101515C03F8011BDDE7BF
:10D6A000A2FB0637B4F57A7F4FEAD7070CD2414A7E
:10D6B000414BA3FB0703DB0803EB8303A7EB430307
:10D6C000D35C01F8013BB4E7A2FB073842F20F73C9
:10D6D0009C424FEAD80821D8364A374BA3FB0803AF
:10D6E000DB0803EB8303A8EB4303D35C01F8013BA6
:10D6F000DEE7324AA3FB080994424FEAD90921D850
:10D700002C4A0B462C49A1FB0901C90801EB8101F8
:10D71000A9EB4101515C03F8011BB5E7274BA2FBC4
:10D7200008099C424FEAD90921D8224A224BA3FB7F
:10D730000903DB0803EB8303A9EB4303D35C01F884
:10D74000013BCAE71E4AA3FB090394424FEAD30AEE
:10D7500021D80B461849174AA1FB0A01C90801EB59
:10D760008101AAEB4101515C03F8011BCAE7144B8C
:10D77000A2FB09029C424FEAD20A13D80E4B0D4A73
:10D78000A3FB0A03DB0803EB8303AAEB4303D35C8D
:10D7900001F8013BCAE70A22BAFBF2F049F04EFB5E
:10D7A0000346D7E70A22BAFBF2F049F047FB0146ED
:10D7B000E4E700BF7C6C0708CDCCCCCC9F86010091
:10D7C0003F420F0070B4344890F8203FA3F130017D
:10D7D000092957D800F57264224600F62F7012F816
:10D7E000015FA5F13001092904D88242F7D1002058
:10D7F00070BC7047141B022C4ADD2848002101E050
:10D8000010F8013B01EB810103EB4103161A303B99
:10D81000022E044603F0FF01F2DC214B03FB01F171
:10D82000A2424FF000030DD903EB830314F8016B00
:10D830005B00303B3344A24203F0FF03F4D11948AC
:10D8400000FB03F32E2D06D01748A0FB032301EBAA
:10D85000930070BC7047013204200024157804EB5B
:10D860008404303D6400092D00F1FF30A4B202D8D9
:10D870002C44A4B2013210F0FF00EFD1642202FB6D
:10D880000433E1E700211D4600F572620B46D9E73B
:10D89000064C0021C4E700BF984E0020B95D00206F
:10D8A0008096980040420F00ABAAAAAAB85D00205B
:10D8B00038B504460D460A460068FF215DF0DFFFDB
:10D8C00021682944216038BD83B50C4616460546BB
:10D8D00033F058FA204633F055FA0021204B084621
:10D8E000002E08BF1E463FF0D7F9002101203FF06F
:10D8F000D3F928463CF0A4F9B0B1012100203FF053
:10D90000CBF928463CF094F9074620463CF094F9C0
:10D910000028FAD0394620463CF096F93846B04700
:10D92000002108463FF0B8F920463CF089F900286C
:10D93000DFD0012100203FF0AFF920463CF078F91C
:10D940000146284601913CF077F901990028F8D06A
:10D9500028463CF079F9002108463FF09DF9C8E7D8
:10D96000DDEF0308F0B500230B604B608B60CB60EC
:10D970000B610268DFF88CC089B004ADC2F3855733
:10D980002E4647FA03F0C007344604D513F80C00BE
:10D9900004F8010B26460133062BF2D11748C2F3D7
:10D9A00003240444002394F8084333708DF818408E
:10D9B00000F5447CC2F305370DF1190647FA03F070
:10D9C000C007344604D513F80C0004F8010B2646B2
:10D9D0000133062BF2D100233370C2F3834406AB2C
:10D9E000CDE90134084602F00F0305490095C2F362
:10D9F00003124DF01FFF09B0F0BD00BF20B90608AB
:10DA0000A46C070820BC060870B5094CD4F8302F68
:10DA1000054662B10026D4F8300F2D21013640F0C2
:10DA2000B3FEAE42F7DBBDE8704042F0C5B870BD52
:10DA3000984E00202DE9F04F5FFA81F8002185B063
:10DA40000746084616463FF027F9002101203FF01F
:10DA500023F93EF0FBFD022E0AD0042E44F6C01935
:10DA600018BF4FF49649B8F1070F07D900200CE012
:10DA7000B8F1FF0F4FF41649F5D10326CE4D95F8B6
:10DA8000343F2BB90020C5F8380F05B0BDE8F08F42
:10DA9000032ECA4C0DD0A044002298F88304032121
:10DAA0003AF0CEFC0028EDD0C4F84C08C3799A07B0
:10DAB000E8D441F2670395F8340FE65400220321BD
:10DAC0003AF0BEFCC4F8500C0028DBD04FF4806163
:10DAD000BB4BC4F80838C4F814180323C4F818184A
:10DAE00041F25801A4F80C380023635441F2540168
:10DAF0004FF0010AB34A24F801A041F2640102F197
:10DB00004800635241F26601C4F81C08032E02F279
:10DB10004C406354C4F81098C4F83438C4F828381A
:10DB2000C4F82438C4F82008C4F83038C4F82C38B5
:10DB3000C2F8583890460ED0D4F84CB89BF8040080
:10DB40003EF0A6FDC4F84808584611F0FBFF5146C8
:10DB5000404612F00BF832203BF07AFB002E63D1E6
:10DB6000D4F8509CD9F8000006F0EAFC4846964AE2
:10DB700022213AF073FA41F26C03944AE25008F61B
:10DB80006401324648463AF0E9F9D4F84C98D9F89D
:10DB9000000006F0D5FC8C4A4FF6FF7148463AF07B
:10DBA0005DFA31464846FEF72BFE41F27003884A83
:10DBB000E25008F66801324648463AF0CFF9C5F817
:10DBC000388F4FF0060A022E12D0D5F8380F3CF0ED
:10DBD00037F868B1012100203FF05EF8D5F8380F22
:10DBE0003CF02EF80146002840F09E803FF054F8AB
:10DBF00038463CF025F888B1012108463FF04CF842
:10DC00004FF0050B4FF0000838463CF019F801467C
:10DC1000002840F0928001203FF03EF8042ED4D03E
:10DC200005203BF015FBCEE7012E09D1D4F8500CAE
:10DC30004946FBF7BFF9D4F84C08FEF76BFEBEE788
:10DC4000022E09D1D4F84C0811F06BFFD4F8500C17
:10DC50004946FBF7AFF9B2E7032E5DD14FF0000A5A
:10DC600041F2680351465B4804F803A040225DF08E
:10DC700006FEDFF864B18DF80FA0DFF860A19DF813
:10DC80000F30072B09D94F48012111F06FFFD4F84D
:10DC9000500C4946FBF78EF991E79DF80F3003EBE6
:10DCA00043030BEBC30393F8453073B39DF80F3078
:10DCB00003EB43030BEBC3039B6C33B39DF80F30B3
:10DCC000234493F8830400B3002203213AF0B8FB05
:10DCD0000190D0B111F025FF9DF80F309AF8001097
:10DCE000019A03EB43030BEBC30305EBC1009B6CF1
:10DCF000C0F83C3FD379DB0748BF012301F10101A4
:10DD000048BF80F8403F8AF800109DF80F3001337B
:10DD1000DBB28DF80F30B2E7042E7FF450AFD4F8A9
:10DD20004C0811F0FEFE81E7D5F8380F3BF080FF7C
:10DD3000014638463BF088FF50E738463BF078FF15
:10DD400095F88A3F01468BB9242803D14FF001038F
:10DD500085F88A3F012E04D1384601913BF074FFCB
:10DD60000199D5F8380F3BF06FFF4DE7012B06D135
:10DD70004D280CBF0223002385F88A3FEAE7022BD7
:10DD800006D13C280CBF0323002385F88A3FE1E736
:10DD9000032B25D10A2802D985F88A8FDAE70423D4
:10DDA00085F87D0F85F87C8F85F87F8F85F87E0F4D
:10DDB00085F88A3FCEE700BF984E0020A82C0020AF
:10DDC00038BC0608B034002040420F00F9FB0108BF
:10DDD00001CD0108D45D002014000010103D00208A
:10DDE000042B09D195F87E3F85F88B0F434085F8C9
:10DDF0007E3F85F88ABFADE7052BABD195F87C3F18
:10DE000095F87D9F95F87E0F4B4509D25A1C2B44FF
:10DE1000484085F87E0F85F87C2F83F8801F99E7AE
:10DE20008842B9D195F88B3F85F88AAFF42B91D110
:10DE3000B9F1000F8ED12421384685F88A9F3BF036
:10DE400003FF4D2138463BF0FFFE3E2138463BF0B4
:10DE5000FBFE494638463BF0F7FEF42138463BF0DE
:10DE6000F3FEF42138463BF0EFFE032E1BD0D4F82E
:10DE70004C08437901689D080223AB40DB439BB209
:10DE80000B828D892B408B810079202111F038FE87
:10DE9000D4F84C084A4649463AF060F8D4F84C3871
:10DEA000186806F04DFB0022D4F8500C11463AF0E9
:10DEB00055F8D4F8503C186806F042FB0120E4E520
:10DEC000114A013002EBC000F0B4D0F84CC30F4E41
:10DED0000023336033613362336333643365336605
:10DEE0003367BCF1000F0DD090F8487357B13F0174
:10DEF00000240CEB04030FCB35191034A74285E83E
:10DF00000F00F6D1F0BC704720B90608245E00204F
:10DF100038B50F4C14F8E51C01F03F018B1C02468C
:10DF200001F10A0504F8E73C04F8EA5CA4F1EC000E
:10DF300004F8E92C08311DF0F5F9254405F8EE0C3C
:10DF400014F8EA3C1C44000A04F8ED0C38BD00BF8C
:10DF5000905F002070B51D4C096854F8C05C1C4EE1
:10DF600054F8C44CD6EDA77ADFED1A6A491B00EECF
:10DF7000901A0168F8EEE00A091B60EEA70A00EEAD
:10DF8000101A20EEA07AB8EEC00A1C46A0EE007A65
:10DF9000B1EE400AF1EEC77A67EEA67AFCEEE77AB8
:10DFA000C2ED007A4DF038FD9FED0B7ADFED0B7A74
:10DFB000E0EE077AFDEEE77A17EE902A002ABCBF62
:10DFC00002F50C42A032226070BD00BF905F0020BD
:10DFD000880100202C7D8E3FA00CB34500A00C468C
:10DFE00038B50B4C002501228021204634F0DCFAA4
:10DFF00030B194F9040034F00BFB08B1006838BD6F
:10E000000135092D04F10C04EDD10020F7E700BF24
:10E01000E45E002038B5041F00F1080554F8043F01
:10E02000D81780EA430017F069FCA542F6D138BD45
:10E030002DE9F041D24CDFEDD37AD4F85C3A94F874
:10E04000F50A07EE103A2DED028BB8EE478A28EE5E
:10E05000278A002840F0CA80D4F8002B94F8F41ADC
:10E0600094F8113B002A19DD07EE902ADFEDC66A0D
:10E07000F8EEE77AC3F1640386EEA77A00EE103A71
:10E08000B8EEC00A20EE070A29B920EE000ADFED3B
:10E09000BF7A20EE270A5BF0C5FD80B2B4F8F63AED
:10E0A000A4F8F60A834200F0A18094F8607AB84E92
:10E0B000DFEDB88A4FF00008002594F8143B2B419F
:10E0C000DB0714D594F8F43A002B7FD1B4F8F63A74
:10E0D00007EE103A002F00F0FB80B8EE477AC8EE4A
:10E0E000877A77EE887A88EE277A86ED027A01358C
:10E0F000042D06F12406E0D194F8F95AB4F8FC6A2C
:10E10000002D40F0E880002F5CD194F8103B84F89B
:10E110001C5B84F8183B002E54D0002D52D007EE23
:10E12000906A0123B8EE678ADFED9A7A84F8203B83
:10E130009D42C7EE888A28D0022D43D1D4F85C1ABC
:10E140009548B0EE480A44F047FD94F81C3B012B7B
:10E1500000F01181022B35D1D4F85C1A8F48B0EE53
:10E16000480A44F039FD94F81C3B012B00F0FE8076
:10E17000022B27D1B0EE480ABDEC028BD4F85C1A12
:10E180008748BDE8F04144F027BD864AD2ED007AC9
:10E1900078EEA76A134687EEA67A002143F8041F9B
:10E1A00083ED017A78EEA76A002187EEA67A99605E
:10E1B00083ED037A77EEA88A002287EEA87A1A61A7
:10E1C00083ED057ABDEC028BBDE8F081B4F8F63A38
:10E1D000D4F85C1A00EE103A301DB8EE400A002F59
:10E1E00070D144F0F9FC94F8607A80E794F8607A92
:10E1F000002F3FF45CAF94F8F95AB4F8FC6A002D94
:10E20000E0D0694A94F8FA3A52F83C2C92F883200C
:10E210001343D7D1D4F8002B94F8113B002A65DDC5
:10E2200007EE902ADFED586AF8EEE77AC3F164034F
:10E2300086EEA77A012D00EE103AB8EEC00A27EE5E
:10E24000000A60D05BF0EEFC80B2A4F8FC0A002F5C
:10E2500079D08642B6D00028B4D094F81C3B002B6D
:10E26000B0D007EE900AB8EE678ADFED4A7A012B4C
:10E27000C7EE888A4ED0022BA4D1D4F85C1A464847
:10E28000B0EE480A44F092FB94F81C3B012B6AD094
:10E29000022B97D1D4F85C1A4048B0EE480A44F0FB
:10E2A00085FB94F81C3B012B58D0022B8AD1B0EE91
:10E2B000480ABDEC028BD4F85C1A3948BDE8F0413D
:10E2C00044F074BB301D44F071FB94F8607A0EE7A3
:10E2D000C6F8048001E7344A94F8FA3A52F83C2C24
:10E2E00092F8832013437FF40EAF93E70023A4F842
:10E2F000FC3A002F7FF466AF94F8103B84F81C5B67
:10E3000084F8183B5EE720EE000ADFED207A20EE6D
:10E31000270A97E7234A1346F3EC017A78EEA76AB7
:10E3200087EEA67A83ED017AD2ED007A78EEA76ABD
:10E3300087EEA67A83ED037A77EEA88A87EEA87A2D
:10E3400083ED057A3EE794F8103B84F81C5B84F873
:10E35000183B00283FF436AF0646E0E6114AD2EDFE
:10E36000007A131DE8E70F4A131DDDE70D4AD2EDD1
:10E37000007A131D1EE70B4AD2ED007A131D11E738
:10E3800014000010BD37863500409C45CDCC4C3C78
:10E39000740A001083F9223E380B00105C0B001049
:10E3A000800B0010A40B0010905F0020F8B5214CEA
:10E3B0001D270E46054604F8387C1DF0D9F80020CC
:10E3C0001DF078F808201DF075F80E201DF072F889
:10E3D00038461DF06FF804201DF06CF804201DF085
:10E3E00069F800201DF066F830201DF063F8002069
:10E3F0001DF060F830461DF05DF800201DF05AF861
:10E400001DF0A2F8A4F137001CF0A8FF234670B15C
:10E4100014F8372C62B914F8362C302A00D03AB9E7
:10E4200013F8352C22B913F8343C2B700120F8BDB9
:10E430000120FCE7905F0020104B034410B5044618
:10E4400093F8200410F0A4FE0D4800EB44040A23C6
:10E4500034F9241CB1F5FA6FA8BF4FF4FA61B1F595
:10E460007A7FB8BF4FF47A71A1F57A71BDE8104098
:10E47000B1FBF3F10920C9B210F0B8BE20B906080B
:10E48000905F00201D4991F8202FA2B3F0B4002620
:10E4900005463346304637461BB991F8204F2D2CA0
:10E4A00023D02E2A19D0CA1800EB800092F8204FF2
:10E4B000A4F13002092A4FEA40009CBFA0F13002CB
:10E4C000A0180E2B14D80133CA1892F8202F002A56
:10E4D000E2D106B14042F0BC70470133002DF8D0C4
:10E4E000CA182A4482F8207FDDE701231E46EBE7A5
:10E4F0000020F0BC70470020704700BF984E0020FD
:10E500001FB503AC8DF80C30009400238DF80D304E
:10E510000FF088F904B010BDF8B50546262025F0A7
:10E520008FFE114C0146D0B9206890F838301E3B60
:10E53000012B01D93BF088FB0C4F0026AE4207DBD4
:10E54000A38C0133A3840A4BD3F800396363F8BD6D
:10E5500017F8011B20683BF077FB0136EEE700233C
:10E5600084F83230EFE700BF905F0020945F002016
:10E57000B01B002010B58021044604F049FE20465F
:10E58000002104F045FE2046BDE8104005F080B9AA
:10E590002DE9F041AB4C94F84B30A06382B0884633
:10E5A0005A2B00F2B080DFE813F0C200AE00AE00DC
:10E5B000D100AE00AE00AE00AE00AE00AE00AE00C8
:10E5C000AE00AE00AE00AE00AE00AE00AE00040184
:10E5D000AE00AE00AE00AE00AE00AE00AE00280150
:10E5E0007200AE00AE007200AE00AE00AE00AE0033
:10E5F000A401AE005701AE00AE007A00AE00F501F6
:10E60000AE00AE00AE00AE005B00AE00AE00AE00ED
:10E61000AE00AE00AE00AE00AE00AE00AE00AE008A
:10E62000AE00AE00AE00AE00AE00AE00AE00AE007A
:10E63000AE00AE00AE00AE00AE00AE00AE00AE006A
:10E64000AE00AE00AE00AE00AE00AE00AE00AE005A
:10E65000AE00AE00AE00AE00AE00AE00AE00D00127
:10E6600094F84C309B0700F14782B4F85230D4F84C
:10E670004D20D4F88C105BBA9BB212BAD0188842E5
:10E68000C4E9252303D904F083FD00284CDB0020D6
:10E69000A4F884000546284602B0BDE8F08194F84D
:10E6A0009030002B40F0F48094F94830002B2ADAA7
:10E6B000D4F8803008469B689847002840F0FF81D6
:10E6C000B4F85200D4F84D20D4F88C3040BA80B25F
:10E6D00012BA15189D42C4E9252005D904F058FD49
:10E6E000002821DBD4E92520D4F88830666C03FBB0
:10E6F00000F003FB02F20225B042C4E9252084F8B1
:10E70000905000F0C98094F85C305A1CD2B204EBEF
:10E71000C30305204FF40051042A84F85C2083F8D9
:10E720006000596600F08F814FF0FF35B3E7636CEE
:10E73000002BE8D1D4F8803008469B6898470546FE
:10E74000002840F0BC81A4F88400A4E73E4B0022DE
:10E7500003F1120103F8012F8B42FBD13B4994F8DE
:10E76000863094F85C0070250D7098424FF00C05CF
:10E77000CD7110D004EBC300013390F860508D7060
:10E78000B0F86400DBB2042B40BA888114BF84F86F
:10E79000863084F8862094F84F3012229342A4F8F1
:10E7A000842098BFA4F884300025284602B0BDE834
:10E7B000F08194F84C30DA0700F12F81D4F88030E2
:10E7C00094F84F00DA6901EBC10102EB81010A798B
:10E7D000531D834228BF0346A4F88430002BE3D0A6
:10E7E000013B1A489BB201331944034411F8012D2F
:10E7F00003F8012D8342F9D1D6E7154E154F354662
:10E800000823073EC5F10700A4F88430002202E087
:10E8100092F840241D462B46B54203F8012900EB2F
:10E82000030217FA82F2F3D1D4F880304046DB6855
:10E8300098470028B8D0AB7863F07F03AB70002511
:10E8400029E700BF905F00201B8300201C8300206D
:10E850002383002020B90608D4F88030BB4A5B68C7
:10E860000846111D98470546002840F02881D4E944
:10E870002213B74A013B180E1070180C09BAD37056
:10E8800050701B0A082093705160A4F8840002E7BE
:10E89000D4E92526D4F88830D4F88050B2FBF3F2BE
:10E8A0004FF48057BE4228BF3E462D69A849A4F8C0
:10E8B00084704046B6FBF3F39BB2A8470028C0F231
:10E8C000B1803346A24AA06B812104F0D5FCD4E983
:10E8D0002520D4F8A4303244851B9E1BC4E925258D
:10E8E000C4F8A460002D7FF45FAF032384F8903058
:10E8F000D1E6974E0027334606F10C0203F8017B60
:10E900009A42FBD1D4F8803040465B686A4601A940
:10E9100098470546002840F0DC80019BBDF80020A8
:10E92000013B190E52BAF3713171190C1B0A717146
:10E930000820B371022172810C23BDF80220F0700F
:10E9400031727272A4F88430A5E6824E824F30464E
:10E950000823073EC0F10705A4F88430002202E036
:10E9600092F8482418460346864203F8012905EB2D
:10E97000030217FA82F2F3D1D4F880304046DB6804
:10E98000984700283FF410AFF37863F07F03F370EB
:10E99000002580E694F89030002B5AD194F9483045
:10E9A000002BFFF6B0AED4F8803008469B6898473D
:10E9B000002840F08480D4F880304046DB689847D7
:10E9C0000546002840F0AA80B4F85230D4F84D2013
:10E9D000D4F88C105BBA9BB212BAD0188842C4E942
:10E9E000252300F29380D4F88810606C03FB01F3B8
:10E9F00002FB01F28342C4E925237FF484AEB3F520
:10EA0000805F28BF4FF480530121A06B504A84F8E7
:10EA100090109BB204F05AFD3DE607234F49A4F83D
:10EA20008430DDE694F85C305A1CD2B204EBC303A8
:10EA300004204FF48851824284F85C2083F86000FF
:10EA400059667FF471AE002384F85C304FF0FF35D7
:10EA500021E6D4F89860D4F88000D4F88830D4F84F
:10EA600094204569B2FBF3F2B6F5805F28BF4FF4FE
:10EA700080560846B6FBF3F335499BB2A8470028F9
:10EA800059DBD4E92525D4F8A4303244AD1B9B1BB7
:10EA9000C4E92525C4F8A43025B9A06B294604F0A3
:10EAA00069FDF8E5B5F5805F28BF4FF48055ABB23E
:10EAB000A06B274A012104F009FD0025EBE594F83D
:10EAC0005C305A1CD2B204EBC30302204FF46851ED
:10EAD00022E694F85C3004EBC3020133DBB202207F
:10EAE0004FF46851042B82F86000516620D084F8FE
:10EAF0005C304FF0FF35CEE594F85C305A1CD2B252
:10EB000004EBC30305204FF4105105E604F040FB6D
:10EB10000028FFF609AED4E9252364E794F85C30B9
:10EB20005A1CD2B204EBC30302204FF41C51F3E58C
:10EB300084F85C70F8E594F85C305A1CD2B204EBAF
:10EB4000C30304204FF4407175E700BF1860002034
:10EB50001C8300202383002020B9060858BD060826
:10EB600010B51C203DF094FD1121044639F022FE21
:10EB700020463EF07DF8C8203AF06AFB2046BDE80A
:10EB800010403EF07BB800BF08B500203DF080FD8E
:10EB9000054BC3F8AC0008B12A23C380BDE8084088
:10EBA000402139F007BE00BF905F00202DE9F04FF3
:10EBB000B34CD4F810325A69D2078BB002D50BB0DF
:10EBC000BDE8F08F5A699B6912EA030AF7D0CAF3CD
:10EBD00007431AF4002F009340F00281009B5D0769
:10EBE00043D41AF0020F5FFA8AF503D0D4F810323A
:10EBF00002225A61BAF1000FC0F20D821AF4006FBE
:10EC0000CAF3072740F082812E0708D59D4B9E4806
:10EC1000D3F8AC329847D4F8103208225A61ED0686
:10EC200000F1E581F80600F1A581B90600F12E8119
:10EC3000009BDA0609D5934B9348D3F8BC3298472A
:10EC4000D4F810324FF480125A61009B9B06B6D55F
:10EC50008C4B8D48D3F8C0329847D4F810324FF41B
:10EC600000125A610BB0BDE8F08FD4F814229369FA
:10EC7000D26913401FFA83FBBBF1000FB1D0DFF85C
:10EC80000882CDF80CA045464FF0000909E05FEA84
:10EC90005B0B09F1010908F1040805F1280500F0F2
:10ECA000D6811BF0010FF2D0D4F814125FFA89F765
:10ECB00008694A6B04EB8703FA40D3F81C32D2018F
:10ECC0009B68D2B202431A40D007D3B216D54B6B21
:10ECD000D8F81820012000FA09F023EA00034B635A
:10ECE000684B6948D3F8A4320121916039469847AE
:10ECF00094F80762012E00F0F88101231A0703D56A
:10ED0000D8F8182008239360DE0603D5D8F8182019
:10ED100010239360580603D5D8F818204023936039
:10ED2000990703D5D8F81820022393601A06AED5A8
:10ED3000D5E94C60D5F82431D8F818C0311A8B4287
:10ED4000DCF8182028BF0B46033392B2B2EB930FC6
:10ED50009DD9D4F81422323704EB8703CDE901980A
:10ED600090469946B04238D2BEB3D5F8241194F8F3
:10ED70000732D5F82821371AB94228BF394601F1A0
:10ED8000030E4FEA9E0E83B98FB20337BF10D9F836
:10ED90000CA20AD0013352F8040BCAF800009F42BB
:10EDA000F8D1D5E94C60D5F82821DCF818300844B2
:10EDB0000A44B042C5F82821C5F834010AD195F8B3
:10EDC0001C11D8F83420012707FA01F122EA0102C8
:10EDD000C8F834209BB29E45C4D3DDE9019856E7BC
:10EDE000D4F814329D69DB691D402D0C3FF4F6AE5A
:10EDF00004F50176DFF88CB0B046B146002708E094
:10EE00006D0807F1010706F1040608F128083FF430
:10EE1000E5AEEB07F4D5F9B204EB8102D4F8143275
:10EE2000D2F8582292685B691A40D007D3B218D53D
:10EE300094F80702726D01239842936007D112691A
:10EE4000D8F87C33C2F312029B1AC8F88C33DBF873
:10EE5000A0324846984794F80732012B00F05381BE
:10EE600001239A0702D5726D022393601B07C7D551
:10EE7000DBF8A83248469847736D08229A60BFE7CE
:10EE8000984E0020880100209C500020D4F81432B5
:10EE9000D4F81C129A680868C2F34102022A08BF1B
:10EEA00003224FF0000514BF65F30A0062F30A0065
:10EEB00008605A6842F480725A6006A805F0EEFBBA
:10EEC000D4E98420D368BE49079D6FF38D23D360B6
:10EED0008068C0F34100014491F85014032900F008
:10EEE000CD80B849B8480126294484F80662814299
:10EEF0004FF04006A4F8086200F213810E2161F37E
:10EF00008D234FF40051D360516191E6AF4B94F8DB
:10EF10001623D3F8B432AE4800218DF817108DF8BF
:10EF200017209847D4E9842194F80E3288684FF46A
:10EF300000615161002B3FF467AEC3077FF564AEFB
:10EF400094F81933012B7FF45FAE9DF81730032B33
:10EF50007FF45AAED4F810339E491A6842F0010289
:10EF60001A601A6842F003021A600B6943F0060344
:10EF70000B6149E6D4F81422954853684FF0000815
:10EF800023F001034146536004F0AEFF94F805629C
:10EF9000414656B1904BFF2203EB860653F8045FBF
:10EFA000D86BAA609E428260F8D1D4F814328848A7
:10EFB0004FF0FF329A614FF00112DA610B2262F3D7
:10EFC000070162F30708C3F8148019611A686FF328
:10EFD0000A121A6004F05CFCD4F810227B4B7C48C7
:10EFE000D3F8B0324FF48051516198471DE6D4F800
:10EFF00010329A6922F010029A611A6AC2F34340F1
:10F00000022802F00F0144D0062823D09A6942F06A
:10F0100010029A6106E694F80E323BB1D4F8102340
:10F02000136823F0030161F307031360D4F814227B
:10F0300066495368D1F8B812654823F0010353605C
:10F040008847D4F810324FF000425A61D6E5DDF817
:10F050000CA0C6E501EB8101D4F8D45204EBC10148
:10F060002E68D1F89005C4F8D067C2F30A120244A2
:10F070002868C4F8D407C1F89025C7E700214FF4E9
:10F08000007084F806120921A4F8080261F38D23A8
:10F0900037E747F6F0701042B8D001EB8100C2F3B9
:10F0A0000A1204EBC00002F1030C5FEAAC0CD0F8CA
:10F0B0008455D4F8D4E24FEA810818BF002006D066
:10F0C0000130DEF8006045F8046B8445F8D1414416
:10F0D00004EBC101D1F88455D1F8900515440244E0
:10F0E000C1F88455C1F8902590E7B9F1000F7FF47D
:10F0F00004AE94F81533042B7FF4FFAD344804F0CC
:10F10000C7FB3346FAE5002F7FF4AAAE94F8152327
:10F11000052A7FF4A5AE4846019304F0B9FB019B94
:10F120009FE62E48A5F57401A1F51051814203D840
:10F130000D2161F38D23E4E629492A4829448142BF
:10F1400003D20C2161F38D23DBE62748A5F18C71F6
:10F15000A1F54341814203D80B2161F38D23D0E611
:10F16000224923482944814203D20A2161F38D2395
:10F17000C7E6204920482944814203D2092161F38E
:10F180008D23BEE61D48A5F1B771A1F55851814206
:10F1900003D2082161F38D23B3E6194919482944A4
:10F1A000814203D2072161F38D23AAE6164917484D
:10F1B0002944814234BF0621052161F38D23A0E655
:10F1C00020B90608401E1BFF3F420F0088010020A7
:10F1D0009C50002000ED00E0B0500020DFC810007F
:10F1E0002013FBFE20D61300FF69180000D3CEFECB
:10F1F00040771B00C05BB3FEC091210040AC2700EC
:10F20000C01D6AFE40E13300803C36FEE09C4100B8
:10F21000704700BF704700BF704700BF704700BF16
:10F220002DE9F0414FF0FF35334A34482C46002396
:10F2300004E001330A2B02F1100215D0917A04295F
:10F24000F7D103F5A17100EB0111C979CF07F0D413
:10F25000661C116801D0A942EBD21C4601330A2B6F
:10F260000D4602F11002E9D1631C02D10120BDE874
:10F27000F081224D04F5A17605EB06139988F9B9C2
:10F28000DFF884802701D8F800381D49D3F81080B2
:10F290001C4A41F218432F4401EB4421F858002343
:10F2A000C047D0B1022808D141F2BC4205EB061696
:10F2B000AB58013B0121AB50B1710020BDE8F0819A
:10F2C000DFF8448005EB0413D8F8002841F2184019
:10F2D000D268185827019047D5E741F2BC4205EBA8
:10F2E0000616AB580321B17105F5A651013B012467
:10F2F000AB500C70BBE700BF38A700201C93002068
:10F300003493002025F30008984E0020044B41F26E
:10F31000D452995C09B90121995401225A7070475D
:10F320001C930020174B002010B503F89A0904E045
:10F3300001300A2803F1100315D053F80E4C8C420B
:10F34000F6D11C78032CF3D172B10F4B03EB4023A1
:10F350009A4201D0FFF7DAFF0C4B00F5A17003EBE6
:10F3600000100123837110BD084A41F2BC4400F52E
:10F37000A173115902EB031304200131987111514B
:10F3800010BD00BFDCA70020349300201C93002098
:10F3900038B5134B00209C7B14B11D688D4205D0FD
:10F3A00001300A2803F11003F5D138BD72B10D4BBD
:10F3B00003EB40239A4210D0FFF7A8FF0A4B00F559
:10F3C000A17003EB00100123837138BD064B00F5DB
:10F3D000A17003EB0010827138BD022CECD1EDE777
:10F3E00034A70020349300201C9300202DE9F84F0F
:10F3F00012F0020E9B4606D028B9FFF787FF0225C0
:10F400002846BDE8F88F804C41F228656559002DEB
:10F410005BD14FF0FF367D4FB146B046B246002576
:10F420003B68984200F0B68097F80EC0BCF1000F20
:10F430005BD0BCF1010F15D105F5A17C04EB0C1CD0
:10F440009CF807C01CF0010F0CD11CF07E0F09D1F5
:10F450005FEADC1340F0A880D7F808C0D44501D299
:10F46000E246A94601350A2D07F11007D8D1751CCF
:10F4700004D1B8F1FF3F00F09F80464641F2B84802
:10F4800006F5A17754F80850013544F8085004EB0C
:10F49000061C41F21C494FEA07184CF8095044F881
:10F4A000085041F2184904EB07154FF000084CF8DA
:10F4B0000900C5F8048004EB0715AD79042D9CD82C
:10F4C000DFE805F01A330F334D0041F2306741F2A7
:10F4D0002C66E759A65907FB0565A84299D3FFF7A3
:10F4E00015FF00252846BDE8F88F2E4601350A2D68
:10F4F00007F1100794D1BAE712F0010C70D104EBB8
:10F500000710D51090F80780BBF1030F65F3C718FB
:10F5100080F8078062D94FF6FF7083455B4628BFAD
:10F5200003469BB204EB07108380BEF1000F16D098
:10F5300004EB061303F5A0531833987B04280ED070
:10F5400041F2B8454FF0040C60590130605141F26E
:10F55000BC45586083F80EC06359013363515007AE
:10F5600005D504EB0710C37943F00103C371D3063B
:10F5700008D504EB0714E379C3F34502013262F3C3
:10F580004603E371224B012503EB46260E60284615
:10F59000BDE8F88F05F5A17704EB07164FEA071CC5
:10F5A000B67986B92E4669E7A84601350A2D07F1D6
:10F5B00010077FF435AF5AE7B9F1FF3F18BF4E4649
:10F5C0007FF45CAF8DE741F2B8482E4654F80850FE
:10F5D000013544F8085044F80C506CE76346A1E745
:10F5E0000C4B0B49D3F800380B4AD3F8088001EBD9
:10F5F00046210023C04700283FF473AF04EB0714F3
:10F600000223A371FCE600BF1C93002034A7002056
:10F6100034930020984E002091F3000870B5114EED
:10F620003378022B104B0D4607BFC4B2010AC0F35A
:10F63000D41100F07F04186882B00844002301222E
:10F6400001A9FFF7D3FE01280AD13378022B019BD1
:10F6500016BF53F8243033F8143023F070432B6076
:10F6600002B070BD1C9300203CA9002010B51446C8
:10F6700002070B4610D50B4941F2B452581C8B5867
:10F68000834204D305D100232360012010BDFFF77E
:10F690003DFE2060012010BD21461846BDE8104007
:10F6A000BCE700BF1C9300202DE9F0414268C2F383
:10F6B00008030B44B3F5007F82B004460D4657D3D0
:10F6C00090F91A30591C0AD0304A03F5A17302EBA5
:10F6D0000313FF21DA796FF30002DA71817694F96E
:10F6E0001B305A1C0FD0294A03F5A17302EB0313F8
:10F6F000FF20DA79C2F34501013921EAE17161F3B2
:10F700004602DA71E0762378022B37D01F4A41F2A5
:10F710003063D358B5EB432F4FEA432824DC41F242
:10F7200038636768D6583E407342AB421CDCAB1965
:10F73000434511D32169207E01AAFFF797FF0128D5
:10F7400012D16768236963614744019B2361A5EB7C
:10F750000801BF1B67608D192046F8F73DFE20B9F0
:10F760003D446560012000E0002002B0BDE8F0816A
:10F7700015444560012002B0BDE8F08161680120B8
:10F780002944616002B0BDE8F08100BF1C930020F5
:10F7900070B5154604460E46FFF786FF50B994F83B
:10F7A000280028B9022384F82830C4E90B5670BD1C
:10F7B000022070BD1DB12046A847012070BD012068
:10F7C00070BD00BF10B4D0E9011390F91A208B422C
:10F7D00038BF0B46511C83600AD0144B02F5A1724E
:10F7E00003EB0212FF21D3796FF30003D37181760B
:10F7F00090F91B305A1C0FD00C4A03F5A17302EB91
:10F800000313FF24DA79C2F34501013921EAE171DA
:10F8100061F34602DA71C4760022436A5DF8044B54
:10F820004261426011460361B2E700BF1C930020B1
:10F8300038B54422002111485CF021F8104B0F48E4
:10F840001A7841F2F2514FF6FF745C5241F2F051D6
:10F8500003245C54022A41F2D85118BF032241F21A
:10F860003C655A5441F2FC5441F2F1525D591D512C
:10F8700010219954FFF7A6FF012038BDF4A80020FD
:10F880001C9300202DE9F041B1F904300F2B82B018
:10F890000C461646054632D02846F8F7C1FD95F9C4
:10F8A0001B80B8F1FF3F074633D02D4B41F2184281
:10F8B00003EB08118A58904211D1183303EB482307
:10F8C000A188013109B203EB4113A18028463360BE
:10F8D000F8F7A6FD2060012002B0BDE8F081FFF737
:10F8E00015FD2846F8F778FD28B100230120336084
:10F8F00002B0BDE8F081002002B0BDE8F0814FF415
:10F900000071FFF7D1FE0028F5D04FF6FF73A380FA
:10F91000C2E72846F8F760FD0028E2D10FB9FFF7EB
:10F92000F5FC38460023112201A9FFF75FFD0128ED
:10F93000D7D1019B0B4A9A1A48BF02F2FF12B2F5C7
:10F94000A05F4FEA622106D24FFA81F885F81B804A
:10F95000002BB5D1C5E7FFF7D9FC019BF6E700BF47
:10F960001C9300203493002030B50446C06983B056
:10F9700010B9012003B030BD0D460023032201A9B8
:10F98000FFF734FD0128F5D1B4F92030002B03DA5C
:10F99000FFF7BCFC0220EDE7019A012D4FEA43116D
:10F9A00002EB431303D0022D12D1E5255554A26872
:10F9B000DA612278032A04D100221A775A779A77DB
:10F9C000DA77626A5A83C2F30F429A8203B030BD7B
:10F9D000E268DA61EDE700BF10B50378023B012B66
:10F9E0000446037E02D913F0060F5AD198063AD482
:10F9F00094F91A30591C0AD02D4A03F5A17302EB71
:10FA00000313FF21DA796FF30002DA71A17694F91A
:10FA10001B305A1C0FD0264A03F5A17302EB0313C7
:10FA2000FF20DA79C2F34501013921EAE17161F37E
:10FA30004602DA71E076237E1B070BD51C4841F2A3
:10FA4000B853C35C072B01D0FFF760FC41F2B853F9
:10FA50000022C254E26A0023237084F82830FAB1ED
:10FA6000BDE81040104700231249E0691A018A5886
:10FA7000904206D001330A2BBAD01A018A5890421C
:10FA8000F8D10B4A03F5A17302EB0313DA79C2F341
:10FA90004501013921EAE17161F34602DA71A7E714
:10FAA00010BD0121FFF760FF0128F9D1237E9DE7FA
:10FAB0001C93002034A7002030B1027822B190F8C6
:10FAC00028201AB1002070470120704710B5D0E9F6
:10FAD0000142A242C16238BF22460321826080F8FF
:10FAE0002810FFF779FF012010BD00BF2DE9F04F6E
:10FAF000DFF864918A4699F80010DAF8003002299C
:10FB0000174683B0834609F5B15240F08A801568E4
:10FB1000DEB2A6EB030805EB1325B8444FF4807260
:10FB20009044BB4208F1FF38B8FBF2F875D2A84404
:10FB3000032906EB0704A4EB03040CBF80224FF457
:10FB40008072944228BF1446A8EB050366B994421C
:10FB50002CBF0A220B2201A92846FFF747FC0128E7
:10FB600009D003B0BDE8F08F0B2201A92846FFF7AA
:10FB70003DFC0128F5D199F80020DAF80010022A9E
:10FB800001F1010321D0A64210D2019906F1804271
:10FB9000013A081F00EB840001EB820242F8043FA7
:10FBA000824203F10103F9D1DAF80010A61B7318A1
:10FBB000BBF1010FCAF800301BD09F4205F10105CF
:10FBC0002BD999F800100026B2E7A642EED2DDF854
:10FBD00004C006F10042013AACF1020000EB44001F
:10FBE0000CEB420222F8023F904203F10103F9D1EB
:10FBF000DCE7BB42E1D199F80030022B20D004F1C0
:10FC00008044019B013C4FF0FF3243F82420DAF896
:10FC100000309F4205F10105D3D8012003B0BDE8B3
:10FC2000F08F126803F07F060329C3F3D415A6EB07
:10FC300003081544B84414BF4FF4807280226FE764
:10FC400004F10044019B013C4FF6FF72584623F833
:10FC5000142003B0BDE8F08F1C9300202DE9F04183
:10FC600090F838300446032B51D8DFE803F0023215
:10FC70003B462D4BC0681978E76A41F23062032990
:10FC800099580CBF80264FF4807601FB06F141F2B3
:10FC9000B45C00EB412041F2985841F29C5E53F86D
:10FCA0000C20E06053F80E0053F808502261A5EBD9
:10FCB0004125A0EB4121901943F8085043F80E105C
:10FCC00043F80C00C4E90C205FBB6262012384F896
:10FCD000383016480021FFF747FE012811D10223D2
:10FCE00084F83830626B04F130010120FFF7FEFE2A
:10FCF000012806D1032384F8383000212046FFF77D
:10FD000033FE431EDBB2012B02D9BDE8F081022095
:10FD100094F82830062B04BF002384F82830BDE86F
:10FD2000F081921B2263D1E71C930020ACA8002035
:10FD30002DE9F04FDFF8248198F80060012887B0A2
:10FD40008CBF00230123032E02930C460B6815463B
:10FD500039D0022E62D14FF480724FEA1329DFB2FC
:10FD600001920138012823D8012203929D421AD919
:10FD7000384E06F1880A06F11C0B32681AB1DBF81E
:10FD8000001099424ED0DAF80000002348440922BE
:10FD900005A9FFF72BFB01281FD002280FD020B1A7
:10FDA00023689D42E9D82560032007B0BDE8F08FA5
:10FDB00087B1FFF7ABFA022007B0BDE8F08F022051
:10FDC00007B0BDE8F08F80220192C3F3D41903F08D
:10FDD0007F07C6E7019A0392C8E7DDE902C1059AE9
:10FDE000DDF804E098F80030022B14D0032BE6D1A4
:10FDF00052F8273023F07043B3FA83F35B0963456D
:10FE00000F44236823D00B4477452360EAD309F1DC
:10FE100001090027C5E732F81730EDE74FF480728B
:10FE20000192D2E70C490968013A02EB41224902EA
:10FE3000B2FBF1F203991344B3FBF1F201FB12326E
:10FE40000AB10B449B1A9D42236096D8ABE7AB42A4
:10FE5000ABD3A8E7B4A800204CA900201C93002035
:10FE600070B5104E3378022B0F4B0D4607BFC4B24E
:10FE7000010AC0F3D41100F07F04186882B008446E
:10FE80000023032201A9FFF7B1FA012807D1337833
:10FE9000022B019B0CBF23F8145043F8245002B0EE
:10FEA00070BD00BF1C9300203CA900202DE9F04349
:10FEB00090F83C30002983B0044614BF0221002191
:10FEC000042B7AD8DFE803F0030C3C476800FFF707
:10FED0004BFD01286FD1626B002A74D184F83C007D
:10FEE0003F4EDFF808813F4D4FF6F7771DE01FFAD0
:10FEF00080F9B94594BF4FF000094FF0010901A9FD
:10FF0000B9F1000F45D1FFF789FB012849464FD1D0
:10FF1000206BFFF7A5FF01284AD1019B2A682363C4
:10FF2000013B934228BF13462B603378206B032B91
:10FF3000DDD1404594BF4FF000094FF00109DEE7E5
:10FF4000426B04F130010020FFF7D0FD012832D1CF
:10FF5000032384F83C30224BE56A234841F2B4562F
:10FF600041F2306299599A589D5141F2985741F2A5
:10FF70009C56491B02FB01F2DD59995905EB4225BC
:10FF800001EB42220021DD519A51FFF7EDFC0128DF
:10FF900011D1042384F83C3094F82830042B04BF9A
:10FFA000002384F82830A36B8BB1204698470120AA
:10FFB00003B0BDE8F0830228FAD194F82830042B6E
:10FFC00009D00220F4E7022384F83C30B9E701208D
:10FFD00003B0BDE8F083002384F828300220E7E76F
:10FFE0001C93002050A90020ACA80020F7FFFF0FB1
:10FFF00038B590F834300446052B46D8DFE803F0D6
:020000040801F1
:100000001F033F101963006B4FF0FF31FFF728FF0C
:1000100001283AD1E06A002839D1032384F834302A
:1000200000212046FFF7A0FC01282ED1042384F8EC
:10003000343094F82830082B2DD0012038BD41F2FF
:100040002863224DEA5800F1300102320120FFF707
:100050006FFE012824D00238C0B2012815D805232C
:1000600084F8343094F82830082B04BF002384F837
:10007000283041F2D5530122EA54022038BDC06A2B
:10008000216BFFF7EDFE0128C7D0002038BD022309
:1000900084F83430F4E7002384F82830012038BD98
:1000A00041F23062E368A958D4E90B2003EB412305
:1000B00041F234616850C4E9033002B9606201233F
:1000C00084F83430A0E7014DCCE700BF1C9300203A
:1000D0002DE9F04F436883B0C3F308081646002AA1
:1000E00000F0E180714B05468946A3F1180B4FF0F3
:1000F000000AC8F5007495F91A70B44228BF344656
:10010000791C28462ED0F8F78BF90BEB071341F238
:1001100018429B58984205D0FFF7F8F8504603B0B4
:10012000BDE8F08F614B03EB47202246494640442F
:100130005BF044FB002221462846FFF729FBA2443E
:100140000028EBD02B7E1B0706D5594B2A691B686C
:100150009A4201D3FFF7DAF8361BA1444FF00008AA
:10016000C7D1DBE7F8F738F9002849D12846F8F776
:1001700057F96968C1F308032BBB21F4FF7323F01F
:10018000010303F50072AB689A422CBF06220722D6
:100190002B7E03F00C030C2B1CD0002301A9FFF7CE
:1001A00025F90128BAD10198404BC31A48BF03F280
:1001B000FF13B3F5A05F4FEA63224FD257B2AF7679
:1001C0000028B2D1AAE72B7E03F00C030C2B4FF0D2
:1001D0000702E2D19BF800C0364BBCF1030F1B684D
:1001E0000CBF4FF0800C4FF4807C03FB0CF34FEA04
:1001F000432C0CF1FF3C0CEA0101A3EB5123CDE7AA
:100200002B7E1A072ED59BF800102A4B95F8282034
:100210001B6803290CBF80214FF4807103FB01F39D
:10022000062A4FEA43233FF479AF23490868834203
:1002300030D891F83D30002B7FF470AF002A7FF466
:100240006DAF6B6985F83820062185F82810EB62C0
:100250002846FFF703FD012888D05FE7FFF756F82F
:100260000198ACE7154B1A78002A7FF457AF95F840
:100270002820002A7FF452AF082185F8342085F821
:100280002810D3F85F206B692846C5E90B32FFF7C9
:10029000AFFEE0E741F2D553012250460BF80320B0
:1002A00003B0BDE8F08F924638E700BF34930020DA
:1002B000D0A800204CA90020B4A80020F1A800205C
:1002C0002DE9F04390F8384083B00546032C00F246
:1002D000A180DFE804F0021A8B0BFFF789FE0128EA
:1002E00011D002280BD1032385F838302B6C002065
:1002F00085F82800002B00F08980984702242046CA
:1003000003B0BDE8F08385F838002B78022B79D054
:10031000414A6F6841F23863D3581F40C7F34F27F3
:100320002846F8F77DF8DFF8F48006463F1A0AE021
:10033000D8F800305A1E91454AD2FFF7B5F908B9EE
:10034000FEF7E4FF0136022201A900233046FFF741
:100350004DF8BC1901281FFA84F94FF400724FF0D0
:1003600000010446CBD101985BF089FAEB694FF4A8
:1003700000712846002BDBD06B68002BD8D1019B85
:100380004FF020324FF02E0C1A605A6083F800C0F4
:10039000C3F807204FF0100E6C6A1A625A6283F895
:1003A00020C083F821C0C3F8272083F80BE0EA6B54
:1003B0005C83C2F30F4CC4F30F4483F82BE05A87DD
:1003C0009C82A3F834C0D8F800305A1E9145B4D3AB
:1003D000C3EBC353590201F500712846FFF764F9D6
:1003E00008B9FEF793FF022385F838302B6C002202
:1003F00085F8282063B1284698470124204603B099
:10040000BDE8F0836F68C7F34F2789E7022476E7DA
:10041000012474E7002472E71C9300204CA90020FB
:100420002DE9F04F90F8303089B00446042B00F2EB
:10043000DB80DFE813F0DC00E5003700BD001C01C5
:10044000C94B41F2F2515A56501C09D002F5A17223
:1004500003EB0212FF25D0795D546FF30000D071D9
:1004600041F2F3501A56511C0FD002F5A17203EB62
:100470000212FF25D1791D54C1F34500013820EA4D
:10048000E0700B4660F34603D371237EDF0640F134
:10049000EB80B648FFF796F94FF6FF7202232284ED
:1004A00084F83030B24E3378002B40F09D80A6F1B6
:1004B0002808474604F11C0B01AD06F1100AC1469D
:1004C0002A4659463846FFF7DDF9012840F04981B0
:1004D0000198002800F026810378E52B01D0002B3D
:1004E000EED1A44BC31A48BF03F2FF13B3F5A05FCC
:1004F0004FEA632280F0798112019F4B1A44937B6B
:10050000042B994B0CD041F2B845042659590131BE
:10051000595141F2BC45516096735A5901325A51B2
:1005200041F2F2515A56561C09D002F5A17203EB62
:100530000212FF26D5795E546FF30005D57141F2A2
:10054000F3555A57511C0FD002F5A17203EB02125A
:10055000FF26D1795E55C1F34505013D25EAE575D4
:100560000B4665F34603D371202200215BF087F927
:100570002346019A53F8311F586850601160198959
:100580009B7A93721181019B627EDA7205A846F014
:100590001FFDBDF81430002B40F02D8144F2817214
:1005A000019903200A82CB810A83CB8284F8300030
:1005B000237E9D0600F1E4802046FFF703F92369BE
:1005C000002B00F0E980237E03F0F70213F0040310
:1005D000227640F0EF80122A00F0F580002384F8A4
:1005E00028302046E36A984709B0BDE8F08F5F489D
:1005F000FFF7E8F84FF6FF720123228484F83030C9
:100600005A4F04F11C0601AD04F131092A46314666
:100610003846FFF737F9012830D00228E4D1524B91
:1006200041F2F2515A56501C09D002F5A17203EB67
:100630000212FF25D0795D546FF30000D07141F2B2
:10064000F3501A56571C0FD002F5A17203EB021299
:10065000FF25D1791D54C1F34500013820EAE0702F
:100660000B4660F34603D371042384F83030002036
:10067000E36A2070984709B0BDE8F08FDDF8048088
:100680000B2249464046B8F1000F3FF4D9AE98F826
:100690000030002B3FF4D4AE5BF01DF90028B5D13B
:1006A000B8F81400B8F81A202F4B41F2306142EA32
:1006B000004259586262D8F81C20A2604902B2FB7D
:1006C000F1F001FB102008B10A44121AE26098F818
:1006D0000B20627641F2F2515A56561C09D002F5AF
:1006E000A17203EB0212FF25D0795D546FF3000075
:1006F000D07141F2F3501A56551C0FD002F5A17279
:1007000003EB0212FF25D1791D54C1F345000138D6
:1007100020EAE0700B4660F34603D371032384F8AC
:10072000303045E798F800301449022B4FF0090E9D
:10073000484699D03378002B96D1C1E9003351F85F
:10074000282C8AF8003001F8083C0B6A86F800E093
:1007500041F8102C41F80C3CFFF7B2FD01283FF4A2
:10076000AFAE022880D03FE71C930020F4A8002001
:100770001CA900203493002034A7002030A90020B9
:10078000E0690023112205A9FEF730FE01283FF49D
:1007900013AF09B0BDE8F08F237E18077FF51EAFB9
:1007A000254A41F2B853D15C00297FF41DAF0721DF
:1007B000D15413E70023E26AA16884F82830204668
:1007C000FEF7E6FF10E7626AE06AA0630421C4E96D
:1007D0000233C4E90B2284F83C30636384F82810A8
:1007E00063622046FEF7EEFFFEE6FEF78FFD0198FE
:1007F0006FF00F0281E6114B05A9B3F9B02002A8F2
:1008000046F03AFC9DF80C309DF80D609DF80A50BA
:100810009DF80B20BDF808109DF80E00DB0243EA9E
:10082000461342EA4512A1F2BC7143EA500342EA80
:1008300041229BB292B2B3E61C930020905F00204D
:100840002DE9F04190F82830013B82B00446082B96
:1008500040D8DFE803F047054C5157643F69420038
:10086000384B4568016B41F2386041F230621E58E6
:100870009B582E408A19B2EB432F4FEA432715D2DB
:1008800057E02169207EFEF7F1FE012822D1216B7D
:10089000656823696361C91B31443D44AD1B019BFD
:1008A00065608F4221634646236142D82046F7F7B0
:1008B00093FD01AA80460028E3D06568A368E26A38
:1008C0009D4238BF1D460023A56084F828300AB138
:1008D0002046904702B0BDE8F081FFF7F1FC02B07E
:1008E000BDE8F081FFF79CFD02B0BDE8F081FFF7A5
:1008F00073F802B0BDE8F0810021FFF7D7FA02B02B
:10090000BDE8F0810121FFF7D1FA0128E2D10023EF
:10091000216C84F828302046FFF7CEF8DAE7FFF79D
:100920009DF902B0BDE8F081FFF762FB02B0BDE8BF
:10093000F0812046F7F750FD0028BFD10D446560D7
:10094000BCE700BF1C93002010B5114C94F80E3288
:1009500023B9104B4FF480225A6110BD0E4A136820
:1009600023F00603136057F0E1F994F80E32002BE0
:10097000EFD0D4F814329B68DB07EAD5D4F8102303
:10098000136823F0030161F307031360E1E700BF7D
:10099000984E0020003C014010ED00E02DE9F047AA
:1009A00004460D469046002144221E46089F5AF0F8
:1009B00066FF01234FF6FF722676628384F82830A3
:1009C0002B782E2B4CD02E4604F1310A307804F1CE
:1009D000390968B12E280BD042F000FEC0B20AF8E7
:1009E000010BCA4506F1010607D030780028F1D185
:1009F00020200AF8010BCA45F7D130782E2808BF0D
:100A0000707804F1380908BF013604F13B0A58B187
:100A100042F0E4FDC0B209F8010FD14506F101062C
:100A200007D030780028F3D1202009F8010FD145F4
:100A3000F7D118F0100F14BF0323012384F8198095
:100A40002370E7622B782E2B26D16B7823BB0323F0
:100A5000204684F83030FFF7E3FC2046BDE8F087FD
:100A60006B78002BAFD1114B41F2E45103F5AF503D
:100A70005958006841F2FC529A586262C4E9020176
:100A800041F2F1529A5C627641F2D8529B5C23703B
:100A9000E7622B782E2BD8D00023204684F8303004
:100AA000FFF7BEFC2046BDE8F08700BF1C93002086
:100AB00008B50121032003F05BFB72B64BF0D8F8B8
:100AC0002DE9F04F8DB0CE4CDFF84893CD4D00901E
:100AD0004FF0000854F80B0C002800F0FE8039F0AD
:100AE000AFF80646002800F0D881D9F8003944F85C
:100AF000073CE0260023C44F04F8033CA4F10B0B91
:100B000006FB08F654F80B0C39F09AF8002800F0B0
:100B1000E48054F80B0C39F08BF814F8023C5A1EA0
:100B200082460B2A0DD8DFE812F01F003A0046007B
:100B3000530083009B00E30016013501400177015B
:100B40008E0124280CD0009A3AB915F83E2C824226
:100B500040F07F81012204F8032C0D2BD2D186E0D6
:100B6000012304F8023CCDE700234D28C4F8C5302A
:100B700084F8CD3084F8CE3004D0582808D004F85A
:100B8000023CBFE7022204F8022C84F8C430B9E723
:100B9000032304F8023C022384F8C430B2E70423A0
:100BA0003C2804F8023C0BD0BAF13E0F0CD00023D5
:100BB00004F8023CA6E70A233C2804F8023CF3D1DF
:100BC000002304F8013C9DE7012304F8013C99E768
:100BD000D4F8C500BB190344421CC4F8C52083F8EF
:100BE00067A894F8CD00022A8AEA000184F8CD10A3
:100BF00088D12378C02BDAD86278FF2A08D1052B58
:100C0000D5D9012384F8C430072304F8023C79E7DE
:100C1000A4F8C12000229342C4F8C93014BF0523B0
:100C2000062384F8C320C4F8C52004F8023C69E711
:100C3000D4F8C500BB190344421CC4F8C52083F88E
:100C400067A894F8CD00D4F8C9308AEA00019A4226
:100C500084F8CD107FF456AF062304F8023C51E728
:100C600094F8CD308342A2D10D2304F8023C14F84D
:100C7000017C002F40F0F380644B08940FCB04AE4E
:100C800086E80F00D4F8C930D4F8D100ADF82C7044
:100C900023440993B4F8C130ADF8283094F8C33038
:100CA0008DF82A3001238DF82E30324603AB08A987
:100CB000039732F0FDF848B1049B059394F8C420E3
:100CC000534B0493314658462FF02AFE039E0023CF
:100CD00004F8023C002E40F0D88008F10108B8F179
:100CE000030F04F1E0047FF4F5AE0DB0BDE8F08F22
:100CF000D4F8C500BA190244431CC4F8C53082F8C0
:100D000067A894F8CD2094F8CE0001938AEA0202F5
:100D1000514684F8CD2046F045FC019B84F8CE0076
:100D2000072B7FF4EFAEB4F80530C02B3FF63FAF92
:100D3000B4F80320A4F8C120A27884F8C3200022CC
:100D40009342C4F8C93014BF08230923C4F8C5204E
:100D500004F8023CD6E6014694F8CE0046F022FCA8
:100D600094F8CD3084F8CE008AEA0303D4F8C500A5
:100D700084F8CD30BB190344421CC4F8C52083F865
:100D800067A8D4F8C9309A427FF4BCAE092304F8AE
:100D9000023CB7E694F8CD30434084F8CD3094F867
:100DA000CE3083427FF403AF56E7D4F8C500BA19BA
:100DB0000244431CC4F8C53082F867A894F8CE00FA
:100DC0000193514646F0EEFB019B84F8CE00052BC3
:100DD0007FF498AEB4F80120B4F80330A4F8C12031
:100DE000227884F8C32000229342C4F8C93014BF8B
:100DF0000B230C23C4F8C52004F8023C82E600BF94
:100E0000FF560020905F0020984E002074BD060819
:100E10000C550120B01B0020014694F8CE0046F08E
:100E2000C1FB84F8CE00D4F8C500BB190344421CB2
:100E3000C4F8C52083F867A8D4F8C9309A427FF473
:100E400061AE0C239BE694F8CE3083427FF4AFAEC4
:100E50000AE7232804BF022204F8032C7DE6012FB1
:100E60004FF0000602D004F8026C36E7D4F8C9301F
:100E700008942344099308A8B4F8C130CDE90A6660
:100E8000ADF828302EF060FCEDE754F80B0C2FF095
:100E900079FF54F80B0CB0471FE714F8033C002B04
:100EA0003FF41BAFD9F8002954F8071C521A632AE3
:100EB0007FF613AF012B30D0022B7FF40EAF54F826
:100EC0000B3CC5F8C030C5E92D330122402385F81D
:100ED000B22085F8C430124A124BC5F8BC20124A21
:100EE000C3F8302F93F8173BC5F80821003B0F4A91
:100EF00085F8C50018BF01230D4882F8AC3B3EF0D1
:100F00005FFE4FF4005031F089FE0A483EF04EFE7D
:100F100085F80C6185F80D61DFE6FFF7C9FD00BFBC
:100F20008D640408984E00204C60002014000010CE
:100F3000B36C0708E96C0708034B93F824000038EA
:100F400018BF0120704700BF101C0020202301485B
:100F50000B80704754040020642301480B807047C5
:100F600074040020432301480B807047D8040020FC
:100F700010B5074CD4F8C800FF2807D0054951F830
:100F8000042BF7F761F9FF23C4F8C830002010BD27
:100F90005404002060A90020EAE700BF08B5D0F89B
:100FA000E4355B6A9847002008BD00BF08B5D0F85B
:100FB000E4351B6A9847002008BD00BFD0F8E4352F
:100FC00010B504461B689847D4F8E8359B689847E5
:100FD000002010BD08B5D0F8E435DB6903B19847AF
:100FE000002008BD08B5042290F81211D0F8E835A9
:100FF00080F8131180F81221DB689847002008BDA3
:1010000010B5D0F8E83504461B699847032384F8E7
:101010001231002010BD00BF0B0630B41CD401EB10
:10102000810200EBC202002300EB810582F87413F9
:1010300082F8753301241A4604FA01F16D6D61F3EB
:101040001F4201696FF3CF332B60CB6923EA0203A0
:10105000002030BCCB61704701F07F0101EB8104BF
:1010600000EBC404012200EB8105002384F81C116D
:1010700084F81D2102FA01F11A46AD6961F30F02ED
:10108000DFE700BF10B581210446FFF7C5FF20460A
:101090000121FFF7C1FF024B0020187010BD00BFF7
:1010A0002060002010B581210446FFF7B5FF2046DF
:1010B0000121FFF7B1FF82212046FFF7ADFFF7F7CF
:1010C00009F9002010BD00BF38B50D460446832144
:1010D000FFF7A2FF29462046FFF7E4FF002038BDB6
:1010E000F0B416460A063AD401EB810500EBC505BB
:1010F0002824002204FB0104022B85F87413C5F890
:101100007C6385F8773385F8752304F55D7448D0E2
:10111000154600EB8107012202FA01F17F6D61F3B0
:101120001F45D7F800C01CF4004F11D1E4882049B6
:1011300046F0805242F4004242EA834204F00F0437
:101140001C4B42EA845211400CEA030319433960F4
:101150000269D3692B430020F0BCD361704701F0D2
:101160007F0101EB810500EBC5052824012204FB6A
:101170000104022B85F81C11C5F8246185F81F3184
:10118000A5F8221185F81D2104F58E740CD00025D8
:1011900000EB8107012202FA01F1BF6961F30F053B
:1011A000BFE722711546B4E700252571F0E700BFBF
:1011B000FF87CC13007833EC002310B519460446A2
:1011C0004022FFF78DFF8021204600234022FFF7B9
:1011D00087FFD4F8E835A078012284F812215B68F3
:1011E0009847002010BD00BF70B44B78012B26D06B
:1011F0000B784A6900EB83035C6D25682369D2B1E3
:101200008A684A6102F07F0223F4002323F07F03FF
:1012100042F4002213432361C378012B04BF0B69FE
:101220006361C5F3076363F07B0363F31F652560A8
:10123000002070BC70478A6802F07F02E4E7826990
:101240004C691568136944B38E68B4428CBF06F0CC
:101250007F0404F07F0423F4002323F07F0344F48D
:10126000002443EA040388BF4E611361C378012B55
:101270001DD0C5F3076464F07B0464F31F6515603B
:10128000002BD5D14B69002BD2D002690878516B65
:10129000012383400B435363CAE723F4002323F065
:1012A0007F0343F400231361C378012BE1D10B7852
:1012B0000C6900EB8300C5F30763816963F07B036E
:1012C00063F31F654C610020156070BC704700BF60
:1012D0002DE9F0434B78012B30D00B784C6900EBB3
:1012E00083035E6D356837691CB38B681C44013C11
:1012F000B4FBF3F4C4F3090203FB02F3C3F31203D8
:101300004B61144643EAC44363F31C073761C37857
:10131000012B04BF0B697361CB78012B44D0C5F35B
:10132000076363F07B0363F31F6535600020BDE84E
:10133000F0838A680124C2F31203E3E791F8008086
:101340004E6900EB880EDEF818C0DCF80050DCF8BF
:10135000107076B3D1F80890384A06EB0904013CC6
:10136000B4FBF9F402EAC444C6F312022243CC7877
:1013700007F060473A43012C174649D0CCF81020BB
:10138000C278012A55D00269516B03FA08F30B4366
:101390005363C5F3076363F07B0363F31F65CCF806
:1013A00000500020BDE8F0834B7973B345F0005541
:1013B000B5E707F0604747F40027CC78CCF8107009
:1013C000C378012B2FD0012CE3D102699268D2059A
:1013D00054BF45F0005545F08055C5F3076262F0F3
:1013E0007B0262F31F65CCF80050002B9ED1B0B297
:1013F00003308010DEF8D04098D0CA6852F8041B41
:10140000216001339842F9D190E745F0805586E795
:1014100064F35E77CCF81070C378012BD5D10A69DC
:10142000CCF81420D1E70A69CCF81420012CB0D1F3
:10143000CBE70B69CCF81430ABE700BF0000F81F16
:101440000E4BDA68D20310D4DA68D1060FD4DA680A
:10145000D20510D4DA6812F0E00F0AD1DB6813F07D
:10146000020F14BF08200920704701207047062092
:101470007047072070470220704700BF003C0240C1
:1014800000207047002070477047704730B1044B10
:1014900093F90C000028D4BF00200120704700BF42
:1014A00060A9002008B5FFF7F1FF50B1054A537B52
:1014B000927B5B0003F00203002A18BF43F0010394
:1014C0000B6008BD60A9002008B5FFF7DFFF10B171
:1014D000014B1B690B8008BD60A9002070B5FFF7A8
:1014E000D5FF78B1084A958A65B196690023B34261
:1014F0001C4607DA02EB44040133A48BAC42DBB296
:10150000F5D30B7070BD00BF60A9002008B5FFF7D0
:10151000BDFF10B100230B70137008BD042070478D
:1015200028B1034B93F9CC00003818BF0120704755
:101530005404002008B5FFF7F3FF50B1054B93F9B1
:10154000CC20012AC3BF93F8CF30C3F340030B6014
:10155000002008BD5404002008B5FFF7E1FF18B1D2
:10156000024B93F8CE300B7008BD00BF540400202E
:1015700070B5FFF7D5FF38B10E4C94F8CF30DB07CC
:1015800003D500230B70137070BD0B4D94F9CD3053
:1015900095F82C6093FBF6F301330B7094F9CD4072
:1015A00095F82C1094FBF1F301FB134301331370F6
:1015B000EAE700BF5404002060A900200320704720
:1015C00070B50A4A92F8303006255E1CB6FBF5F479
:1015D00005FB146492F83150AC4205D002EBC30312
:1015E000C3E90D0182F8304070BD00BF60A9002042
:1015F000002230B504461046914200DC30BDA35CA9
:101600000825584010F0800F4FEA400318BF83F0C0
:10161000D503013DD8B2F5D10132EDE710B5D9B10E
:101620000E4B586E814217DCB2B1DB6A9A4213DC72
:101630000B4C013A013903FB012184F8DA1004F163
:10164000D6000521FFF7D4FF062184F8DB0004F162
:10165000D600BDE81040B3E710BD00BF60A9002070
:1016600054040020024B93F868300B60012070474F
:1016700060A90020024BB3F86A300B80012070474C
:1016800060A90020024B93F86C300B70012070476A
:1016900060A9002000230B700120137070470038F0
:1016A00018BF012070470120704770470023038056
:1016B00083708380C3800372704700BF074A084964
:1016C00092F86D3009780133DBB2994282F86D30BF
:1016D00004BF002382F86D30704700BF60A900206E
:1016E000C40B0010F8B5774C236F83B1764B1B68A1
:1016F00093F82E305BB1754B94F87420A3FB001364
:10170000012A4FEA93132FD0022A08D002B1F8BD64
:101710006F4B9842FBD9012384F87430F8BDA26F57
:1017200064329A423CD894F86D3004EB031393F87A
:101730008C20FF2A06D067490132012083F88C20D3
:1017400081F8DC00FFF7BAFF634B1B780122092BFD
:1017500084F87420DBD1B4F80E31604A01339BB2B7
:10176000A4F80E315380F8BD5D4D94F86D105A48C1
:10177000A3678C2303FB015300789A70002384F83D
:101780008A3004F180050A2202230928E56784F8DB
:101790008B2084F87430BAD1504B01311980F8BDD8
:1017A00094F88A2094F88B309A42B0D104F17F00EB
:1017B00004F18805002310F8012F082153405A0036
:1017C00013F0800F08BF5B0082F0070214BFD3B292
:1017D000DBB20139F3D18542EDD194F889209A42E8
:1017E00039D194F86D6094F8875094F88830B4F843
:1017F0008300B4F8852094F881C004EB061743EA0F
:10180000052394F8825087F88C1040BA52BA81B2FE
:1018100092B245EA0C202F4DC7F890101BB294F9F4
:101820008010C7F89420032E4FF00102A7F88E0015
:10183000A7F8983087F88D1085F8DC2008D8264A5C
:1018400012780C2A29D00D2A02D1244B23F8161025
:10185000FFF734FF5FE794F86D3004EB031393F860
:101860008C20FF2A06D01B490132012083F88C20EE
:1018700081F8DC00FFF722FF174B1B780122092BB0
:1018800084F874207FF443AFB4F80C31134A013369
:101890009BB2A4F80C319380F8BD1249124A897E9C
:1018A0000E4803EB830303EB830349089B0093FB80
:1018B000F1F382FB0312DB17C3EBA20320F816300F
:1018C000C6E700BF60A900205C090010D34D62107C
:1018D0003F4B4C0054040020892800208C28002015
:1018E0004440002024310020676666660A4B93F866
:1018F0008A1093F88B2091420DD010B493F88A206F
:10190000DC6F511CD2B2C0B2C9B283F88A10A054A5
:101910005DF8044B7047704760A90020FD2870B542
:1019200022D0F02804D0EF2822D00224204670BD17
:10193000114D0320052641282E444FF0000405F1E7
:10194000010580F080030DD0042B0BD9FFF7E6FFD3
:101950002044B542C4B2E9D015F8010B412880F00B
:101960008003F1D10420F3E7044D0B200426E2E7C5
:10197000034D0C200626DEE7ACC20608A8C2060806
:10198000B4C206080E4B0F4AD3F81031B2F9040066
:101990005B0707D400EB8000400080B200F5C87000
:1019A00080B27047084B094A9B6B323382FB0312AB
:1019B000D817C0EBA20080B200F5C87080B27047A3
:1019C00060A90020C40B00100C50002067666666FA
:1019D0000C4AD2F8283130B41C68D2F820515D602E
:1019E00019810025611C19609D812070D2F8283171
:1019F000D2F820111A685A604FF6F67230BC19609E
:101A00009A81704760A900200E4B30B4D3F8CC22E5
:101A1000C3F8D02203F5D67503F52F7403F596703D
:101A200003F5DE710132C3E94954C3E96B0030BCF0
:101A3000C3E9AF11C3F8CC22C3F81C01C3F82011CD
:101A4000704700BF60A9002000B583B00268084B52
:101A50008188CDF801203222D3F8D432ADF80510B8
:101A60008DF800206846984703B05DF804FB00BF7E
:101A700060A900205E2810B511D05D2805D00D4B5F
:101A8000BDE81040D3F8D83218470A4CD4F8D83201
:101A90009847D4F8D8323D20BDE810401847054C8F
:101AA0005D20D4F8D8329847D4F8D8323E20BDE82B
:101AB0001040184760A9002070B5094E0546D6F8B9
:101AC000D8325E200C469847D6F8D8322846984738
:101AD000E0B2FFF7CFFFC4F30720BDE87040C9E7CD
:101AE00060A9002003682DE9F041002B3D4D3E4FD9
:101AF0003E4EB8BF5B42A5FB0321890D07FB0137B2
:101B0000C7EB0717BF0096F8E23285FB0725FA17E7
:101B10000446C2EBA555002B57D101EB810101EB27
:101B2000810105EB810109B2DFF8BC801320FFF7CA
:101B3000C3FF2F4908FB057581FB0531ED17C5EB88
:101B4000A11109B21B20FFF7B7FF2368254D002B19
:101B5000B4BF53214E212320FFF7AEFF636896F8F0
:101B6000E22283EAE376A6EBE376A5FB0631890D54
:101B700008FB0168C8EB08184FEA880885FB0835A0
:101B80004FEAE873C3EBA5552ABB01EB810101EBDA
:101B9000810105EB810109B21220FFF78DFF124B85
:101BA000134903FB058581FB0531ED17C5EBA11139
:101BB00009B21A20FFF780FF6368002BBDE8F041EF
:101BC000B4BF57214521222076E7C1EB011105EB77
:101BD000810109B2A8E7C1EB011105EB810109B24E
:101BE000DAE700BF6BCA5F6B806967FF60A90020FE
:101BF000D34D6210044BD3F8FC3230EA030314BF18
:101C000001200020704700BF60A90020024803693E
:101C100003B11847704700BFC85B002030B40023F1
:101C2000022515244FF4167140F2D93205808471D3
:101C3000018130BC42814380838083817047134B94
:101C400010B400220F2483F80213090A83F8010359
:101C500083F80313C3F80423C3F80823C3F80C2341
:101C600083F8004303F54070012110F8014F013162
:101C700022440E29D2B2F8D183F80E230449D3F8B6
:101C800010035DF8044B102237F0AABF60A90020B2
:101C900060AC0020054B002183F81413C3F818131F
:101CA000D3F8103303B1CAE7704700BF60A9002022
:101CB00013B50446FFF734FC08B300230DF1060208
:101CC0002046ADF806300DF04BFCC0B10D4C9DF830
:101CD000062094F9CC1084F8E120032908BF62F0B3
:101CE0007F024FF00501084808BF84F8E120FFF7A4
:101CF0007FFC062184F8E2000348FFF761FC02B094
:101D000010BD00BF540400203105002008B5044B6D
:101D1000D3F81C0337F094FFB0FA80F0400908BDF7
:101D200060A900202DE9F84F1B4C05461E2094F8B1
:101D300020A394F821B394F82263B4F82493B4F860
:101D4000268394F8287322F07BFA30B1B8F1000FA3
:101D500003D0C14601264FF0000A94F82A33DA076F
:101D60000AD494F82F233AB9012F12D0022F03D1AD
:101D700013F0020F08BF012685F800A085F801B016
:101D8000AE70A5F80490A5F806802F722846BDE82D
:101D9000F88F3E46F0E700BF60A900202DE9F84F1C
:101DA0002DED028BFFF7BCFB002844D0264B93F9A6
:101DB000CC0001283FDD93F8E340DFF894809FEDED
:101DC000238A0FF27C0BDBE900AB15468E1E02EB7B
:101DD00044094D4504D1BDEC028B2046BDE8F88F87
:101DE00038F8027B26F8027F07EE907AF8EEE77A61
:101DF00067EE887A17EE900A56F0A4F952465B46D1
:101E000056F0F8F941EC100B59F06AFA51EC100B4E
:101E100056F018FD0E2F80B20AD919303223B0FBCC
:101E2000F3F080B200EB800000EB8000400080B255
:101E300025F8020BCDE70024CDE700BFAFF300800B
:101E40001655B5BBB16B024054040020CDCCCC3D3F
:101E5000B4AC002038B50D46FFF762FB044638B13C
:101E60000C4890F8CF30DB0704D5B0F8D0002880BC
:101E7000204638BD084A90F9CD3092F82C2093FBCB
:101E8000F2F102FB113201320131E4300DF07CFB42
:101E9000EDE700BF5404002060A9002038B5134CC2
:101EA00094F8313094F830209A4219D004EBC303EF
:101EB0000F49D3E90D200023984212DC93780D4A94
:101EC000C4F864035B081370FCF726FB94F8313008
:101ED00006210133B3FBF1F201FB123384F83130F8
:101EE00038BDD55C01F8015B0133E5E760A900204E
:101EF000945F0020C25F0020A1F5AF53B3F5AF7F20
:101F000070B541D8214BD3F86803A3F86A10B0B973
:101F10004FF47A744C434FF4C8714BF03FFA2823C6
:101F2000B4FBF3F303F03F034FF420610120B4FB53
:101F3000F1F1BDE8704043EAC1114BF02FBA144CE7
:101F40004068A1FB0445802155F024F943F210209C
:101F50004BF084FA0A2037F05DF80E4A0023204641
:101F6000294656F0DFFCC0F30510460129462046FD
:101F7000094A002356F0D6FC46EA003040F0110032
:101F8000BDE870404BF06ABA70BD00BF60A9002088
:101F90000084D71740420F000000093D13B500230D
:101FA0000DF106020C46ADF806300DF0D9FA30B14D
:101FB000044B9DF8060083F86C404BF087FA02B0A2
:101FC00010BD00BF60A90020194B37B593F86820F9
:101FD00004461D4651B13AB9D3F86C03012283F887
:101FE000682008B13AF04AFE03B030BD002AFBD0A9
:101FF000D3F86C0383F8681008B13AF039FE4FF457
:10200000AF7037F025F995F96C1000230DF1060239
:102010002046ADF806300DF0A3FA9DF806004BF00F
:1020200055FAB5F86A102046FFF766FFDCE700BFF7
:1020300060A900202DE9F04FAB4B1B788BB0804698
:10204000002B40F0B980A94DD5F87063002E00F048
:10205000B380A74AD2F8E84004F0F021B1F1E02FB4
:1020600070D1C2F8E830D5F8742394426AD0049352
:102070000593ADF81830B5F8243395F820E3ADF8A2
:10208000143095F821C395F8283395F822B38DF8CC
:1020900018300DF1100A8DF810E08DF811C08DF890
:1020A00012B09AE8070007AB03C3924F1A80C4F33B
:1020B00042533B44C4F30342997CC5F874438E45B4
:1020C00002F1010201D1944508D030468DF81C1070
:1020D0008DF81D200DF058FAADF8200030460DF0B7
:1020E00009FD032804F0070937D0042838D0012857
:1020F0003AD14F44FB7D9B4501A9304618BF8DF86E
:102100001E300DF085FA48B1019BC4F3001103F0B5
:1021100001038B4202D030460DF08AFC0A2207A947
:10212000504659F084FB68B19DF81E30BDF81C2064
:1021300085F82233BDF82030A5F82023A5F82433F4
:1021400045F08AFB95F878A304AF95F87833032B14
:102150007CD8DFE803F00B3477A44F44FB7FCAE759
:102160004F4497F82730C6E70023C4E73946304686
:102170000DF054FA044658B107A8FFF7D3FD9DF8B7
:102180001E109DF810308B4260D030460DF053FC8D
:1021900095F87833013303F0030385F878330CB9ED
:1021A0009A45D2D195F82A33DB0700D524B133689C
:1021B00041461B68304698470BB0BDE8F08F01A838
:1021C000FFF7B0FD95F82A939DF8044009F0010946
:1021D000ECB1B9F1000F39D13A460DF103013046A7
:1021E0000DF086FA044688B307A8FFF79BFD9DF81B
:1021F0001C109DF803309DF81D208B4203D19DF8E3
:102200001030934222D030460DF020FCC0E7B9F1E7
:10221000000FBDD1394630460DF0FDF90446A8B196
:1022200007A8FFF77FFDBDF82010BDF810308B42E6
:102230000CD085F8799385F87A93336830469B699A
:102240009847A5E795F82A33D80701D500249FE7DA
:1022500007A930460DF0DCF904460028F6D01E2010
:1022600021F0EEFF95F87B3383428146EED085F86E
:102270007B0360B1B5F82633002BE7D1079BD90764
:10228000E4D4012130460DF0D3FB4C4680E7079B98
:10229000DA07DBD5014630460DF0CAFB78E7384651
:1022A000FFF740FD97E8070007AB03C31A809DF8CE
:1022B00010309BB10DF11D0207A930460DF018FA40
:1022C0000DF11E0130460DF0A9F90A2207A9384682
:1022D00059F0ADFA041E18BF012459E708A9304689
:1022E0000DF099F9ECE700BF4260002060A90020E2
:1022F00054040020A8C20608024B0146D3F87C0310
:1023000037F0A2BC60A900202DE9F041FD2984B07E
:10231000044600F0DE80F02900F0BD80EF2900F0D7
:1023200031814AB10346861803AD002003F8010B42
:102330009E4205F8010BF9D19A4B0B2003F10905D8
:1023400001E013F8010F814200F0C880AB42F8D1E0
:102350004B1E832B00F29380DFE813F0320139012A
:1023600043014E01BE018400580163016F019100D9
:1023700091007501750175018B018B018B016F0156
:102380009100910096019E019100910091009100B1
:1023900091009100910091009100910091009100B5
:1023A00091009100910091009100910091009100A5
:1023B0009100910091009100910091009100910095
:1023C0009100910091009100910091009100910085
:1023D000910091009100910091009100B401910051
:1023E0009100910091009100910091009100910065
:1023F0009100910091009100910091009100910055
:102400009100910091009100910091009100910044
:102410009100910091009100910091009100910034
:102420009100910091009100910091009100910024
:102430009100910091009100910091009100910014
:102440009100910091009100910091009100910004
:1024500091009100910091009100910091009100F4
:102460001F011F01504BB3F8AC13002900F0668127
:1024700001922DF031FF019A80B2ADF80C003AB113
:10248000224403AB13F8011B04F8011BA242F9D14B
:1024900004B0BDE8F081454F03214FF00508B84472
:1024A000002501370CE0FFF739FA0646601932467D
:1024B000FFF72AFF70194745C5B2E9D017F8011B8D
:1024C000412981F08003084601D0042BEBD8042673
:1024D000ECE7374F0B214FF00408E0E7324BD3F81D
:1024E000100180060CD4002AD2D0224403AB13F88A
:1024F000011B04F8011B9442F9D104B0BDE8F0813E
:1025000093F88003870742D52A4D287D052834BFDC
:1025100002260326142917D97C39C8B20628E2D826
:102520000629E0D801A050F821F000BF15270108C6
:1025300015270108FF260108E724010825270108BF
:102540001F2701082B2701080929CCD90A390A2994
:10255000C9D801A757F821F0E5260108312701085D
:10256000E7240108E7240108E7240108E72401081B
:10257000E7240108E7240108E7240108F7260108F9
:10258000152701080C4F0C214FF0060887E7094B6F
:102590000B29187DA7D10126CBE0084B5B6B039379
:1025A0006DE700BFD8C2060860A90020ACC20608CB
:1025B000A8C20608CC5E0020B4C206080C50002059
:1025C0000192FFF7DFF9019AADF80C0057E76B4B6A
:1025D000D3EDE77AFDEEE77A17EE903AADF80C30DE
:1025E0004DE7664B93F8E702B3F88413002840F0F8
:1025F000AB80ADF80C1042E76049B1F8843391F834
:102600008C13B3FBF1F3ADF80C3038E75B4D95F864
:102610002A33DE0700F19D80B5F8AC33ADF80C30FD
:102620002DE7564B5649B3F9D03381FB0301DB1735
:10263000C3EBA103ADF80C3021E7504BB3F8D23314
:10264000ADF80C301BE74F4BDFED4F6AD3ED027A4C
:102650000C39C9B203EB810393ED167A67EEA67AC3
:1026600067EE877AFDEEE77A17EE903AADF80C3018
:1026700005E7424B03EB4101B1F8AE3303EB8303B3
:102680005B00ADF80C30FAE63C4B93F82A3303F0CC
:102690000103ADF80C30F2E6384BB3F8C813CD05A2
:1026A0005ABFCB4303F00103032311F0440F18BFBB
:1026B000042311F0020F18BF072311F4806F18BF15
:1026C0000923ABE70192FFF75DF9304B019ADB6B11
:1026D00043EAC0400390D2E6284BD3F8BC33ADF8B0
:1026E0000C30CCE62B8A03EB830303EB83039B00C4
:1026F000ADF80C30F7E6EB89ADF80C30F3E6EB897A
:10270000234903EBC3039B00A1FB03135B09ADF853
:102710000C30E8E6B3F88233ADF80C30E3E66B68D2
:102720000393E0E62B680393DDE6AB680393DAE6F8
:10273000F6B28DF80C608DF80D00D4E6D3F8C40322
:1027400080F3100080B298E693F88C33B1FBF3F17C
:102750004FE7019221F084FFD5EDE77A019AFCEE74
:10276000E77A17EE903A9BB200287FF457AF0949F9
:10277000096811F0100F18BF00234FE760A900206F
:1027800067666666C40B001000007A440C50002097
:102790001F85EB51A85D002070B5214D95F8D4330D
:1027A000EA181C4692F8D8238AB11E4E09225C1CF6
:1027B000A6FB04135B0803EBC303E31AE918DCB2BE
:1027C00091F8D81309B1013AF1D185F8D4430268E0
:1027D0001549561C06600C2616700268561C0660C9
:1027E000002616700268561C066003EB430603EBD6
:1027F0008603147019440D223FF06AFB95F8D41338
:10280000084B4A1CA3FB02035B08294403EBC303E8
:102810000120D31A81F8D80385F8D43370BD00BFE6
:1028200060A90020398EE33844AD00202DE9F04145
:102830006A4ED6F8707384B0044638460D460DF0E3
:1028400059F986F8590457B10DF1090202A9384621
:102850000CF04EFF002840F0838096F859040023C6
:10286000ADF808308DF80A301A46431EDBB200215D
:10287000FF20FD2B8DF80C20ADF80E108DF80B000D
:1028800003D9002004B0BDE8F0819DF80830042B86
:1028900000F09D80052B00F09D80032B00F09C80B4
:1028A000022B00F09380012B08BF042100F08F80E1
:1028B0009DF809309DF80A10D6F87003013B0DF120
:1028C0000E028DF809300CF04BFE96F85934032BAC
:1028D0007AD0042B76D0012B64D0D6F85C24029BEE
:1028E0003F4F9A420DF108084FD023680D22591C22
:1028F00021601A7023680022591C21601A70236815
:102900009DF80820591C21601A7023689DF8092041
:10291000591C21601A7023689DF80C20591C2160F5
:102920001A7023689DF80A20591C21601A70BDF89E
:102930000E1020463FF014FB23689DF80B20591C15
:10294000216020461A700721FAF7B2FF98E80300C9
:1029500087E803000120C6F8645404B0BDE8F081A4
:1029600001A938460CF054FE00283FF476AF3846F3
:102970000DF10A010CF052FE00283FF46EAF019BEE
:1029800096F8590403F001026FE77A68D8F804302A
:102990009A42AAD1D6F86434124AEB1A93427FF6CF
:1029A00070AFA2E7104A9DF80A000121002304E05D
:1029B0000133082B91D012F8011F8142F8D38DF812
:1029C0000A308AE7094AEEE7094AECE703218DF865
:1029D00008106DE70121FAE70221F8E760A900205D
:1029E000BCAD002080841E00BFC20608CFC206080E
:1029F000C7C206082DE9F0412A4C2B4AD4F8BC3353
:102A0000B4F86874B4F8C46382FB0352DB17C3EBF9
:102A1000A2031FFA83F8474582B00D4603D1B4F8EC
:102A20006A34B34233D002680190511C34230160F0
:102A3000137002680023511C0160137041463FF07F
:102A40008FFA019831463FF08BFA019847F6FF71F3
:102A50003FF086FA019847F6FF713FF081FA01983E
:102A600047F6FF713FF07CFA019847F6FF713FF09F
:102A700077FA01980221FAF71BFF0120A4F8688475
:102A8000A4F86A64C4F86C5402B0BDE8F081D4F8CC
:102A90006C34064ACB1A9342C5D8002002B0BDE878
:102AA000F08100BF60A900206766666680841E0012
:102AB000026810B57F21541C046011700268002464
:102AC000511C01600E211470FAF7F2FE012010BDB6
:102AD0002DE9F04FC24B1B68804613F0800083B095
:102AE00000F07181BF4B93F8800310F0020000F0FA
:102AF0006A81DFF810B39BF81430052B40F268812F
:102B0000DBF80030B84D0093002BB8BF5B42A5FB4B
:102B10000342B648B649920D00FB0233C3EB0313E0
:102B20009B0085FB034502EB8202DC1702EB82026D
:102B3000C4EBA55400FB043304EB8204A4B281FB74
:102B40000321DB17C3EBA111BCB10025A94F2E4611
:102B5000A7FB0432D20802EB8203A4EB4303E8B2E2
:102B6000A4469BB280008340BCF1090F94B246EAB0
:102B7000030605F10105EBD8340489B2B9B100258B
:102B80009C4F2E46A7FB0132D20802EB8203A1EB39
:102B90004303E8B28C469BB280008340BCF1090F2E
:102BA00091B246EA030605F10105EBD83443DBF8A0
:102BB00004E08D4D8D4E8E498EEAEE70A0EBEE70E6
:102BC000A5FB0032920D06FB0200C0EB0010830053
:102BD00085FB035002EB8202DD1702EB8202C5EB9C
:102BE000A05506FB053305EB8205ADB281FB032141
:102BF000DB17C3EBA111C5B10020DFF8F8C1064611
:102C0000ACFB0532D20802EB8203A5EB4303C7B24B
:102C1000A9469BB2BF00BB40B9F1090F95B246EA85
:102C2000030600F10100EBD8350489B2C1B10020E0
:102C3000DFF8C0C10646ACFB0132D20802EB8203CA
:102C4000A1EB4303C7B289469BB2BF00BB40B9F1B9
:102C5000090F91B246EA030600F10100EBD83543B3
:102C6000DBF80830634A0193002B1846B8BF58427E
:102C7000A2FB0030604E6149030AA6FB0363DB0937
:102C800001FB03F1C1EBD00189B2B9B10026914635
:102C90003746A9FB0132D20802EB8203A1EB4303C2
:102CA000F0B28C469BB280008340BCF1090F91B218
:102CB00047EA030706F10106EBD8B9B2BBF810707A
:102CC000DFB10026DFF82CA1B446AAFB0732D208F8
:102CD00002EB8203A7EB43035FFA86F938469BB207
:102CE0004FEA890903FA09F3092897B24CEA030C61
:102CF00006F10106E9D81FFA8CF7BBF812303D4AFD
:102D0000A2FB0306F608632E28BF6326092B63D9AE
:102D1000002093468146ABFB0632D20802EB8203C9
:102D2000A6EB43035FFA80FAB4469BB24FEA8A0AE5
:102D300003FA0AF3BCF1090F96B249EA030900F15C
:102D40000100E8D85FFA89F9009B019A002BCCBFFB
:102D5000392338231616BEF1000F26F07F0635DD25
:102D6000274A3343964543F00206C8BF43F00606A0
:102D7000D8F800301622581CC8F800001A70D8F88D
:102D800000300022581CC8F800001A7040463FF07E
:102D9000E7F8214640463FF0CBF8294640463FF051
:102DA000C7F8404639463FF0DBF8D8F800305A1CE7
:102DB000C8F8002083F80090D8F800305A1CC8F8F2
:102DC000002001201E7003B0BDE8F08F1E43CFE746
:102DD000002003B0BDE8F08F4FF00009B4E700BF5A
:102DE000A85D002060A900206BCA5F6B806967FF47
:102DF000D34D6210CDCCCCCCC55A7C0AA086010044
:102E0000FFC99A3BCC5E00202DE9F047AB4B1B6815
:102E1000064613F0800084B000F09E80A84B93F823
:102E2000800310F0020000F09780A64F397D05293D
:102E300040F29780632900F292800024DFF898C264
:102E400089B22546ACFB0132D20802EB8203A1EB2A
:102E50004303E0B28E469BB280008340BEF1090F6F
:102E600091B245EA030504F10104EBD8EDB2BB6869
:102E7000954A82FB0312D917C1EB623189B200294E
:102E800000F018814FF0000CDFF84CE26446AEFB16
:102E90000132D20802EB8203A1EB43035FFA8CF00C
:102EA00088469BB280008340B8F1090F91B244EA92
:102EB00003040CF1010CEAD8E4B2FB8983494FF416
:102EC000F36707FB03F7A1FB0737C7F38F1742F23E
:102ED0000F739F4249D8CFB10020DFF8FCE1844650
:102EE000AEFB0732D20802EB8203A7EB4303C1B269
:102EF000B8469BB289008B40B8F1090F97B24CEAF3
:102F0000030C00F10100EBD81FFA8CF7704BD3E9EA
:102F1000002313433ED14FF0FF3833681722591C6A
:102F200031601A7033680022581C306039461A70BC
:102F300030463FF015F8414630463EF0F9FF336821
:102F40005A1C32601D7033685A1C326030461C7047
:102F50000621FAF7ADFC012004B0BDE8F087992501
:102F600085E7002004B0BDE8F0870021DFF868C1E4
:102F70000F46ACFB0302D20802EB8200A3EB400336
:102F80009BB28B400431102947EA030793B2F0D17A
:102F9000BFB2BBE701A844F01BF89DF80810002958
:102FA00000F08A804FF0000CDFF82CE1E046AEFB29
:102FB0000132D20802EB8203A1EB43035FFA8CF0EB
:102FC00089469BB280008340B9F1090F91B248EA6B
:102FD00003080CF1010CEAD84FEA08289DF8091003
:102FE000E1B10020DFF8F0E08446AEFB0132D20808
:102FF00002EB8203A1EB43035FFA80F98A469BB29E
:103000004FEA890903FA09F3BAF1090F91B24CEAC0
:10301000030C00F10100E8D848EA0C089DF80A10FA
:103020004FEA0828E1B10020DFF8ACE08446AEFBAF
:103030000132D20802EB8203A1EB43035FFA80F96D
:103040008A469BB24FEA890903FA09F3BAF1090FDC
:1030500091B24CEA030C00F10100E8D848EA0C08F0
:10306000BDF80C301B49632BA1FB03214FEA081864
:103070004FEA51117FF651AF0020DFF85CE0844643
:10308000AEFB0132D20802EB8203A1EB43035FFAED
:1030900080F98A469BB24FEA890903FA09F3BAF12B
:1030A000090F91B24CEA030C00F10100E8D848EA9C
:1030B0000C0832E70C4600E788468FE7A85D002041
:1030C00060A90020CC5E002089B5F814D34D6210B1
:1030D000D0AD00201F85EB51CDCCCCCC08B5A0F1F4
:1030E0000103B3FA83F302284FEA531301D01846C1
:1030F00008BD0F2021F01CF830B9064B93F82A3395
:1031000003F00103184608BDBDE808400F2021F078
:1031100097B800BF60A9002010B5084CE26D138974
:103120009907FCD513891B06F9D40A2035F072FFE4
:10313000206EBDE8104039F0A1BD00BF101C00207A
:10314000014B1B681B6A184798560020024B1868F1
:1031500008B183691847704798560020024B1868D9
:1031600008B14369184770479856002010B5074CBE
:10317000606D40B13AF032FD94F8513013B180F0F7
:103180000100C0B210BD012010BD00BF101C002006
:1031900030B40A490A480A78531CDBB20525042BCF
:1031A00000EBC20400F8325008BF00234FF4045271
:1031B0000B7062604FF0FF3030BC7047EC5F002056
:1031C000F05F0020037870B4FBB10446C0F1010643
:1031D000A31914F8015FDBB2002DF9D101335B00B4
:1031E000DCB2032513800C704D7004785CB10223AF
:1031F00000255A1CD2B2CC548D5410F8014F023322
:10320000DBB2002CF5D170BC704702242346E8E7FE
:103210000B0617D401EB810300EBC30310B400EBE2
:1032200081000124002283F8764383F8741383F825
:103230007523426D5DF8044B136843F400130020BE
:103240001360704701F07F0101EB810300EBC303C2
:10325000012200EB810083F81C1183F81E2183F802
:103260001D2182691368002B01DA43F0804343F487
:10327000001313600020704770B501F07F0505EB67
:10328000850400EBC404282101FB05010126C4F8D4
:1032900030310023C4E94A2284F81C5184F81D61AE
:1032A000C4F8343101F58E711DB9FDF79DFF002082
:1032B00070BDFEF70DF8002070BD00BF2249F8B5C3
:1032C000D1F878340F2B04D05A1CC1F87824002090
:1032D000F8BD1E4C25780023C1F87834002DF6D1B6
:1032E0001B4E1C4B3268B2F5006F17D01B689A4218
:1032F00027D017D9C2F50063402B15D9403B02F106
:103300004005C1F87C3401232370356092B240231C
:1033100011490A448121FFF7AFFFD8E71B683560E8
:103320007BB12A469B1AE7E74FF0000502EB030743
:10333000C1F87C540CBF02210121376092B2217088
:10334000E6E700232370C2E760A9002020290020BF
:10335000882400208C24002024290020AEE700BF10
:10336000F8B51D4C2378012B03D0022B09D0002087
:10337000F8BD01461948D0F87C3453B923700020B9
:10338000F8BD00231A468121FFF776FF0023237042
:10339000F5E7402B11D9124C2268403B02F1400561
:1033A000C0F87C34256092B240230E4C084622447B
:1033B0008121FFF761FF0020F8BD094D2A684FF019
:1033C000000603EB0207C0F87C6408BF02202F60F0
:1033D00092B208BF2070E8E72029002060A90020F1
:1033E000882400202429002038B5134602250A46E7
:1033F000C0E94E3380F811510021FFF73DFF002056
:1034000038BD00BF10B50C7814F0600413D0202C28
:103410000AD14B78023B092B18D8DFE803F01B21B7
:10342000171717171717272E22490122FFF7DCFF5E
:103430000024204610BD4B78062B24D00A2BF3D055
:103440001D4B8A78C3F88824204610BDFBF792F8FC
:103450000224EEE719490122FFF7C6FF0024E8E73E
:1034600017490122FFF7C0FF0024E2E74B88124A08
:103470001B0AC2F884340024DBE70F4B8A78C3F8B8
:1034800080240024D5E74B881B0A222B0CD0212B4B
:1034900004D021462246FFF7A7FFCAE7CA88094998
:1034A000092A28BF0922F6E7CA880749262A28BF21
:1034B0002622F0E7E8AD002060A90020E4AD00205E
:1034C000E0AD00207A0500204005002038B501EB72
:1034D000810400EBC4040D46002184F87453C4F841
:1034E0008C1384F87513C4F88833C4F88023C37828
:1034F0002821012B01FB050108BFEDB201F55D712B
:1035000008BFC4F884231DB9FDF76EFE002038BD46
:10351000FDF7DEFE002038BD144B9A6870B50446F6
:1035200062B1134A1B7B92F88C542B4316D0812135
:103530002046FFF76DFE022D09D070BD0C4B93F8AD
:103540008C5481212046FFF763FE022DF5D12046E1
:10355000064ABDE870401F230121B7E70121FFF7AC
:1035600057FE20468121BDE8704051E6CC5F002027
:1035700060A9002070B5094A094D1173094B136009
:103580000021044629700D238121FFF775FE204696
:10359000054ABDE870401F23012197E72C600020F9
:1035A0002060002055534253CC5F002010B5064BDD
:1035B000597B0446FAF7ECFF002800DB10BD2046DB
:1035C0000121BDE81040D5E7CC5F00202DE9F04196
:1035D000314D2C7834B1012C01D1FFF7E7FF0020E9
:1035E000BDE8F0812D4FDFF8D080B0F8B4337A68B1
:1035F000C8F804201F2BBA68C8F80820064606D170
:10360000274B3A689A4202D1797B01291AD9254A77
:1036100025491378052401F8334001EBC300013339
:10362000DBB2042B08BF00234FF4005113701F4B73
:1036300041600222304683F88C24FFF76DFF0020A2
:10364000BDE8F081BB7B013B0F2BE0D8FAF7A0FF70
:10365000002819DB2B78013B022BC0D9144B1988A9
:10366000B1B1BB68D8F8082088F80C408B4228BF5D
:103670000B46D11A0424C8F808100E4A2C703046A4
:103680008121FFF7F9FDAAE73046FFF745FFA6E7DE
:103690003046FFF76FFFA2E720600020CC5F0020DC
:1036A00055534243EC5F0020F05F002060A90020EA
:1036B000146000201C8300202C60002008B5084BFB
:1036C0001B78022B07D0033B012B02D80021FFF708
:1036D00051FF002008BDFFF769FF002008BD00BFB3
:1036E0002060002010B501EB8101084A00EBC10108
:1036F0000446B1F88C131046F4F77CFD034A2046CB
:1037000040230121FFF7E2FE002010BDF0AD0020B4
:10371000E8E700BF70B50A7812F060050C4606466F
:1037200011D0202D16D1CD88D5B113062AD52A4621
:103730001F496078F4F788FDE2881D493046FFF79D
:1037400053FE00250AE04B780A2B16D00B2B0ED027
:10375000062B03D13046FAF70DFF0225284670BD2F
:10376000022260781144F4F76FFD284670BD8B7813
:10377000D3B9104BC3F8D054F0E70F490122FFF73B
:1037800033FEEBE70D4964780A4AC1F8C8400321CB
:10379000C0E9E45542F8045B2B4680F81111002182
:1037A000FFF794FE0025D9E7FAF7E4FED6E700BF5D
:1037B00064A9002060A9002030AE0020540400203D
:1037C0000B7803F00303012B03D0022B04D000205D
:1037D00070478B881BB915E68B88832BFBD099E744
:1037E00010B50223044640228121FDF779FC2046D2
:1037F000022340220121FDF773FC8221204603238E
:103800000822FDF76DFC064B02229A80F4F76AFD50
:10381000044A204640230121FFF758FE002010BD36
:10382000A0010020F0AD002038B508220D46044666
:1038300003238321FDF754FC29462046FFF7D0FFE0
:10384000002038BD82B00023016801930B69019309
:103850000E4B03E00A690192013B13D0019A002A42
:10386000F8DA019A094B42F001020192019A0A61C9
:103870000A69019203E00A690192013B02D0019AB0
:10388000D207F8D4002002B0704700BF400D0300FB
:10389000436D064A1A61C278012A06D100F2CC5063
:1038A00058614FF0802219681A607047180008604C
:1038B00010B5002304220446194680F811211A4647
:1038C000FFF7DAFC2046FFF7E3FF002010BD00BF42
:1038D00010B5044629B990F81131032B0DD0002002
:1038E00010BDD0F8E4359B69002BF8D090F8122178
:1038F000032AF4D19847002010BDD0F89013D0F8D7
:103900007C33994214D9C078D4F880230128A1EBE4
:10391000030104BFD218C4F880238B4228BF0B4692
:10392000C4F890139BB220460021FFF7CFFDD6E7E5
:10393000D0F8E4351B691BB190F81221032A03D09B
:103940002046FFF7B5FFCAE79847F9E7F0B5012130
:1039500090F8D17590F8D36590F8CFC590F8CE5512
:1039600090F8D03590F8D22580F8111190F8CC1548
:1039700085B005EB0C2503EB072302EB062201F0D3
:103980001F06AFB292B290F8CD558DF808109BB2D9
:10399000012E0446ADF80A70ADF80C30ADF80E20DB
:1039A000C0F840218DF8095017D0022E1FD036B133
:1039B00001F08001FFF72CFC002005B0F0BD092DBF
:1039C0000FD8DFE815F0BF00AC000E00D5000E00E8
:1039D000EA0085000E007700540090F81221032AB7
:1039E0002FD02046FAF7C6FD002005B0F0BD01F04B
:1039F00060012029DAB234D0012D00F02081032D9E
:103A000000F00681002DD7D190F81211022900F0A4
:103A1000DF800329E5D11B0600F14B8102EB820216
:103A200000EBC20393F87633002B00F04D81BF4BBF
:103A30000122C3F8E424BE4920460222FFF7D4FC49
:103A4000BAE7DAB2012ACCD8D0F8E43502A99B68EB
:103A50009847BDF80E30002BAED12046FFF728FF67
:103A6000AAE7D0F8E43502A99B689847A4E7F9B221
:103A7000AE4D012985F8D414B3D890F81231022B39
:103A800000F02781032BACD1002900F0868190F84B
:103A900010110129E1D0D0F8E4355B68984795F81A
:103AA000D41484F810112046FDF788FA2046FFF759
:103AB000FFFE81E7012A94D190F81231022B00F029
:103AC0001781032B8DD100F58871FFF78DFC73E70B
:103AD0003D0A022DADF8062000F05081032D00F0C4
:103AE0000B81012D7FF47DAFD0F8EC3580781B6819
:103AF0000DF106019847BDF80620002A3FF45CAF9F
:103B0000BDF80E30002B3FF457AF9A4228BF1A463B
:103B100001462046ADF80620FFF766FC4CE790F81A
:103B20001231023B012B3FF65CAF012F7FF444AF13
:103B3000D0F8E43500229B68C0F8182102A920467D
:103B400098478AE790F81231023B012B3FF649AFC4
:103B5000764BD0F818210021C3F8DC1412B10222F0
:103B6000C3F8DC24734920460222FFF73DFC23E71B
:103B7000012F00F09880022F7FF41EAF13F0FF0F8B
:103B80007FF41AAF02691B0A023B5268032B00F252
:103B90001D81DFE803F0393531241A437FF421AF6A
:103BA00090F81231032B3FF41CAF036907F07F0537
:103BB00080F81451196867F30A120A431A60FFF774
:103BC00077FE002D00F0E580022384F81231F3E641
:103BD00051063FF4F1AE1146FFF71AFBECE6052360
:103BE00063F30612514B012184F816112046C3F8E5
:103BF000E024FFF75DFEDFE6042363F30612F1E73E
:103C0000032363F30612EDE7022363F30612E9E7E9
:103C100090F81231022BDBD0032B7FF4E2AE27B9F0
:103C2000550602D01146FFF7F3FAD4F8E43502A99D
:103C30009B68204698472046FFF73AFEBCE690F87E
:103C400012110229C4D003297FF4CBAE002F7FF4D8
:103C5000B3AE12F07F013FF400AF180600F1A78069
:103C600002EB820304EBC30304EB810083F8767359
:103C700083F8741383F87573282303FB0243416DA3
:103C800003F55D73DA780B68023A6FF35553012A36
:103C9000D4F8E42598BF43F080530B602046936826
:103CA00002A99847D9E6D0F8E435C0F818719B68A6
:103CB00044E702F07F0202EB820200EBC20393F8BA
:103CC0001E31002B7FF4B3AE184B0022C3F8E4245E
:103CD000B1E600293FF4C1AE0121032380F81011A1
:103CE00080F81231FDF76AF92046FFF7E1FD63E63F
:103CF0001149FFF779FB5FE6FDB2052D3FF671AE86
:103D0000DFE805F0342C241C0B03D0F8EC35807868
:103D10009B690DF106019847EDE6D0F8EC35807807
:103D20005B690DF106019847E5E600BF60A9002038
:103D300044AE00203CAE002038AE0020D0F8EC3578
:103D400080781B690DF106019847D4E6D0F8EC3570
:103D50008078DB680DF106019847CCE6D0F8EC35A9
:103D600080789B680DF106019847C4E6D0F8EC35E1
:103D700080785B680DF106019847BCE6D0F8E43521
:103D800080789B6A0DF1060198474570C4F8F005EC
:103D9000B1E6012384F812310EE60222D0F8E435B0
:103DA00080F8101180F812215B68984755E62822A8
:103DB00002FB014304EB810083F81E7183F81C11A0
:103DC00083F81D51816903F58E735BE7012363F36B
:103DD000061207E770B5044649B990F81131022B75
:103DE0001BD094F81631012B0DD0002070BDD0F8F7
:103DF000E4355B69002BF8D090F81221032AF4D146
:103E00009847002070BD2A4A2369D2F8E0245A60FE
:103E1000002384F81631002070BDD0F83831D0F876
:103E20002451AB4217D9C278012AD0F82821A3EB3C
:103E3000050308BF5219C0F8383108BFC0F828215F
:103E40009BB20021FFF718FA00231A4619462046B4
:103E5000FFF73CFBC5E7D0F83C31B3FBF5F605FBBB
:103E6000163666B99D420AD8D0F84021934206D250
:103E700033463246FFF700FAC4F84061E4E7D4F86D
:103E8000E435DB681BB194F81221032A0CD000231F
:103E9000052284F8112119461A462046FFF716FB21
:103EA0002046FFF7F5FC9CE720469847EFE700BF68
:103EB00060A9002082B000230193019A094B42F0CF
:103EC00010020192C168019A0A610A69019203E035
:103ED0000A690192013B02D0019AD206F8D400206F
:103EE00002B07047400D030082B000230193019A95
:103EF0000B4B42F020020192019A61F38A12019267
:103F0000C168019A0A610A69019203E00A69019293
:103F1000013B02D0019A9206F8D4002002B070470B
:103F2000400D0300F8B50B7813F060050C4606460B
:103F30001CD0202D17D14A78FE2A44D0FF2A3DD12B
:103F40004A88002A56D1CD88002D53D11B0651D462
:103F50003749384B0D70012183F88C14364A1F23E2
:103F6000FFF7B4FA00E000252846F8BD4B780A2B8D
:103F70004BD00B2B44D0012BF6D191F9043089881A
:103F8000002B47DBFFF796FF21792A4F3046FDF7DC
:103F900043F80223217940223046FDF7A1F897F833
:103FA0008C34022B3BD094F90420002ADCDA012B5C
:103FB000DAD030460121FFF7DDFAD5E70225FAF71E
:103FC000D9FA2846F8BD4D88A5B9CC88012C11D165
:103FD0001A060FD5194B1B689B6998471549C0B243
:103FE00081F8E80430B1224601F59D613046FFF7C3
:103FF000FBF9B9E730460225FAF7BCFA2846F8BDC6
:104000000C4B4A8883F8E924AEE70D490122FFF7FB
:10401000EBF9A9E701F07F01FFF766FFB4E730464F
:104020008121FFF7F5F8002387F88C349CE700BF67
:104030002060002060A90020CC5F002010600020DC
:1040400049AE002038B50446FDF71CF8204602238F
:1040500040228121FDF744F820460223402201211D
:10406000FDF73EF80C4B0D491B680D4A00250D70FD
:104070001B6882F88C54284698472046FFF71AFFA1
:1040800020460121FFF730FF064A20461F23012169
:10409000FFF71CFA284638BD106000202060002081
:1040A00060A90020CC5F0020012905D008B50321BC
:1040B000FFF71AFF002008BDFFF752B9104B70B48C
:1040C000DA684378017886780E4CD243C2F3022234
:1040D000C2F10405E8B283400F2040FA02F23240F8
:1040E000DBB2134360181B0101F01F0501224909CF
:1040F000DBB2AA4080F8003344F8212070BC70473E
:1041000000ED00E000E100E0C27802B1D6E70378FC
:1041100005485A09203203F01F03012101FA03F375
:1041200040F82230704700BF00E100E000B583B0E6
:1041300009238DF80730FDF783F98DF807009DF806
:104140000730012BF7D09DF8070003B05DF804FBA2
:1041500082B0064B002201920193019B03EB800089
:104160000190019B186802B0704700BF50280040C2
:1041700082B0064B002201920193019B03EB800069
:104180000190019B196002B0704700BF50280040A9
:104190000023C0E90033C0E90233C0E90433C0E9B9
:1041A0000633C0E90833C0E90A33C0E90C3383633E
:1041B000704700BF0B6870B4D1E90524CD682B436C
:1041C0001343D1E9072523431343D1E909422B4384
:1041D000D1E90D652343134304680B4A334322405E
:1041E0002B4313430360D1E90B3442690D6922F07C
:1041F000070223431343D1E90142436145608460D0
:1042000070BCC260704700BF3F801CF00268364936
:10421000002310B422F001022124884202600360CE
:1042200043608360C3600361446138D02F4B984280
:104230002ED02F4B98423CD02E4B984240D02E4B44
:10424000984232D02D4B984241D02D4B984246D0C7
:104250002C4B984217D02C4B98423CD02B4B984279
:1042600016D02B4B984224D02A4B984228D02A4B68
:1042700098421AD0294B984229D0294B98422ED0E7
:10428000284B984208D14FF03D5243F8AC2C03E044
:104290004FF4746243F8202C5DF8044B7047224BB6
:1042A0005DF8044B3D229A607047204A43F8642C25
:1042B000F2E74FF474125DF8044B43F8382C704762
:1042C0004FF074625DF8044B43F8502C7047184A65
:1042D00043F87C2CE0E73D2243F8082CDCE7154A44
:1042E00043F8942CD8E700BF1060024028600240D9
:1042F00040600240586002407060024088600240A6
:10430000A0600240B860024010640240286402408D
:104310004064024058640240706402408864024075
:10432000A0640240B8640240006002403D000020EA
:10433000400F002000003D200B88F0B433BB028CFE
:104340004C880E898B88C98822F001021204120C55
:104350000284058B028CADB225F0F30592B22B439B
:1043600022F00A0243EA061322439BB242F0010202
:1043700003830284038B23F00C031B041B0C0383B5
:10438000038B9BB21943F0BC01837047042B048C50
:104390002CD0082B4E888A880D89C98851D024F4E6
:1043A00080542404240C0484838B078C2C0344EA5B
:1043B000022440F6FF421A4045F6FF733B4043EAB1
:1043C000063322439BB292B243F480538283038428
:1043D000828B22F440621204120C8283838B9BB284
:1043E00043EA01239BB2F0BC8383704724F010049E
:1043F0002404240C4D880F898A88C9880484068B7C
:10440000038C12029BB242EA073423F0A00340F669
:10441000FF42324043EA051322439BB292B243F07B
:10442000100302830384028B22F440621204120CF4
:104430000283038B9BB243EA01239BB2F0BC03834C
:10444000704724F480742404240C0484848B038C2B
:10445000A4B29BB224F0F30423F42063224343EA82
:10446000062342EA05129BB243F4807392B2828320
:104470000384838B23F00C031B041B0C8383838B2B
:104480009BB21943F0BC8183704700BF214A038867
:1044900090429BB212D002F5806290420ED0B0F1F1
:1044A000804F0BD0A2F58032904207D002F5806297
:1044B000904203D002F58062904203D14A8823F0F3
:1044C00070031343144A904218D002F58062904260
:1044D00014D030B423F440730C894D6802F56C425B
:1044E0009BB2234390420C880380C56204850DD1A2
:1044F0008B7A0386012330BC8382704703800B884C
:104500004A68C2620385012383827047034B984245
:10451000EED0EFE700000140001000400004014031
:10452000024A536A23EA0000506270470038024092
:10453000024A136A23EA0000106270470038024002
:10454000484B98422ED0B0F1804F32D0464B984223
:1045500036D0464B98421ED0454B984237D0454BFB
:1045600098423BD0444B98423FD0444B98424BD06A
:10457000434B984240D0434B98424CD0424B9842D8
:1045800051D0424B984256D0414B98425AD0414B61
:1045900098425ED07047404A136A43F004031362A6
:1045A0000420C5E73C4A536A43F0010353620120EB
:1045B000B6E7394A136A43F0010313620120B7E7F3
:1045C000354A136A43F0020313620220B0E7324A0D
:1045D000136A43F0080313620820A9E72E4A136AFE
:1045E00043F0100313621020A2E72B4A136A43F032
:1045F0002003136220209BE7274A536A43F4803349
:1046000053624FF480308BE7234A536A43F002032E
:104610005362022084E7204A536A43F40033536212
:104620004FF400307CE71C4A536A43F48023536202
:104630004FF4802074E7184A136A43F04003136272
:10464000402075E7144A136A43F080031362802008
:104650006EE7114A136A43F4807313624FF480705B
:1046600066E700BF00000140000400400008004071
:10467000000C004000100040001400400004014005
:104680000040014000440140004801400018004043
:10469000001C00400020004000380240224A93687D
:1046A00003F00C03042B10B421D0082B22D01F4B95
:1046B00003601D4C1E4AA168C1F30311114491F817
:1046C0003811CB404360A168C1F38221114491F8B5
:1046D000381123FA01F18160A1685DF8044BC1F340
:1046E00042310A4492F83821D340C3607047114BDD
:1046F0000360DEE75468516852686302C2F38812AF
:104700004CBF0C4B094B01F03F01B3FBF1F303FB32
:1047100002F3054A5268C2F3014201325200B3FB70
:10472000F2F30360C5E700BF003802400024F40044
:104730005404002000127A002DE9F04700230F688E
:1047400001264FF0030C02E00133102B41D006FA92
:1047500003F232EA0704F7D1D0F800E05C000CFA6B
:1047600004F52EEA050EC0F800E091F80490D0F8A8
:1047700000A009FA04FE09F1FF394EEA0A0EB9F168
:10478000010FA846C0F800E06FEA050515D8D0F87B
:1047900008E005EA0E0585604D79D0F808E0A540EF
:1047A00045EA0E058560456825EA020242608A797D
:1047B00045689A4092B22A434260C26822EA0802DF
:1047C000C260CA79C568A24001332A43102BC26077
:1047D000BDD1BDE8F0870D4B93F82A23D20703D54E
:1047E000012283F8EA24704793F8EA2462B9D3F8E7
:1047F00070234AB193F82023104493F8212383F8BF
:104800002003114483F82113704700BF60A90020E2
:10481000044B93F90C00012806BF02221A730020F2
:10482000704700BF60A90020114AD2F8EC04A0B183
:10483000D2F8F0348BB188420DD88B4234BF0023BC
:1048400001239BB11369C2F8F41499421CBF1423CD
:1048500082F8F834DCE70023F3E7A1F59C53083B2A
:10486000B3F57A7F2CBF00230123EAE7704700BF2E
:1048700060A9002007B500230DF10602ADF806304F
:104880000AF06EFE60B1084BBDF80620998AA3F8C5
:10489000FA2491421CBF142283F8FC24FFF7B8FFCE
:1048A00003B05DF804FB00BF60A9002013B5044607
:1048B000262001911FF0C4FC019948B9054BD3F89B
:1048C00010332BB1204602B0BDE81040FDF7B7B958
:1048D00002B010BD60A90020B1FA81F14909492058
:1048E000E4E72DE9F341BE4C94F90C3001330D4659
:1048F00000F06681D4F81033002B00F0B38002275B
:1049000000264FF00108D4F8100335F099F900287B
:1049100000F0A880D4F8100335F08AF9D4F81833E1
:104920005A1C2344C4F8182383F8FD0494F8143364
:10493000012B09D0022B15D063B90F280CBF84F8C6
:104940001483C4F81833DEE7A0F17203012B06D9F3
:10495000762804D084F81463C4F81863D3E784F885
:104960001473D0E7102ACED19E490023012211F8FA
:10497000010F013203440E2ADBB2F8D194F80B2563
:1049800084F814639A42C4F81863BCD194F80C35C7
:10499000002BB8D194F8FE34732B59D0762B1BD052
:1049A000722B5FD194F8002594F8FF3494F90C1021
:1049B00053EA022356D0C4F8EC340029B4F8013588
:1049C000C4F8F0344EDC94F81A2501232373002A2E
:1049D00048D184F81A3545E094F8002594F8FF345E
:1049E00053EA02233ED0D4F8102594F8021594F827
:1049F0000605236193421CBF142284F8F82494F81E
:104A00000125C4F8103542EA0122B4F81415A28237
:104A100091421CBF142184F8FC1494F803156173AF
:104A200094F80415A17394F80515A4F8142541EA27
:104A30000021A4F81615D4F8F41409B9C4F8F43414
:104A4000B4F8FA340BB9A4F8FA240223237309E06A
:104A500094F8042594F8033543EA02231AB20BB103
:104A6000A4F8182594F90C30022B35D00FDCDAB2FB
:104A7000012A15D9636E13B1A369002B6CD15A4971
:104A80005A481F2202B0BDE8F04156F036BF032B52
:104A9000F0D1D4F81C35564AEB1A9342EADD13E004
:104AA000D4F81C255349AA1A8A42E3DD2BB9722097
:104AB000FDF7F0F8C4F81C55DCE7D4F820355A1C93
:104AC000D907C4F8202503D47620FDF7E3F8F1E7F1
:104AD0007320FDF7DFF8EDE7D4F8F414D1B194F8C2
:104AE000F834BBB12369994214D0637BDA0703D44D
:104AF00089B24620FFF7DAFE94F8F834013B84F8D7
:104B0000F83405F59225032305F578752373C4F869
:104B10001C55AFE7B4F8FA14A38A81B194F8FC24C9
:104B20006AB18B420BD0637BDB0702D45020FFF7C6
:104B3000BDFE94F8FC34013B84F8FC34E1E701222B
:104B40002273A4F8FA342269C4F8F424002384F808
:104B5000FC3484F8F8348DE7274DD4F870732A2399
:104B600085F848310DF1070220230DF10601384682
:104B700085F849310AF0BCFD30B19DF806109DF86A
:104B8000076051EA06031ED1552385F84A314623B2
:104B900085F84B3122691948202385F84C31002AC9
:104BA00034D0174946F046FEB4F8163515488BB395
:104BB000A28A15499A420CBF20222A2246F03AFEC8
:104BC00002B0BDE8F08138460AF010FD314685F8A4
:104BD0004A0138460AF0F6FC037885F84B31D9E7EC
:104BE00060A900205DAE0020EE6C07089C05002047
:104BF000400D030040420F0054040020A105002096
:104C000067A60708A5050020086D0708034946F0B8
:104C100011FEC9E7024946F00DFED1E7106D070805
:104C20000F6D070810B50E4C40F0080284F86B2198
:104C300094F9CC20022A06DD420704D583071CBF65
:104C4000012384F8D43005210648FCF7D1FC062165
:104C500084F86C01BDE810400248FCF7B1BC00BF0D
:104C600054040020BB05002010B5FCF759FCA8B384
:104C70001B4C94F9CC30012B30DD59B3022B2DD0D5
:104C800094F8D4309BB971B180230521154884F87C
:104C90007131FCF7ADFC062184F87201BDE81040CB
:104CA0001048FCF78DBCBDE810400420BAE700298D
:104CB00014BF0020042094F8CF301A0748BF40F0FA
:104CC00002005B0701D411B108B940F00100BDE852
:104CD0001040A7E7022BD3D10420ECE710BD00BFA2
:104CE00054040020C1050020F8B5224C04F27317CB
:104CF000030A84F8780105460621384684F877319E
:104D0000FCF776FC94F8CF3084F87901DB072AD4DD
:104D1000B4F8D020AA4226D1174DD4F87331C5F883
:104D20002435C3B285F82A3541F26F714FF6FF730F
:104D30008A4218BF0123134405F22456C3F3072205
:104D40000621304685F8282585F82935FCF750FCE2
:104D5000072185F82A053046FCF732FC052104F5C9
:104D6000BD70FCF72DFCBDE8F84004480721FCF7B6
:104D700027BC00BF5404002060A90020C705002004
:104D800008B5FCF7CDFB48B1A1F59C53083BB3F542
:104D90007A7F03D2BDE808400846A5E708BD2DE9A3
:104DA000F0476B4E3368002B3AD06A4D6A4C05F1E0
:104DB000CC07306834F044FF002833D1674B1988A2
:104DC00009291D4609D95F8864227A43B2FBF1F2B2
:104DD000452A40F3A4811880588094F86535012B4A
:104DE00000F0C881022B00F0E38133B95C48052153
:104DF000FCF7E6FB012384F865355A4B1D685A4BD6
:104E00001B78002B00F0DE81584B1B68EB1A782BC7
:104E100040F2D881D4F86403F9F77EFBC4F86855F2
:104E2000BDE8F087306834F003FF94F82B358046F6
:104E3000052BBED8DFE803F00309171D3745AA2864
:104E4000B7D1012384F82B35B3E7552803D10223CA
:104E500084F82B35ADE7414A9388013393800023D2
:104E600084F82B35A5E7032384F82C0584F82B352B
:104E70009FE7132884F82D05C4F8480507DD374A55
:104E8000D3880133D380002384F82B3591E718B9F8
:104E9000052384F82B358CE70023C4F84C35042314
:104EA00084F82B3585E7D4F84C35E218013382F8C5
:104EB0002E05D4F84825C4F84C3593427FF479AFD9
:104EC000E6E7D4F848352A4803F1020A4FFA8AF196
:104ED000FCF78EFB804594F82C9540F01781262036
:104EE0001FF0AEF9204B48B100221A701B4A5388BC
:104EF00001335380002384F82B355AE71A784A454A
:104F000019D100221A7009F1FF33102B00F2F98039
:104F1000DFE813F030008E008E00E1008E00F70015
:104F2000F700F7003000F700F700F700F700F70090
:104F3000F700F7003000B9F1090F02D0B9F1110FF5
:104F400001D1012ADDD0054A538901335381DAE7C3
:104F5000905F00205404002060A90020B45F00206E
:104F6000CE050020B0240020C25F0020C45F0020D6
:104F70008CAE0020BAF1060F5ADDB9F1010F06D050
:104F8000B9F1090F0CBF4FF002094FF0030994F873
:104F9000310594F8321594F8302594F92EE594F9FA
:104FA00030C594F82F3585F8CC9041EA002109B23C
:104FB000900785F8CDE085F8CFC0A5F8D01006D5CC
:104FC00012F00C0F14BF0122002285F8D420B9F191
:104FD000030F13D1BAF1090F2ADD94F93425082AF9
:104FE000A8BF082222EAE27285F8E320002043B23B
:104FF0009A4200F101005CDC94F83335D4F818A033
:10500000002002469BB2524590465ADB7D4B85F804
:10501000CE001B78232B0BD109EB89037A4A03EBD3
:1050200083030CEB83031380A2F802E09180D0800D
:10503000764977480A2256F0FAFB10B1002384F82B
:105040005A35724B3A681A607A685A603A891A81FE
:1050500094F85A3543BB95F8D43094F8202384F85B
:105060005C25002B14BF0223012384F85A3595F8E0
:10507000CF3094F8220384F8600513F001031CBFBD
:10508000B2FA82F35B0994F8212384F85D25D9B242
:10509000B4F8242384F85B15A4F85E2513B10AB193
:1050A000A4F8622584F864150FF0A2F90FF0A0F9B6
:1050B0001CE704EB4308234493F83635A8F854332F
:1050C00095E704EB48080132B8F81C8052B29845C5
:1050D00008BF104697E7BAF1040FA9DD94F82E2512
:1050E00094F82F3543EA022359041AB204D5C3F3C6
:1050F0000D03A5F8D2309BE7002AF8DBA5F8D030E5
:1051000096E7444A938901339381EFE619F0010F42
:105110007FF4F0AE3F4A138901331381EAE63E4B38
:10512000D3F88021B3F88411012A1AD141F2563202
:10513000914203D14FF0FF32C3F88021D3F8802190
:10514000306802EB820202EB820201EB420189B27B
:10515000A3F8841103681B69984700232B806B8098
:105160003BE60132EAD1B1F5965F04BF0122C3F8F4
:105170008021E3E7284D95F9CC60002E3FF43DAE49
:10518000022E11D14FF48040FFF7AEFD84F8656523
:1051900095F9CC30012B7FF730AE95F8CF30C3F3C3
:1051A000400385F8D43028E6032384F86535EFE71B
:1051B000194BB3F8D230002B3FF41FAE032384F811
:1051C00065351AE694F8302094F831309A4204D0CC
:1051D000FCF764FEC4F8685522E6D4F86835EB1A8B
:1051E000B3F57A7FBFF41CAE0C4B1B68ED1A952DFE
:1051F0007FF616AE0A480521FCF7E2F9BDE8F04754
:10520000FCF74CBE892800208C280020B0AE00207E
:1052100020050020B45F002054040020C45F00205B
:10522000CE05002010B5134CD4F8700300B394F8E9
:10523000201359B194F821230AF0A6F9B4F82433C5
:1052400083421ABFA4F8240301210021B4F82623C5
:1052500062B141F288339342B8BF13469A4205D0F7
:10526000A4F82633BDE8104042F0F6BA0029F9D17F
:1052700010BD00BF60A9002010B401440446002006
:1052800014F8013B08225840430010F0800F08BF7B
:10529000400083F0070314BFD8B2C0B2013AF3D183
:1052A0008C42EDD15DF8044B704700BF30B54FF430
:1052B000806085B02DF08CF940B3154C90F9040056
:1052C00094F86C35134A002B18BF08234FF4E131D2
:1052D0000125CDE90153009100234FF480612DF0A9
:1052E000D8F9FF232067003818BF012084F88C30DC
:1052F00084F89C3084F8AC3084F8BC3084F8CC302E
:1053000084F8DC3084F8EC3084F8FC3005B030BD33
:1053100060A90020ED180108374B1B6813F00063EB
:105320005CD02DE9F04F354B1F78B84251D3FF28A0
:1053300056D1334B93F8DC30002B47D0DFF8D4A0A4
:105340000022CAF87025CAF87425CAF87825AAF888
:105350007C25002F4CD00AF18C03104614461146D0
:105360001546164603EB071BB946B3F802C09F89E2
:1053700093F8008093F901E061443A444645D3E94B
:1053800001C738BF464610337545B8BF75469B45C3
:1053900009B212B264443844E7D191FBF9F192FBAF
:1053A000F9F28AF870658AF87155CAF87445CAF836
:1053B0007805144BAAF872151B781149AAF87C25B8
:1053C000092B4FF0000281F8DC200CD00E48BDE81C
:1053D000F08F0E4A02EB0010BDE8F08F18467047C0
:1053E0000020BDE8F08F0A4B9AF87025DA80EDE7CF
:1053F0003A463946DDE700BFA85D0020C40B001027
:105400005404002089280020D0AE0020ECA9002000
:105410008C28002060A900200268F8B53A4E3B4C69
:10542000B6F98035511C01607E2111700168054676
:1054300003EBC30384FB0302481CDC170023286032
:105440000B70FF20C4EB6204FFF766FF2034304B83
:10545000A4B200284DD01B78B0F90C102BBB2D4BFB
:10546000A1F57A729A4246D82B48B0FBF1F189B285
:1054700028463CF04FFD96F8E732B6F8841383B126
:1054800096F88C33B1FBF3F128463CF043FD2146FE
:1054900028463CF03FFD28460821F8F709FA01208C
:1054A000F8BD28463CF036FDF1E71C4B1F78002F75
:1054B000D5D01B48002300EB830201339289BB4205
:1054C0001144F8DB174B9FED186A9B7E07EE103AEC
:1054D00007EE901AB8EEC77AF8EE676AC6EE077A5A
:1054E00067EEA67AFCEEE77A17EE901AB1FBF7F1B9
:1054F000B5E71B7813B94EF69C21B9E7074B1F7827
:10550000002FF8D00146D4E760A9002067666666E0
:10551000600900101783930300879303C40B0010E6
:105520002C0C001024310020000048432DE9F843E2
:105530004A4C427894F8823502F00F05C3B9EDB9B0
:105540002B46002184F88415EB1AD9B20E290BD80A
:10555000234493F8E81239B102F0F002802A4AD0CD
:10556000902A5FD0A02A0DD000273846BDE8F883E6
:105570000021AB4284F88415F6D8E5E784F882551B
:105580002B46DEE7412966D081F08003042B62D9E7
:105590000846FCF7C3F9031D0246DBB2304884F825
:1055A000843565F05F0584F88555FCF7ADFE94F809
:1055B0008475002FD8D0BE1E16F0FF0024D1FF2521
:1055C000A946022756B1DFF89C80464418F8011B13
:1055D000D4F8A80534F038FB4645F7D1D4F8A8052F
:1055E000494634F031FBD4F8A805294634F02CFBA9
:1055F0003846BDE8F88365F07F050427022684F865
:10560000855584F884753046164A4FF6FF7110446C
:1056100012F8015B491B904289B2F9D15FFA81F916
:105620000D0ACFE7412914D081F08003042B10D953
:105630000846FCF773F965F06F050627042684F821
:10564000870584F8855584F8861584F88475304676
:10565000DAE70420EFE7082304229FE760A900208F
:10566000E6AE0020E4AE00202DE9F047C31DDFF8D0
:10567000348182B003F4FC7300AFD8F82861ADEB3D
:10568000030DC7F800D03268D8F8203168449A4238
:105690000C4698F8AC3578606D4658D0591C0DF121
:1056A000010203F00F0388F8AC158DF800303A6062
:1056B000A0EB0209D6E900125FFA89F9521A09F142
:1056C00007035FFA82FA03F4FC73CA45ADEB030DDE
:1056D00055D25246684656F071F8336853443360E9
:1056E0005246694638463CF0F3FBD8F82821D8F8F2
:1056F00020313068117A7060C21A4A40D2B28342B7
:10570000336088F8AD2509D00133336013F8011CEC
:10571000984282EA0102F7D188F8AD253B68591C0E
:1057200039601A70D7E90032D21A012A08DD002147
:105730005A1C3A601970D7E90032D21A012AF7DCF4
:105740002846A04700200837BD46BDE8F087B6F9D7
:105750000C20591C03F00F0343F01003002A2A46C3
:10576000B8BF43F0200302F8023B88F8AC15691C6F
:105770003960D6E900135B1A3A606B7098E74A46C5
:10578000684656F01BF833684B4433604A46694616
:1057900038463CF09DFB2846A04701200837BD460F
:1057A000BDE8F08760A900202DE9F04F7A4C83B066
:1057B000D4F82851D5E900535B1B002B00AF83467A
:1057C0000D46164628DD002384F8AE35FCF71CF99B
:1057D00000200BEB05030BF1010AC4E945A39BF87C
:1057E0000050D4F824816909012940F09D8005F01A
:1057F0000F0915F0100514D150B194F8B0250132FD
:1058000002F00F024A4500F0988084F8AE55284611
:105810000C37BD46BDE8F08F94F8AE050028D8D10E
:10582000D4E70BF10203C4F814310BF103029BF827
:105830000130D4F81C01C4F814219BF80250C8F8B8
:105840000000C218C8F804206B4084F8AF35D4E9D2
:1058500045A34FF0000C84F8AE15A8F80850A8F83E
:105860000CC0A3EB0A03DDB2121AEB1D5FFA82FB38
:1058700003F4FC73AB45ADEB030D6BD25A465146B6
:10588000684655F09BFF0AEB0B035A4640466946B3
:10589000C4F814313CF01CFBD4F81C31D8F80000DB
:1058A00094F8AF258342C8E900300AD00133C8F824
:1058B000003013F8011C984282EA0102F6D184F804
:1058C000AF25D4F814311B78934239D1B8F9083098
:1058D000FA2B54D0D8F80020D4F81C31D4F8241175
:1058E000D4F8D002C8E90032D4F82821D4F8203105
:1058F00053600025158195813B1D84F8AE557D6070
:105900002DF0D6FA01303FD07B680BB100209847CC
:10591000D4F82831D4F82021196801200C37C3E9C4
:105920000021BD46BDE8F08F00210846FCF750F885
:1059300001200C37BD46BDE8F08FD8E9000290E7A2
:1059400000230120B8F9081084F8AE35FCF740F8C0
:1059500001205DE72A465146684655F02FFF0AEBC5
:10596000050340462A466946C4F814313CF0B0FAB3
:1059700000200C3784F8B095BD46BDE8F08F002EAE
:10598000A8D005233370A5E7D4F828211368022195
:10599000581C10601970B7E760A900200B4B93F8F2
:1059A000AA2312B1B3F8F8224AB9B3F9D033084A9E
:1059B000D81782FB0323C0EBA30000B27047D3F8D3
:1059C000C40390FBF2F000B2704700BF60A9002052
:1059D00067666666F8B5184CC6B205463146D4F817
:1059E000B40534F031F994F8B815D4F8B405C5F31A
:1059F00007274E40394684F8B86534F025F994F805
:105A0000B815D4F8B405C5F307464F40314684F8BD
:105A1000B87534F019F994F8B815D4F8B4052D0E0A
:105A20004E40294684F8B86534F00EF994F8B8155C
:105A30004D4084F8B855F8BD60A9002070B50C4DF4
:105A4000C6B231460446D5F8B40534F0FDF895F8F1
:105A5000B815D5F8B405240A4E40214685F8B86536
:105A600034F0F2F895F8B8154C4085F8B84570BD9B
:105A700060A9002038B50B4C002305462421D4F83A
:105A8000B40584F8B83534F0DFF8D4F8B4055421FF
:105A900034F0DAF8D4F8B4052946BDE8384034F0DB
:105AA000D3B800BF60A900202DE9F047DFF858A364
:105AB0002DED028B9AF8B94582B00F461646002CA0
:105AC00000F0E781013C8AF8B945DFF840839FED9B
:105AD000C88ADFF83C933B78002B00F090809AF85E
:105AE000B945002C40F08B8036B133F033FB33687E
:105AF000C01A002880F2DB839AF8BA15002940F01A
:105B00007A839AF8BB55062D40F28481B94B93F8FD
:105B10008D0193F88C21824200F0AB81D3F888216B
:105B20009AF8BC1532F810400C440135013003F5E9
:105B3000C473A4B2EDB2C0B2B4F5C06F8AF8BB555D
:105B4000587100F07E817CD8B4F5806F00F0298216
:105B500024D8B4F5067F4FD8B4F5007F54D3A4F50C
:105B60000073182B48D8DFE813F0E701DE01DE01EF
:105B7000DE01DE01DE01DE01DE01DE01470047005D
:105B800047004700470047004700C601AB01AB0193
:105B9000AB01AB01AB01AB01AB01AB01B4F5846F61
:105BA00000F0E68140F2E280B4F5A06F00F064827C
:105BB0006FF4A06C04EB0C03072B1DD8601EC0B261
:105BC000FFF7AAFBC0B1B0F90C308B4AADF8014029
:105BD000917EDAF8D42203EB830303EB83034908B5
:105BE0009B0093FBF1F31021CDF803308DF80010EA
:105BF0006846904700233B70002E7FF46CAF02B0E4
:105C0000BDEC028BBDE8F087B4F5807F00F0FD812C
:105C1000B4F5887FF0D1BAF9D233CDF80330012240
:105C200010238DF800308DF801308DF80220DAF85D
:105C3000D4326846002498473C70002E7FF44BAF66
:105C4000DDE7B4F5046F00F0A48265D8B4F5006F09
:105C500000F082821AD9B4F5026F00F0F181B4F538
:105C6000036FC9D19AF880339D07C5D5634BDAF825
:105C7000D422D9894FF4F36303FB01F3A8FB031388
:105C80005B091020CDF8033030218DE2B4F5E26FCE
:105C900000F03782B4F5E46F1FD1594B93ED180A29
:105CA000D3ED027A20EE270A002420EE080A53F0F2
:105CB000B9FF102320228DF800300723CDF8030010
:105CC0008DF802308DF80120DAF8D4326846984712
:105CD0003C70002E7FF4FFAE91E7B4F5E06F8BD1FE
:105CE000474B93ED160AD3ED027A20EE270A0024E3
:105CF00020EE080A53F096FF10220723CDF8030088
:105D00008DF802308DF80020DAF8D4328DF8014099
:105D1000684698473C70DCE740F678339C4248D8A8
:105D2000B4F5376F00F2E281B4F5116F00F08081B5
:105D3000B4F5376F7FF460AFFF20FFF7EDFA00286E
:105D40003FF45AAF90F90130CDF8033010217022A2
:105D50000B238DF802308DF80010DAF8D4328DF86C
:105D600001206846002498473C7066E740F20143F2
:105D70009C4200F02882B4F5826F7FF43DAFDAF8E0
:105D80001031980600F146821E4B1B681B0640F13D
:105D900094820024102304228DF800308DF8013005
:105DA0008DF803408DF804408DF805408DF80640CD
:105DB000BBE145F230239C4200F0848145F2402350
:105DC0009C427FF419AFBAF9CC33CDF803301021DF
:105DD000402252238DF802308DF80010DAF8D432C8
:105DE0008DF801206846002498473C7025E700BFE5
:105DF0000000C8425404002024310020CC5E002062
:105E0000C40B0010A85D002060A900201F85EB5185
:105E1000C5B3A2910135CA4BEDB293F8952193F821
:105E20009411914220D0501CC0B25200D3F890116E
:105E3000C44B8C5A8AF8BB55B4F5C06F58717FF4C7
:105E400082AEDAF8C433CDF80330102200240623E2
:105E50008DF802308DF80020DAF8D4328DF8014048
:105E6000684698473C7034E7002283F8952101206A
:105E7000DCE7B5489AF8BC25007883F88D1101322B
:105E8000D2B2013082428AF8BC2500F0B0810125EF
:105E9000C3E700283FF419AE0378303B012B3FF6EF
:105EA00014AE01300AF2B9520621FFF77DFC9AF8D0
:105EB000B9358AF8BA05002B3FF407AE3C7004E60A
:105EC000A4F11100C0B2FFF727FA00283FF494AE06
:105ED000B0F90230CDF8033010238DF80030ADF862
:105EE0000140DAF8D4326846984700233B70002E10
:105EF0007FF4F1AD83E69AF8E722BAF88433002AFA
:105F000040F0CF8110220221CDF803308DF800201F
:105F1000DAF8D4328DF801208DF80210684600249A
:105F200098473C7089E6601EC0B2FFF7F5F900287B
:105F30003FF462AE4368CDE7DAF8BC338349DAF860
:105F4000D42281FB0301DB17C3EBA1030024102142
:105F5000CDF8033002238DF800108DF801408DF844
:105F60000230684690473C70002E7FF4B4AD46E6A0
:105F70009AF880339A077FF53FAEBAF88233CDF8AE
:105F800003301021202204238DF802308DF80010F8
:105F9000DAF8D4328DF801206846002498473C7026
:105FA0004BE69AF8C4350133DAB2042A00F06E8168
:105FB00042F210738AF8C42503FB02F3DAF8C8250D
:105FC000002A00F0258102339AF82A23D507BAF86F
:105FD000C82348BF0433D40748BF0A33900748BFDB
:105FE0001433D10548BF2833550748BF64335406DE
:105FF00048BF03F57A63102100240422CDF8033052
:106000008DF800108DF801408FE0DAF8C035CDF83A
:1060100003301022002401238DF802308DF8002077
:10602000DAF8D4328DF80140684698473C7050E663
:106030009AF88C33002B40F02F811022092163E75E
:106040009AF880339B077FF5D7AD414ADAF8D4320E
:106050009268CDF80320102220218DF8002008221C
:106060008DF801108DF802206846002498473C7096
:10607000002E7FF430ADC2E5FF20FFF74DF9002878
:106080003FF4BAADB0F90C303249DAF8D422897E47
:1060900003EB830303EB83031020490800249B00D8
:1060A00093FBF1F305218DF80000CDF803308DF856
:1060B00001408DF80210684690473C70002E7FF436
:1060C0000AAD9CE5BAF9CE33CDF803301021302269
:1060D00052238DF802308DF80010DAF8D4328DF8A2
:1060E00001206846002498473C70A6E5A4F17100A1
:1060F000C0B2FFF711F900283FF47EAD90F90130EE
:10610000E8E6114B93ED170AD3ED027A20EE270A49
:10611000002420EE080A53F085FD1023CDF803007B
:1061200007228DF800308DF80130DAF8D4328DF87E
:106130000220684698473C70002E7FF4CCAC5EE5A8
:1061400054040020E4050020C40B00106766666656
:10615000CC5E0020243100209AF880339C077FF524
:106160004BADC107814B40F1B5805A6882EAE273BA
:10617000A3EBE27303EB5303A8FB0313DB08002A32
:10618000ACBF43F0004343F04043102100240822F9
:1061900034E7BAF9D033DAF8D42203EB83035B0097
:1061A0001020CDF80330402108238DF800008DF831
:1061B00001108DF802306846002490473C70002E94
:1061C0007FF489AC1BE5BAF98035CDF80330102196
:1061D000012204238DF802308DF80010DAF8D43251
:1061E0008DF801206846002498473C7025E58AF820
:1061F000BC15012511E65E490620FFF735FA00239C
:106200008AF8BA053B7002B0BDEC028BBDE8F0879E
:106210000133D9E6554A9AF88013538A643BC3EB9D
:106220004370C3EBC00389FB03401844DB17C3EB87
:1062300020230933092BA8BF092323EAE37303EBC7
:10624000830311F0020F03EB830314BF4FF47A7042
:1062500000209B00C90748BF00F5FA60117DDAF8FD
:10626000D4229BB203440B44042010218DF8020079
:10627000CDF803308DF800108DF801106846002429
:1062800090473C70002E7FF426ACB8E401238AF8D6
:10629000C43542F2107391E6BAF88423B2FBF3F3EB
:1062A000CBE69AF88C23002A57D113462AE63C7095
:1062B00002B0BDEC028BBDE8F0879AF8E632002B05
:1062C0003FF49AAC9AF8CC35032B49D8DFE803F0B9
:1062D0003B3122111A6882EAE273A3EBE27303EB0B
:1062E0005303A8FB0313DB08002AB8BF43F0804325
:1062F0004BE7DAF8D025537A907AD17A03F14073DC
:1063000003EB0023002203EB01438AF8CC25102283
:106310000421F9E5174A11688A7D087C897A1204FC
:1063200002EB00220A44591C8AF8CC1502EB0363E5
:10633000EDE7104A11684A7DC87B497A120402EBE6
:1063400000220A44EFE70B4A11680A7D887B097A2C
:10635000120402EB00220A44E5E7B3FBF2F3D1E5B5
:106360005A1C8AF8CC251B06D1E700BFCC5E002062
:10637000491A0108545F0020CA4A38B50820002392
:1063800082F89531FBF736FC002800F08C80D2F8BB
:1063900090314FF4806102204FF48264198082F8BA
:1063A000950101465C804FF40020FBF723FC50B1BF
:1063B0004B1CD2F89001DBB240F2014482F89531D7
:1063C00020F811401946B84C94F8A933002B6CD131
:1063D00094F8AA33002B40F088804FF40070FBF74C
:1063E00009FC50B14B1CD2F89001DBB24FF40465AC
:1063F00082F8953120F811501946D4F81041A507BC
:1064000000F10181600700F1DB80A84B1B681B06CF
:1064100000F1938000234FF4803082F8941182F8C9
:10642000953182F88D31FBF7E5FBD0B3D2F8883196
:1064300001214FF4047082F88D1118804FF4004050
:10644000FBF7D8FB50B14B1CD2F88801DBB24FF4FC
:10645000007482F88D3120F8114019464FF4003055
:10646000FBF7C8FB50B14B1CD2F88801DBB24FF4EC
:10647000A06482F88D3120F8114019464FF4802035
:10648000FBF7B8FB38B1D2F888014FF437644B1CE6
:1064900020F81140D9B2002382F88C1182F88D3196
:1064A00038BD0146CAE701467DE70120FBF7A2FBA4
:1064B00000288DD04FF48030FBF79CFBD2F8905130
:1064C00028B94FF4047325F811300131C9B20BB269
:1064D000481CC1B24FF4116082F8951125F81300E1
:1064E00094F8AA33002B3FF478AF0220FBF782FB2D
:1064F00000283FF472AF4FF40040FBF77BFB50B92C
:106500004B1CD2F89001DBB24FF4007582F8953144
:1065100020F8115019460420FBF76CFB00283FF4CB
:106520005CAF4B1CD2F89001DBB24FF4C06582F82F
:10653000953120F8115019464FE74FF40050FBF702
:1065400059FB50B14B1CD2F89001DBB24FF40364FD
:1065500082F8953120F8114019464FF48050FBF72E
:1065600049FB68B1D2F890014B1C4FF40064DBB2D8
:106570008D1C20F81140E9B282F8951120F81340E3
:106580004FF48040FBF736FB50B14B1CD2F8900122
:10659000DBB24FF4846482F8953120F8114019463B
:1065A0004FF48060FBF726FB00283FF433AFD2F8AE
:1065B00090014FF402644B1C20F81140D9B229E736
:1065C0004FF48060FBF716FB50B14B1CD2F89001E2
:1065D000DBB24FF4807482F8953120F811401946EF
:1065E0004FF40060FBF706FB00283FF40EAF4B1C96
:1065F000D2F89001DBB24FF4887482F8953120F81C
:106600001140194601E78020FBF7F4FA50B14B1C0A
:10661000D2F89001DBB245F2302582F8953120F8AE
:10662000115019464FF48070FBF7E4FA50B14B1C3F
:10663000D2F89001DBB245F2402582F8953120F87E
:10664000115019461020FBF7D5FA50B14B1CD2F867
:106650009001DBB24FF4E06582F8953120F81150DB
:1066600019462020FBF7C6FA50B14B1CD2F8900116
:10667000DBB24FF4E26582F8953120F811501946EB
:106680004020FBF7B7FA00283FF4BCAE4B1CD2F811
:106690009001DBB24FF4E46582F8953120F8115097
:1066A0001946AFE65404002060A90020A85D002030
:1066B00030B5A0F17D03012B044683B00D46104692
:1066C00008D9214633F0C0FA15B1288804442C803B
:1066D00003B030BD7D21019233F0B6FA019884F009
:1066E000200133F0B1FAEFE730B50F4B85B0D3F8A6
:1066F0001C2300230446C51DADF80E3014F8010B11
:1067000001920DF10E01FFF7D3FFA542019AF5D1D9
:106710000DF10E0014F0FAFD019A9DF80E00002113
:10672000FFF7C6FF05B030BD60A900207E28F8B590
:106730000F4652D0324E96F8984164B9314D95F8D3
:10674000DC1551B11B2885F8DC453DD00D2837D02C
:10675000012386F898310020F8BD7D284AD095F8AD
:10676000E0251AB180F0200085F8E01595F8DB25CA
:10677000062A14D8B5F8DE45511C2A440444C9B28F
:10678000A5F8DE4585F8DB1582F8D405002BE2D1AB
:106790000729E0D101231C4886F89831F8BDB5F8E7
:1067A000DE351844C0F3072353FA80F0FF284FF07A
:1067B0000103A5F8DE0586F89831CCD11248F8BD62
:1067C000A5F8DE452046F8BD90470028C0D001233B
:1067D00020463B7086F89831F8BD0A4B084A0024E1
:1067E000012183F8DB4583F8DC153C7082F8984181
:1067F0002046F8BD0123084685F8E035F8BD00BF06
:106800005404002060A9002034AF0020044AD2F8CC
:10681000E43543F4DF2343F48063C2F8E435704782
:1068200060A90020013070B5094EC4B203E045F004
:1068300037F8013448B9E5B2152D21463046F6D96E
:10684000162D04BF034B93F8E855284670BD00BFD2
:1068500044AF002060A9002000B1D7E7044AD2F875
:10686000E43523F4DF2323F48063C2F8E435704772
:1068700060A9002070B5114C84B00546D4F8EC0531
:106880000E462BF077FE94F8E02294F8E132003ABD
:1068900018BF01220BB142F00802CDE901620023CA
:1068A0004FF4964195F9000000911A4608212BF00B
:1068B000F0FEC4F8EC0504B070BD00BF60A9002074
:1068C00010B5064C03E0D4F8EC0533F0B1F9D4F878
:1068D000EC0533F0B5F90028F5D110BD60A9002012
:1068E00010B50D4CD4F8F0351B791E3B012B0DD99A
:1068F000D4F8EC0501213830FFF7BCFF0023C4F8C1
:10690000F43584F8F835BDE81040D9E7D4F8EC0543
:10691000012133F085F9F1E760A90020F0B5C64CFC
:1069200094F80036D4F81011C4F8FC050133880738
:1069300085B084F8003612D411F0340F34D1090731
:1069400094F8002641D412F007055AD0282A00F006
:10695000BA80D4F8D8325E20984705B0F0BD7020D8
:10696000FBF748F90028E7D0B44E2425A6F15807D4
:10697000F6EC017A97ED027A67EE877A2846FDEE0B
:10698000E77A013517EE901AC1EB411301EB830151
:10699000C90009B2EDB2FBF78FF8272DE8D1D4F882
:1069A000101111F0340FCAD04FF40060FBF722F938
:1069B000002840F0058194F8002612F0030100F051
:1069C000DB80D4F810110907BDD54FF40070FBF738
:1069D00011F90028B7D012F00305B4D1984AB4F9E0
:1069E000D033D91782FB0323C1EBA30109B21420D2
:1069F000FBF762F829461C20FBF75EF894F80026A6
:106A0000A1E7FF20FEF788FC002800F0DF80037874
:106A1000FF2B7AD090F901100220FBF74DF8FF20F0
:106A2000FEF77AFC002872D00378FF2B6FD0B0F904
:106A30000C20844B8248997E02EB820202EB820298
:106A40009300490893FBF1F3D91780FB0320C1EBB6
:106A5000A00001B20320FBF72FF894F8A933002B14
:106A60005DD1D4F810319A067AD54FF40050FBF777
:106A7000C1F8002840F0C980734D4FF48060FBF7E7
:106A8000B9F8002840F04C816B8A94F80026297DE3
:106A9000B3F5967F02D9100740F1118194F8E332E3
:106AA000002B40F0958009B20520FBF705F84FF464
:106AB0008050FBF79FF8002840F0D88094F800261B
:106AC000282A7FF446AF614A614B15686149A3FBF0
:106AD0000535AD09A1FB05367609A1FB063149094B
:106AE000C1EB0111A6EB81010902C6EB06160023DA
:106AF00009B21720A5EB860684F80036FAF7DCFF0A
:106B000031B21820FAF7D8FF23E7294684E700219D
:106B10000320FAF7D1FF94F8A933002BA1D001206C
:106B2000FBF768F8002840F00D8194F8AA33002B99
:106B300097D00220FBF75EF8002840F05C8104202B
:106B4000FBF758F800288CD0B4F8AC33002B00F0D9
:106B50005F8129F0C1FB01B20420FAF7ADFF80E7A5
:106B60001B07ABD53C4B93E8030002AB83E8030063
:106B70001846FAF7B7FFA1E74FF48060FBF73AF841
:106B800000283FF41EAF354BD4F8FC25D4F8C0558F
:106B90009A4240F20D81324BE91783FB0523C1EB8A
:106BA0006313642101FB13510DB219B21020FAF7DF
:106BB00083FF29462120FAF77FFF94F8002600E79B
:106BC000B4F9D2133020FAF777FFF4E6014623E751
:106BD000A1F1200307EE903A9FED227AF8EEE77AD2
:106BE000F6EE006A67EE877ABEEE007AF5EEC07ABE
:106BF000F1EE10FA58BFB0EE667A77EE877AFDEEC6
:106C0000E77A17EE903A19B24EE794F880339F076F
:106C10005BD44FF48060FAF7EDFF0B4D00283FF492
:106C200033AF002631460120FAF746FF31460920EE
:106C3000FAF742FF28E700BF60A900201C0C0010F3
:106C40006766666624310020CC5E0020B0240020F8
:106C5000D34D621089888888E4C206083F4B4C00F7
:106C60001F85EB51E4380E3F0050C34794F8802352
:106C700000239207CDE9003347D494F80436012B62
:106C800043D0B4F9DC325FED086A07EE103AB4F98C
:106C9000DE3207EE903AB8EEC77AF8EEE77A27EEE2
:106CA000267A67EEA67ABDEEC77AFDEEE77A02A8ED
:106CB0008DED027ACDED037AFAF714FFFEE642F28B
:106CC0000F719942A8BF1946E8E6544D544BE98923
:106CD0004FF4F36606FB01F14909A3FB0131C90931
:106CE0001120FAF7E9FEE9894E4B06FB01F1A3FBFF
:106CF00001214909A3FB01235B09642202FB131153
:106D000009B21920FAF7D8FEB7E6D5E90023012128
:106D10006846CDE9002384F80416FAF7E3FECDE6D1
:106D200094F880339E077FF57CAFAB683D4AD91756
:106D300082FB0302C1EB6211642606FB113636B2F8
:106D400009B270E794F88C1300293DD10B46062058
:106D5000A4F80236FAF7B0FEB4F802360133A4F80C
:106D6000023629F0ADFA94F8E43294F88C23012B22
:106D700094F8E7321ED000EB800086B213B10AB15E
:106D8000B6FBF2F6274BA3FB062343F34F113A2041
:106D90005D09FAF791FE642101FB1561224B89B26E
:106DA0000531A3FB0131C9083B20FAF785FEBCE69B
:106DB0000D46FBE61BB112B1B0FBF2F080B201B29E
:106DC0003920FAF779FEB0E6B4F80206B4F8842365
:106DD000B0FBF1F301FB1303642000FB02129BB232
:106DE0004900B2FBF1F2110241EA0311C2F303229E
:106DF000114309B2ABE7D4F8BC330C49DA1781FB75
:106E00000313C2EBA30319B22820FAF755FE96E646
:106E1000D4F8C43383F3100319B29DE6CC5E00208E
:106E2000C55A7C0A1F85EB51CDCCCCCC6766666613
:106E30000B2814D810B401EB4103094C01EB830378
:106E40002344184490F8E433934205D021440023AE
:106E500080F8E42381F8D8335DF8044B704770471D
:106E600060A90020F0B5454C94F80536012B83B09D
:106E700005464FD994F806064149424E94F80776E4
:106E8000421CA1FB02C1184406EB800001F4FE760F
:106E900006EB9101521A466C84F806262FB1D4F8FD
:106EA000081604F20C6291420DD06EB9364A0133D5
:106EB000A2FB031222F0010101EB52029B1A84F89B
:106EC000053603B0F0BD314E94F8203693B9304BFF
:106ED000019348F2A501123B15226F46A4F824162F
:106EE000009384F8262629463846B04758B994F8C6
:106EF0000536DBE76F46384611F078FD29463846FF
:106F0000B0470028F3D094F8201651B1384611F05C
:106F1000E7FCECE71B4A02EB8302566C002EC5D05F
:106F2000D2E7009E1B4A964214D9013A013E41F233
:106F3000210512F8013F81EA0321082311F4004FD3
:106F400085EA41000ABF490081B289B2013BF5D10F
:106F50009642EED138463BF003F80F49009D6D1A7A
:106F6000152DA8BF15252A4601F1180054F026FC5E
:106F700094F8053684F8515698E700BF60A90020C0
:106F8000CDCCCCCCA8C20608ABAAAAAA99270108E6
:106F900099AF002087AF002084AF002070B50B4E62
:106FA000054606F2566140F0BDFA2C686C6006F2A8
:106FB0005461641A402CA8BF40242960224606F27E
:106FC000946054F0FBFB86F8D44670BD60A90020A5
:106FD00030B50C4B0C4AC3F8542683B0C822014686
:106FE00003F2946503F2596483F8582668463A22FE
:106FF000CDE900453AF06CFF6846FFF7CFFF03B0DC
:1070000030BD00BF60A90020C83E7BEA03685A0675
:1070100007D513F4057F04D007298CBF0020012079
:10702000704703F48253B3F5825F03BFC81FB0FA01
:1070300080F040090020704770B5BC4C94F8D536FC
:10704000012B84B000F04C8194F8E106FCF746F87F
:1070500094F8E236834205461FD0002800F0D58020
:10706000D4F8F035CBB194F8E12293F90400002A6A
:1070700018BF08224FF4964100230325CDE90152A1
:1070800000911A4608212BF004FBC4F8EC0520B14E
:10709000FFF726FC012384F8E23694F8E336012B4F
:1070A00000F0C080D4F8EC663EB1A14B3046597870
:1070B000FFF7ACFF002840F0F18094F8F106FCF7F0
:1070C0000DF894F8F0368342054621D0002800F0F0
:1070D000F580EEB1337A002B00F01781954A02EB70
:1070E00083031B6E94F8E02296F904000093003AA3
:1070F00018BF012202210023CDE901121A461021F6
:107100002BF0C7FAC4F8B40510B1012384F8F036A7
:10711000D4F8F4663EB1864B30465978FFF776FFD7
:10712000002840F0AB8094F80007FBF7D7FF94F8F5
:10713000F8368342054622D0002800F0C880F6B118
:10714000337A002B00F0E4807A4A02EB83031B6E53
:1071500094F8E02296F904000093003A18BF012247
:1071600002210023CDE901121A464FF400712BF0E1
:1071700090FAC4F8FC0610B1012384F8F83694F8AC
:107180000107FBF7ABFF94F802378342054630D086
:1071900088B3694BD4F804674FF47A72C3F8AC260D
:1071A0003EB34FF48052402130462BF0FDF90546A6
:1071B000F8B994F8E03296F90400002B14BF0921C5
:1071C000082103224FF4E133CDE9012100932A463F
:1071D0002B464FF480512BF05CFAC4F8080740B1FD
:1071E0000123C4F8A80584F8825584F80C5784F864
:1071F000023704B070BDD4F808072BF0BBF9C4F80F
:10720000085784F8025704B070BDD4F8EC052BF091
:10721000B1F994F8E336C4F8EC55012B84F8E25642
:107220007FF440AF94F8E406FBF758FF05460028CA
:1072300071D0D4F81C33002B7FF434AFD4F8E82697
:10724000002A3FF42FAF94F8E15294F8E01292F93B
:107250000400002D14BF08220022002908BF42F0BC
:10726000010203254FF46141CDE9015200911A4614
:1072700020212BF00EFAC4F81C0313E794F8F8361B
:10728000002B7FF47CAFD4F8DC36002B3FF477AFD3
:107290000122C4F8FC3684F8F82670E794F8F0363A
:1072A000002B7FF435AFD4F8DC36002B3FF430AF41
:1072B0000122C4F8B43584F8F02629E7D4F8B405DF
:1072C0002BF058F9C4F8B45584F8F05620E7D4F8F8
:1072D000FC062BF04FF9C4F8FC5684F8F8564EE73C
:1072E000D4F8D856124B28465978FFF78FFE28B3AA
:1072F000D4F87C33002B7FF4A7AED4F8DC36002B17
:107300003FF4A2AEC4F87C339EE64FF49643E9E620
:107310004FF461431CE7D4F81C0300283FF4C2AECD
:107320002BF028F9C4F81C53BCE600BF60A900206C
:107330006C5A0020A8C206085404002094F8E00605
:10734000FBF7CCFE0646D8B1D4F87C33002B7FF493
:107350007BAE002D3FF478AE94F8E02295F904005E
:10736000B2FA82F252094FF416510225CDE90152C8
:1073700000911A4604212BF08CF9C4F87C0363E6D3
:10738000D4F87C0300283FF45FAE2BF0F3F8C4F888
:107390007C6359E670B5B14C94F8D536002B00F0FB
:1073A000218108202BF014F9C4F8F00500283BD007
:1073B00008212BF003F900260346A949A94884F8BF
:1073C000E136C4F8146736F00BFE41F2085301228F
:1073D000A448A4F8183784F81C270DF07DFF314627
:1073E0002B22A14854F04BFA48F67C607D25E0231F
:1073F00031462B22A4F824079C4884F8273784F8C8
:107400004F5754F03CFA48F67C21A0224EF27B0301
:1074100084F87B5784F87E6784F82758A4F85017BF
:1074200084F85327A4F87C3794F8E336002B00F057
:10743000C38010202BF0CCF81021C4F8EC062BF000
:10744000BDF88B4B84F8F1063A2140F23B1094F8DA
:10745000A92318809F254AF21E40197100219D71B1
:1074600098601973002A40F08E8094F8AA33002B9C
:1074700048D1D4F8103158077ED4990773D41A072D
:107480006AD47C4D2868C0F3C010FFF7E5F90020EE
:10749000FFF7C8F903464FF4007084F8E8352BF085
:1074A00097F84FF40071C4F8F4062BF087F8D4F87D
:1074B000283884F80007002B14BF0123002384F828
:1074C0002C3826D1D4F89C280023C4F89838002AF8
:1074D00069D0012284F8203684F8A0284FF4805027
:1074E0002BF076F84FF48051C4F804072BF066F8BF
:1074F000002384F8010784F80237FAF785FABDE81B
:10750000704099E5D4F8E43543F00403C4F8E43559
:10751000AFE7D4F81021002312F0020284F82D38CE
:1075200084F82E3840F0828094F8A93323B10120EA
:10753000FAF760FB002873D194F8AA33002B6AD1C4
:10754000A3182868042183F83018030602F101010A
:1075500075D484F83418B5E7D4F8E43543F480736F
:10756000C4F8E4358DE7D4F8E42542F4601242F023
:10757000C002C4F8E42582E7D4F8E42542F402729C
:10758000C4F8E42579E7D4F8E43594F8AA2343F065
:107590000201C4F8E415002A3FF46BAF43F0360350
:1075A000C4F8E43565E7D4F8A4387BB3012384F844
:1075B000A03884F8203691E720202BF009F8C4F891
:1075C000E80600283FF435AF20212AF0F7FF2A4BC8
